S01400005354345F52433030375F34302E73726563E7
S315080080000000022001BC020851BC020851BC02084B
S3150800801051BC020851BC020851BC0208000000000D
S3150800802000000000000000000000000051BC02082B
S3150800803051BC02080000000051BC020835BB02080A
S3150800804051BC020851BC020851BC020851BC0208C6
S3150800805051BC020851BC020851BC020851BC0208B6
S3150800806051BC020851BC020851BC020851BC0208A6
S3150800807051BC020851BC020851BC020851BC020896
S3150800808051BC020851BC020851BC020851BC020886
S3150800809051BC020851BC020851BC020841BB020887
S315080080A051BC020851BC020851BC020851BC020866
S315080080B0B9BB0208D1BB020851BC020851BC020870
S315080080C051BC020851BC020851BC020851BC020846
S315080080D051BC020885BB020851BC020851BC020803
S315080080E06DBB020851BC020851BC020851BC02080B
S315080080F051BC020851BC020851BC020851BC020816
S3150800810051BC0208F9BB020851BC020851BC02085E
S3150800811051BC020851BC020851BC020851BC0208F5
S3150800812051BC020851BC020895BB0208E9BB02080B
S3150800813051BC0208000000000000000051BC020803
S3150800814051BC020851BC020851BC020851BC0208C5
S3150800815051BC0208F1BB0208A9BB020851BC0208BF
S3150800816051BC020851BC020851BC020851BC0208A5
S3150800817051BC020851BC020851BC020800000000AC
S315080081800000000051BC02080000000000000000CA
S3150800819051BC0208000000000000000051BC0208A3
S315080081A000000000000000000000000051BC0208AA
S315080081B051BC020851BC020851BC020851BC020855
S309080081C051BC020896
S315080081D010B5054C237833B9044B13B10448AFF3F3
S315080081E000800123237010BD200A00200000000033
S315080081F01CF702080C4B43B10C480D4910B5AFF3F8
S3150800820000800C48036823B910BD0A48036833B9CF
S315080082107047094B002BF7D0BDE810401847064BAE
S31508008220002BF5D0184700BF000000001CF7020815
S31508008230240A0020200A00200000000081F00041E6
S3150800824002E000BF83F0004330B54FEA41044FEA2D
S31508008250430594EA050F08BF90EA020F1FBF54EAC8
S31508008260000C55EA020C7FEA645C7FEA655C00F064
S31508008270E2804FEA5454D4EB5555B8BF6D420CDD35
S315080082802C4480EA020281EA030382EA000083EAB8
S31508008290010180EA020281EA0303362D88BF30BD58
S315080082A011F0004F4FEA01314FF4801C4CEA1131AE
S315080082B002D0404261EB410113F0004F4FEA03330D
S315080082C04CEA133302D0524263EB430394EA050F98
S315080082D000F0A780A4F10104D5F1200E0DDB02FA07
S315080082E00EFC22FA05F2801841F1000103FA0EF29B
S315080082F0801843FA05F359410EE0A5F120050EF161
S31508008300200E012A03FA0EFC28BF4CF0020C43FA91
S3150800831005F3C01851EBE37101F0004507D54FF09E
S31508008320000EDCF1000C7EEB00006EEB0101B1F5EE
S31508008330801F1BD3B1F5001F0CD349085FEA300034
S315080083404FEA3C0C04F101044FEA445212F5800F3F
S3150800835080F09A80BCF1004F08BF5FEA500C50F1DC
S31508008360000041EB045141EA050130BD5FEA4C0CBF
S31508008370404141EB010111F4801FA4F10104E9D148
S3150800838091F0000F04BF01460020B1FA81F308BF3F
S315080083902033A3F10B03B3F120020CDA0C3208DD0B
S315080083A002F1140CC2F10C0201FA0CF021FA02F1E6
S315080083B00CE002F11402D8BFC2F1200C01FA02F156
S315080083C020FA0CFCDCBF41EA0C019040E41AA2BF7B
S315080083D001EB0451294330BD6FEA04041F3C1CDA43
S315080083E00C340EDC04F11404C4F1200220FA04F063
S315080083F001FA02F340EA030021FA04F345EA03010D
S3150800840030BDC4F10C04C4F1200220FA02F001FACE
S3150800841004F340EA0300294630BD21FA04F0294650
S3150800842030BD94F0000F83F4801306BF81F48011E9
S315080084300134013D4EE77FEA645C18BF7FEA655C5C
S3150800844029D094EA050F08BF90EA020F05D054EA2E
S31508008450000C04BF1946104630BD91EA030F1EBF33
S315080084600021002030BD5FEA545C05D14000494137
S3150800847028BF41F0004130BD14F580043CBF01F52A
S31508008480801130BD01F0004545F0FE4141F4700110
S315080084904FF0000030BD7FEA645C1ABF19461046EB
S315080084A07FEA655C1CBF0B46024650EA013406BFEC
S315080084B052EA033591EA030F41F4002130BD00BFAB
S315080084C090F0000F04BF0021704730B54FF4806468
S315080084D004F132044FF000054FF0000150E700BFE9
S315080084E090F0000F04BF0021704730B54FF4806448
S315080084F004F1320410F0004548BF40424FF0000135
S315080085003EE700BF42004FEAE2014FEA31014FEA77
S3150800851002701FBF12F07F4393F07F4F81F06051C6
S31508008520704792F0000F14BF93F07F4F704730B535
S315080085304FF4607401F0004521F0004120E700BFC8
S3150800854050EA010208BF704730B54FF000050AE04F
S3150800855050EA010208BF704730B511F0004502D550
S31508008560404261EB41014FF4806404F132045FEA52
S31508008570915C3FF4DCAE4FF003025FEADC0C18BFF7
S3150800858003325FEADC0C18BF033202EBDC02C2F1ED
S31508008590200300FA03FC20FA02F001FA03FE40EA7F
S315080085A00E0021FA02F11444C1E600BF70B54FF07F
S315080085B0FF0C4CF4E06C1CEA11541DBF1CEA135561
S315080085C094EA0C0F95EA0C0F00F0DEF82C4481EAC9
S315080085D0030621EA4C5123EA4C5350EA013518BFE9
S315080085E052EA033541F4801143F4801338D0A0FBD6
S315080085F002CE4FF00005E1FB02E506F00042E0FB83
S3150800860003E54FF00006E1FB03569CF0000F18BF88
S315080086104EF0010EA4F1FF04B6F5007F64F5407430
S3150800862004D25FEA4E0E6D4146EB060642EAC621C3
S3150800863041EA55514FEAC52040EA5E504FEACE2E30
S31508008640B4F1FD0C88BFBCF5E06F1ED8BEF1004F33
S3150800865008BF5FEA500E50F1000041EB045170BDAF
S3150800866006F0004646EA010140EA020081EA0301F3
S31508008670B4EB5C04C2BFD4EB0C0541EA045170BDEF
S3150800868041F480114FF0000E013C00F3AB8014F169
S31508008690360FDEBF002001F0004170BDC4F10004B2
S315080086A0203C35DA0C341BDC04F11404C4F1200533
S315080086B000FA05F320FA04F001FA05F240EA02008E
S315080086C001F0004221F0004110EBD37021FA04F6C4
S315080086D042EB06015EEA430E08BF20EAD37070BD7E
S315080086E0C4F10C04C4F1200500FA04F320FA05F0DD
S315080086F001FA04F240EA020001F0004110EBD370DF
S3150800870041F100015EEA430E08BF20EAD37070BD4E
S31508008710C4F1200500FA05F24EEA020E20FA04F327
S3150800872001FA05F243EA020321FA04F001F00041D6
S3150800873021FA04F220EA020000EBD3705EEA430E47
S3150800874008BF20EAD37070BD94F0000F0FD101F076
S315080087500046400041EB010111F4801F08BF013CAF
S31508008760F7D041EA060195F0000F18BF704703F0ED
S315080087700046520043EB030313F4801F08BF013D74
S31508008780F7D043EA0603704794EA0C0F0CEA135530
S3150800879018BF95EA0C0F0CD050EA410618BF52EAEA
S315080087A04306D1D181EA030101F000414FF00000F0
S315080087B070BD50EA410606BF1046194652EA4306FE
S315080087C019D094EA0C0F02D150EA013613D195EA72
S315080087D00C0F05D152EA03361CBF104619460AD1BA
S315080087E081EA030101F0004141F0FE4141F47001C4
S315080087F04FF0000070BD41F0FE4141F4780170BDB4
S3150800880070B54FF0FF0C4CF4E06C1CEA11541DBF18
S315080088101CEA135594EA0C0F95EA0C0F00F0A7F81A
S31508008820A4EB050481EA030E52EA03354FEA013147
S3150800883000F088804FEA03334FF0805545EA13135A
S3150800884043EA12634FEA022245EA111545EA106522
S315080088504FEA00260EF000419D4208BF964244F1B9
S31508008860FD0404F5407402D25B084FEA3202B61AD8
S3150800887065EB03055B084FEA32024FF480104FF4AC
S31508008880002CB6EB020E75EB030E22BFB61A754620
S3150800889040EA0C005B084FEA3202B6EB020E75EBB3
S315080088A0030E22BFB61A754640EA5C005B084FEA1B
S315080088B03202B6EB020E75EB030E22BFB61A7546E8
S315080088C040EA9C005B084FEA3202B6EB020E75EBF3
S315080088D0030E22BFB61A754640EADC0055EA060EB4
S315080088E018D04FEA051545EA16754FEA06164FEAF7
S315080088F0C30343EA52734FEAC2025FEA1C1CC0D1A3
S3150800890011F4801F0BD141EA00014FF000004FF02F
S31508008910004CB6E711F4801F04BF01430020B4F1F0
S31508008920FD0C88BFBCF5E06F3FF6AFAEB5EB030CA8
S3150800893004BFB6EB020C5FEA500C50F1000041EBA5
S31508008940045170BD0EF0004E4EEA113114EB5C0472
S31508008950C2BFD4EB0C0541EA045170BD41F4801145
S315080089604FF0000E013C90E645EA060E8DE60CEA4D
S31508008970135594EA0C0F08BF95EA0C0F3FF43BAF6A
S3150800898094EA0C0F0AD150EA01347FF434AF95EA21
S315080089900C0F7FF425AF104619462CE795EA0C0F05
S315080089A006D152EA03353FF4FDAE1046194622E7D2
S315080089B050EA410618BF52EA43067FF4C5AE50EAAC
S315080089C041047FF40DAF52EA43057FF4EBAE12E79C
S315080089D04FF0FF3C06E000BF4FF0010C02E000BF7D
S315080089E04FF0010C4DF804CD4FEA410C7FEA6C5C60
S315080089F04FEA430C18BF7FEA6C5C1BD001B050EA03
S31508008A00410C0CBF52EA430C91EA030F02BF90EAED
S31508008A10020F0020704710F1000F91EA030F58BFAC
S31508008A20994208BF90422CBFD8176FEAE37040F00E
S31508008A30010070474FEA410C7FEA6C5C02D150EAAC
S31508008A40013C07D14FEA430C7FEA6C5CD6D152EA67
S31508008A50033CD3D05DF8040B704700BF844610462C
S31508008A6062468C461946634600E000BF01B5FFF72B
S31508008A70B7FF002848BF10F1000F01BD4DF808EDFB
S31508008A80FFF7F4FF0CBF012000205DF808FB00BFCC
S31508008A904DF808EDFFF7EAFF34BF012000205DF826
S31508008AA008FB00BF4DF808EDFFF7E0FF94BF012073
S31508008AB000205DF808FB00BF4DF808EDFFF7CEFF74
S31508008AC094BF012000205DF808FB00BF4DF808EDB3
S31508008AD0FFF7C4FF34BF012000205DF808FB00BF84
S31508008AE04FEA410C7FEA6C5C02D150EA013C0AD19C
S31508008AF04FEA430C7FEA6C5C02D152EA033C02D18E
S31508008B004FF0000070474FF0010070474FEA4102EE
S31508008B1012F5001215D211D56FF47873B3EB6252C1
S31508008B2012D94FEAC12343F0004343EA505311F0E8
S31508008B30004F23FA02F018BF404270474FF000007A
S31508008B40704750EA013005D111F0004008BF6FF0B8
S31508008B50004070474FF00000704700BF4A0011D22E
S31508008B6012F5001211D20DD56FF47873B3EB625279
S31508008B700ED44FEAC12343F0004343EA505323FA85
S31508008B8002F070474FF00000704750EA013002D1FA
S31508008B904FF0FF3070474FF0000070474FEA410230
S31508008BA0B2F1E04324BFB3F5001CDCF1FE5C0DD93D
S31508008BB001F0004C4FEAC0024CEA5070B2F1004F87
S31508008BC040EB830008BF20F00100704711F0804F8A
S31508008BD021D113F13872BCBF01F00040704741F44F
S31508008BE080114FEA5252C2F11802C2F1200C10FA53
S31508008BF00CF320FA02F018BF40F001004FEAC12337
S31508008C004FEAD32303FA0CFC40EA0C0023FA02F3DA
S31508008C104FEA4303CCE77FEA625307D150EA0133B0
S31508008C201EBF4FF0FE4040F44000704701F0004080
S31508008C3040F0FE4040F40000704700BF034613F8BA
S31508008C40012B002AFBD1181A0138704700000000D2
S31508008C5001F0FF01102A2BDB10F0070F08D010F8DF
S31508008C60013B013A8B422DD010F0070F42B3F6D1E3
S31508008C70F0B441EA012141EA014122F007047FF0FC
S31508008C8000070023F0E80256083C85EA010586EA53
S31508008C90010685FA47F5A3FA87F586FA47F6A5FA8F
S31508008CA087F68EB9EED1F0BC01F0FF0102F007029B
S31508008CB032B110F8013B013A83EA010313B1F8D146
S31508008CC00020704701387047002D06BF3546033827
S31508008CD0073815F0010F07D1013015F4807F02BF60
S31508008CE0013015F4C03F0130F0BC0138704700BFB1
S31508008CF070470120704790F85000704790F8790047
S31508008D007047E02914BF00200120704740F65C2315
S31508008D10994209D043690BB9038BD3B140F24C533E
S31508008D20994208D00020704742F2E810824214BFE8
S31508008D30002001207047B2F51A7F0CD040F22F436D
S31508008D409A420AD040F2D530824214BF0020012050
S31508008D507047002070470120704701207047019A2C
S31508008D60C3BB80F85D10D37803F00301032920D034
S31508008D7013F0020F2ED092F90230002BB4BF022353
S31508008D80032303EB43030344917801F00F0183F8AF
S31508008D905110918883F85210937990F878209A4266
S31508008DA0B8BF80F8783090F85E30013380F85E30CE
S31508008DB0704792F90210002904DB13F0020F09D05C
S31508008DC00323DEE790F85610012363F3870180F842
S31508008DD05610D6E77047A0F10400FFF7C0BFF8B5F4
S31508008DE005460146002214464FF0080C4FF00F0EB8
S31508008DF0012736E005F1640405F1740601E0B44282
S31508008E0007D054F8040B0028F9D003689B689847E4
S31508008E10F5E7002385F8413085F8423085F8463075
S31508008E2085F8473085F87C3085F85030012285F87A
S31508008E305E202B6685F8783085F87930F8BD81F89C
S31508008E40524081F853403E4603EB43032B4493F8C4
S31508008E50530066F3870083F8530001320331042A6E
S31508008E60C8D0134681F8514012F0FF0FE7D181F8B8
S31508008E7052C081F853407646E6E7000010B504462E
S31508008E801B4B03F1080202603C334360002380F861
S31508008E90413080F8433080F8463080F84830C16465
S31508008EA080F85030012280F85E20036680F878301A
S31508008EB080F8793043668366C3660367FFF78FFFDA
S31508008EC0E06C68B1836F6BB101231A4602F11E018B
S31508008ED050F8211039B10133DBB21A460F2BF5DDF4
S31508008EE0204610BD00221E3240F82240F8E700BF97
S31508008EF038F702082DE9F04788B004460E461746AB
S31508008F001D46FFF76CFF94F8503023B1D925284643
S31508008F1008B0BDE8F087D4F84C80D8F800301B6854
S31508008F20002140469847814600283AD0D0F800A04C
S31508008F30BAF1000F37D004F151030360857103AB12
S31508008F400093122300221146E06C02F00AFCC9F8CD
S31508008F5000A0054640B10D280CBF0546E12523684B
S31508008F609B6820469847D2E7D8F800305D683B46AC
S31508008F70002231464046A84784F85000A8B19DF81B
S31508008F80133084F852309DF81D3084F85430BDF8FB
S31508008F901430A4F87630BDF81630A4F87430E025FD
S31508008FA0B5E7D625B3E7D725B1E7D425AFE710B59A
S31508008FB00446FFF714FFE06C03689B6894F85010AA
S31508008FC09847002010BDF0B585B0054604AB402291
S31508008FD023F8022D00F1C90690F8572090F8501092
S31508008FE090F8780001900096E86C02F0C3F918B181
S31508008FF005F16404743515E0BDF80E30002BF7D082
S3150800900005F1640405F1740701E0BC42F0D054F898
S31508009010040B0028F9D003681B6831469847F4E723
S31508009020A54207D054F8040B0028F9D003685B68FA
S315080090309847F5E705B0F0BD30B589B0B0F8863089
S3150800904023F00103A0F8863090F8515090F850406C
S31508009050C06C00230793069105920492039302932A
S315080090600193009320232A46214602F0C2FA09B04A
S3150800907030BD10B501460023A0F88630032280F8DB
S3150800908089200C2480F88A4080F88B308931FFF7D4
S31508009090D3FF10BD08B5B0F8863023F01003A0F84A
S315080090A086301A2380F889300C2380F88A30012309
S315080090B080F88B30C36843B1032380F88C300422D0
S315080090C000F18901FFF7B8FF08BD022380F88C304C
S315080090D0F5E708B50146B0F8863023F02003A0F876
S315080090E08630092380F88930102380F88A300023D7
S315080090F080F88B3003228931FFF79EFF08BD08B53B
S315080091000146B0F8863023F04003A0F886300123E4
S3150800911080F88930102380F88A30002380F88B3055
S3150800912003228931FFF788FF08BD08B50146B0F864
S31508009130863023F00203A0F88630092380F88930A8
S31508009140042380F88A30072380F88B30037F80F861
S315080091508C30437F80F88D30837F80F88E30C37FD4
S3150800916080F88F3090F8203080F8903090F82130D1
S3150800917080F89130002380F892300A228931FFF76F
S315080091805BFF08BD08B50146B0F8863023F0080332
S31508009190A0F88630192380F88930042380F88A30AD
S315080091A00A2380F88B30037F80F88C30437F80F861
S315080091B08D30837F80F88E30C37F80F88F3090F8AB
S315080091C0203080F8903090F8213080F891300123D3
S315080091D080F89230002380F8933080F8943080F835
S315080091E095300D228931FFF727FF08BDF8B50746E8
S315080091F00E46132380F889300C2380F88A300846F7
S31508009200FFF71CFD013087F88B000024E5B23046D5
S31508009210FFF714FD631CA84206D9725D57FA84F459
S3150800922084F88C201C46F1E757FA84F4002384F866
S315080092308C303046FFF702FD021D92B207F1890114
S315080092403846FFF7F9FEF8BD08B50146B0F886308E
S3150800925023F08003A0F88630012380F889300423A0
S3150800926080F88A30052380F88B30332380F88C30D9
S315080092708B2380F88D309E2380F88E30302380F83B
S315080092808F300A2380F8903008228931FFF7D4FE00
S3150800929008BD08B50146022380F88930042380F802
S315080092A08A30002380F88B3003228931FFF7C4FE09
S315080092B008BD08B5B0F8862022F48172A0F8862089
S315080092C0052280F88920042280F88A200D2280F859
S315080092D08B200A7880F88C204A7880F88D208A7846
S315080092E080F88E20CA7880F88F200A7980F8902036
S315080092F04A7980F89120182280F89220CC2280F8AA
S315080093009320012280F89420002280F8952080F886
S31508009310962080F8972080F89820102200F189017D
S31508009320FFF78AFE08BD08B500F11C01FFF7C1FF6B
S3150800933008BDF8B506460D2380F88930042380F861
S315080093408A30172380F88B30037F80F88C30437F70
S3150800935080F88D30837F80F88E30C37F80F88F3019
S3150800936090F8203080F8903090F8213080F89130CD
S3150800937090F8433063B3062380F8923090F87A3039
S31508009380D3B100F1140300F193021A3013F8011B4C
S3150800939002F8011B8342F9D106F1980306F1A201EE
S315080093A0002203F8012F9942FBD11A2206F18901FE
S315080093B03046FFF741FEF8BD00F11C0300F19302A9
S315080093C0223013F8011B02F8011B8342F9D1E3E7A7
S315080093D007693846FFF732FC86F892000024E5B2A2
S315080093E03846FFF72BFC631CA84206D97A5D56FA65
S315080093F084F484F893201C46F1E72C460F2DD4DC20
S315080094000023344484F893300135EDB22C460F2DF1
S31508009410F7DDCAE708B501460E2380F8893004232C
S3150800942080F88A30062380F88B30037F80F88C30EA
S31508009430437F80F88D30837F80F88E30C37F80F835
S315080094408F3090F8203080F8903090F8213080F8EE
S31508009450913009228931FFF7EFFD08BD08B50146AD
S315080094600C2380F88930042380F88A30062380F894
S315080094708B30037F80F88C30437F80F88D30837F74
S3150800948080F88E30C37F80F88F3090F8203080F8CF
S31508009490903090F8213080F8913009228931FFF711
S315080094A0CBFD08BDF0B585B0044604AB402223F8D1
S315080094B0022D90F8542090F8501090F878000190FA
S315080094C004F189000090E06C01F054FF10F0FB00F5
S315080094D068D194F88930013B162B63D8DFE813F07E
S315080094E045006400DB002201F6005F01040162000A
S315080094F06200620062006200620017006200620099
S31508009500620062006200620062004A015B0194F830
S315080095108E30002B46D1B4F8860040F00103A4F83B
S315080095208630B4F88C3041F20102934214D041F2ED
S315080095300902934236D104F1140304F18F0204F1AF
S315080095401A0512F8011B03F8011BAB42F9D140F0CA
S315080095502100A4F8860025E094F88F3084F840307E
S3150800956040F04100A4F886001CE094F88830042BEB
S3150800957013DD94F8433013B994F848306BB10023DF
S3150800958084F8883084F8413084F8433084F84630CB
S3150800959084F848300A2384F8803094F888300133F8
S315080095A084F8883005B0F0BD94F88B30002BF9D0DC
S315080095B09E46002BF6D0DB00DBB294F843704FF0E2
S315080095C0000C2FE084F87E1084F87D60002384F870
S315080095D07F30012384F87B300CEB4C0204EB42020B
S315080095E08C3204F11C0304F1220012F8011B03F863
S315080095F0011B9842F9D1B4F8863043F08003A4F8E9
S315080096008630CFE794F848502DB111F0050F02D0F7
S3150800961016F0C80F1CD10130C0B284460333DBB242
S31508009620704531DAE21892F88D6092F88E1092F849
S315080096308F20002FE6D0002AE4D111F0050FEAD0DA
S3150800964016F00C0FBED194F84850002DE0D1E2E791
S3150800965084F87E1084F87D6084F87F200CEB4C0338
S3150800966004EB43038C3304F11C0204F1220013F8C3
S31508009670011B02F8011B8242F9D1B4F8863043F087
S315080096808003A4F886308DE784F87E1084F87D6020
S3150800969084F87F2086E7B4F8863043F48072A4F80D
S315080096A0862094F88B206AB994F88D20120202F469
S315080096B0706294F88C100A43628343F48173A4F8A9
S315080096C086306FE7062384F880306BE794F88B3092
S315080096D0002B7FF467AFB4F8863023F0020343F01B
S315080096E00403A4F886305DE794F88B30002B7FF4EA
S315080096F059AF94F8923084F8223063B104F122030A
S3150800970004F1920104F13F0011F8012F03F8012F2B
S315080097100AB18342F8D1B4F8863043F00803A4F8B6
S3150800972086303FE704F11C0304F18B0204F12200A2
S3150800973012F8011B03F8011B8342F9D194F8912012
S3150800974084F87D2094F8923084F87E3094F893104B
S3150800975084F87F1013F0050F05D012F0C80F1CBF50
S31508009760012384F84730B4F8863043F01003A4F890
S31508009770863017E794F843302BB923693BB1204666
S31508009780FFF7D7FD0EE72046FFF7D3FD0AE7204689
S31508009790FFF740FE06E72046FFF760FE02E794F86B
S315080097A0433013B194F841306BB194F84830002B2C
S315080097B03FF4F8AE94F84630002B7FF4F3AE01235D
S315080097C084F84630EEE6012384F84130EAE608B527
S315080097D00146112380F88930042380F88A30022351
S315080097E080F88B30438B80F88C30C3F3032380F8E2
S315080097F08D3005228931FFF71FFC08BD10B5B0F87A
S31508009800862022F00402A0F88620062280F8892005
S31508009810042480F88A40032480F88B4080F88C1052
S31508009820C1F3032180F88D10132180F88E1000F102
S315080098308901FFF701FC10BD08B50146242380F80D
S3150800984089300C2380F88A30032380F88B30042370
S3150800985080F88C30082380F88D30002380F88E300D
S3150800986006228931FFF7E8FB08BD000070B50446FB
S3150800987090F88030102B1CD8DFE813F01100250073
S315080098804E005900640075007E008F00A400B300E6
S31508009890C500E100F60054011B006A017B01B0F81F
S315080098A0823001339BB2A0F88230B0F8842093420C
S315080098B000DC70BDFFF7DDFB012384F88030002350
S315080098C0A4F8823070BDB0F8823001339BB2A0F89C
S315080098D08230B0F8862012F0010F14D1B0F8842037
S315080098E09342E6DD02EB82035B009BB2B3F5FA6FA7
S315080098F0C8BF4FF4FA63A0F88430002380F880309C
S31508009900A0F8823070BD0023A0F88230022380F8C8
S315080099108030FFF791FF70BDB0F8863013F0010F65
S31508009920C7D0032380F88030FFF7D3FB70BDB0F8AB
S31508009930863013F0200FBCD0FFF7E1FB042384F830
S31508009940803070BDB0F8863013F0400FB1D0C168D2
S3150800995029B1FFF74BFC052384F8803070BD062338
S3150800996080F8803070BDB0F8863013F0010FA0D0B3
S31508009970062380F8803070BD90F8483013B990F807
S31508009980433033B12046FFF75FFC072384F8803065
S3150800999070BD0A2380F8803070BDB0F8863013F0A9
S315080099A0800F86D0FFF775FC94F87B301BB9082327
S315080099B084F8803070BD2046FFF7E4FB0C2384F85A
S315080099C0803070BDB0F8863013F0010F3FF471AFE8
S315080099D0002380F87B30FFF7A6FC092384F8803043
S315080099E070BDB0F8863013F4807F3FF462AF13F091
S315080099F0020F05D0FFF7EBFE0A2384F8803070BD0E
S31508009A00FFF791FC70BD90F84130002B7FF451AF01
S31508009A1090F84330002B7FF44CAF90F84630002B7B
S31508009A207FF447AF90F84830002B7FF442AFFFF73A
S31508009A3031FB012323720B2384F8803070BDB0F804
S31508009A40863013F0100F07D113F0040F3FF431AF2F
S31508009A50102380F8803070BD00230372FFF792FB55
S31508009A600C2384F8803070BDB0F8863013F0080FE8
S31508009A703FF41FAF00F1220508225249284623F079
S31508009A80E1FD90B9012384F84230002384F844307C
S31508009A9084F8453084F87A3016224B49284623F054
S31508009AA0D1FD80B9012384F84430B4F87E30252BE3
S31508009AB022D094F8433073B394F87B305BB3082311
S31508009AC084F8803070BD16224049284623F0BAFD36
S31508009AD038B9012384F87A3084F8443084F845305C
S31508009AE0E3E713223A49284623F0ACFD0028DCD1E7
S31508009AF0012384F87A30D8E794F87D30082BD8D13A
S31508009B0013223449284623F09DFD0028D1D101238C
S31508009B1084F87C30CDE72046FFF707FB0D2384F851
S31508009B20803070BDB0F8863013F0020F3FF4C1AE36
S31508009B3090F87C3013B1012380F846300023637215
S31508009B40A372E372A4F886300F2384F8803070BDC0
S31508009B50B0F8823001339BB2B3F57A7F02DCA0F805
S31508009B60823070BD0023A0F882300A2380F8803046
S31508009B7070BDB0F8863013F0040F3FF49AAE002596
S31508009B80A0F88650402632462946893023F017FC2D
S31508009B903246294604F1C90023F011FC84F84350E3
S31508009BA084F8425084F8415084F87B5084F8485031
S31508009BB084F8475084F8465084F87C500A2384F881
S31508009BC0803076E6407603084C7603086476030808
S31508009BD07C7603089076030890F879300BB9002054
S31508009BE0704710B5044605F0B5F8236EC01A00286C
S31508009BF00EDB05F0AFF894F8783018442066204656
S31508009C00FFF750FC2046FFF731FE2046FFF7DBF949
S31508009C10002010BDF0B583B002AF03F10F0424F0A5
S31508009C200704ADEB040D0DF1080C8DF80810C1F30F
S31508009C30032141F020018CF80110191D8CF802103F
S31508009C4009128CF803108CF8043000218CF80510E2
S31508009C50397E8CF80610397F8CF807105BB11E46E2
S31508009C60E646002421467444555C2572013189B2C2
S31508009C700C468E42F7DC90F85A2090F85010C06CCB
S31508009C80CDF800C0083301F096FC10B90437BD467C
S31508009C90F0BD642005F064F8F8E770B582B0BDF849
S31508009CA01850022680F8096180F80A21042280F8F3
S31508009CB00B21002280F80C2180F80D512D1280F816
S31508009CC00E511D7880F80F515B7880F8103101929B
S31508009CD001230093082300F20912FFF79BFF02B045
S31508009CE070BD70B582B0069D032680F8096180F8BC
S31508009CF00A21082280F80B21002280F80C211E7800
S31508009D0080F80D615B7880F80E312B7880F80F317A
S31508009D106B7880F810319DF81C3080F8113180F886
S31508009D20122180F8132180F814210192012300934F
S31508009D300C2300F20912FFF76DFF02B070BD30B5B3
S31508009D4083B0042580F8095180F80A21082280F892
S31508009D500B21002280F80C211D7880F80D515B78C4
S31508009D6080F80E3180F80F2180F81021012380F841
S31508009D701131022580F81251FF2580F8135180F819
S31508009D801451019200930C2300F20912FFF742FFC7
S31508009D9003B030BD70B582B0052580F8095180F84A
S31508009DA00A210A2280F80B21002280F80C211D784E
S31508009DB080F80D515B7880F80E3180F80F2180F815
S31508009DC0102180F8112180F81221012380F813311F
S31508009DD0022580F81451A02680F8156180F81651DE
S31508009DE0019200930E2300F20912FFF713FF02B047
S31508009DF070BD70B582B0069D062680F8096180F8A8
S31508009E000A21042280F80B21002280F80C211E78F2
S31508009E1080F80D615B7880F80E312B7880F80F3169
S31508009E206B7880F81031019201230093082300F221
S31508009E300912FFF7EFFE02B070BD70B582B0069D3D
S31508009E40072680F8096180F80A21042280F80B2188
S31508009E50002280F80C211E7880F80D615B7880F866
S31508009E600E312B7880F80F316B7880F8103101921B
S31508009E7001230093082300F20912FFF7CBFE02B074
S31508009E8070BD10B58AB001238DF820300AAA0023C8
S31508009E9002F8073D8B1D13F8014D02F8014F8B425E
S31508009EA0F9D190F8512090F85010C06C0023079310
S31508009EB008AC069408240594049403930323029398
S31508009EC0F523019309230093212301F092FB0AB09D
S31508009ED010BD10B58CB005238DF8243010238DF8ED
S31508009EE02B3001238DF82C3002238DF82D301223C8
S31508009EF08DF82E304B1E09AA053113F8014F02F8CA
S31508009F00014F8B42F9D190F8512090F85010C06C4F
S31508009F100023079309AC06940B2405940494039331
S31508009F20032302930523019309230093212301F0B8
S31508009F3060FB0CB010BD00002DE9F04792B0044656
S31508009F401F4690F85480002380F85430C66C336856
S31508009F501B6890F8501030469847002800F0EF80AC
S31508009F6081464FF4967004F0FBFE94F850300022B8
S31508009F701146E06C01F046FC054638B1002389F825
S31508009F80063023689B6820469847D9E0002389F85D
S31508009F90063033681B6894F85010304698470028F6
S31508009FA000F0D280877104F151094B46012294F8DA
S31508009FB05010E06C00F0A9FF05460028E1D1B4F87E
S31508009FC0762040F24C539A4246D04746B8F1000FE5
S31508009FD000F08B805D4EDFF87881DFF878A1636F3B
S31508009FE0B3420CBFCDF80CA0CDF80C80231D04930A
S31508009FF000228DF82820ADF82A208DF83C208DF80F
S3150800A0003D208DF83E208DF844200BABCDF8153059
S3150800A01007939DF814108DF821108DF820100993D8
S3150800A02094F8501003AB00932B46E06C01F0C1FB8B
S3150800A030002840F0828094F85E20032A59DC013516
S3150800A040EDB2BD42CBDB00231A4694F85010E06C03
S3150800A05001F0D8FBD12594E7B4F87430B3F51A7F2C
S3150800A06007D040F22F42934203D040F2D5329342B2
S3150800A070ABD1642004F074FE012394F8512094F8BF
S3150800A0805010E06C01F0D5FB054600287FF479AF47
S3150800A09063690BB9238B6BB1B4F87430B3F51A7FC7
S3150800A0A003D040F22F42934219D104F114012046FD
S3150800A0B0FFF7E7FE002394F8512094F85010E06C5F
S3150800A0C001F0B7FB00231A4694F85010E06C01F033
S3150800A0D099FB23689B6820469847D12530E004F110
S3150800A0E014012046FFF7F5FEE4E794F85E20032AFC
S3150800A0F0A9DD4B4694F85010E06C00F006FF0546C3
S3150800A10000287FF43EAF94F85D3094F8512094F817
S3150800A1105010E06C01F08DFB054600287FF431AF46
S3150800A1206423A4F884300023A4F8823084F88030AD
S3150800A1302372012384F8793002E0054621E7D62503
S3150800A140284612B0BDE8F087D625F9E7E8215C0A6B
S3150800A1503C7603083076030870B582B004460E468E
S3150800A160154690F83030042B00F2E480DFE803F05F
S3150800A170030D1E254A0002230372D0F80920026146
S3150800A18043750375012380F830302A46314604F1B9
S3150800A190100002F0C5F90346002874D0D4F8093037
S3150800A1A01A7884F831205B7884F8323004F1220377
S3150800A1B0C4F80930032384F8303094F83230023B6F
S3150800A1C01F2B16D8DFE803F01315104315151515C0
S3150800A1D01515151515151515151515151515151521
S3150800A1E01515151515151546002384F8333007235C
S3150800A1F02372D4F809302361237A637523750423FF
S3150800A20084F8303094F83230042B3FD0052B6AD0CE
S3150800A210022B24D0237F002B00F08580012B40F0F1
S3150800A2208D80E28B002A00F087802B886BB1013A7B
S3150800A230E2833368013333602B88013B9BB22B8062
S3150800A240E28B002A78D0002BF1D100231BE00523EE
S3150800A2502372CEE794F83130023B2372C9E72A46C7
S3150800A260314604F1100002F05BF9034658B194F840
S3150800A270253084F8343004F12003C4F8093000236B
S3150800A28084F830300123184602B070BD2A4631469C
S3150800A29004F1100002F044F903460028F3D094F8BC
S3150800A2A02530E02BE7D194F82630012BE3D194F83A
S3150800A2B038309BB194F82730002BDCD0012384F882
S3150800A2C0333094F8223084F8363094F8233084F802
S3150800A2D0373094F8273084F83530CCE794F82730AF
S3150800A2E0012BC8D1EAE72A46314604F1100002F0EC
S3150800A2F017F903460028C6D094F83330002BBAD095
S3150800A30060680028B7D094F8373094F8362094F867
S3150800A3103410056804F12006019694F83560009615
S3150800A3202D68A847A7E794F83130023BE383012359
S3150800A330237776E70123A6E700232377E38B002B11
S3150800A34099D000239FE710B582B00446ADF80610F1
S3150800A3500092BDF806303BB10DF10602694620466B
S3150800A360FFF7FAFE0028F4D102B010BD70B582B02E
S3150800A37004460E46154690F83030042B00F2E48069
S3150800A380DFE803F0030D1E254A0002230372D0F806
S3150800A3900920026143750375012380F830302A4687
S3150800A3A0314604F1100002F0BBF80346002874D0C9
S3150800A3B0D4F809301A7884F831205B7884F832307A
S3150800A3C004F12203C4F80930032384F8303094F8E2
S3150800A3D03230023B1F2B16D8DFE803F01315104363
S3150800A3E0151515151515151515151515151515150F
S3150800A3F0151515151515151515151546002384F883
S3150800A400333007232372D4F809302361237A63751E
S3150800A4102375042384F8303094F83230042B3FD067
S3150800A420052B6AD0022B24D0237F002B00F08580D1
S3150800A430012B40F08D80E28B002A00F087802B8864
S3150800A4406BB1013AE2833368013333602B88013BF1
S3150800A4509BB22B80E28B002A78D0002BF1D1002307
S3150800A4601BE005232372CEE794F83130023B2372B2
S3150800A470C9E72A46314604F1100002F051F80346AE
S3150800A48058B194F8253084F8343004F12003C4F820
S3150800A4900930002384F830300123184602B070BD15
S3150800A4A02A46314604F1100002F03AF8034600281D
S3150800A4B0F3D094F82530FF2BE7D194F82630012BFA
S3150800A4C0E3D194F838309BB194F82730002BDCD0D0
S3150800A4D0012384F8333094F8223084F8363094F81F
S3150800A4E0233084F8373094F8273084F83530CCE7B1
S3150800A4F094F82730012BC8D1EAE72A46314604F1F9
S3150800A500100002F00DF803460028C6D094F8333040
S3150800A510002BBAD060680028B7D094F8373094F882
S3150800A520362094F83410056804F12006019694F84C
S3150800A530356000962D68A847A7E794F83130023BA6
S3150800A540E3830123237776E70123A6E7002323770E
S3150800A550E38B002B99D000239FE710B582B0044601
S3150800A560ADF806100092BDF806303BB10DF10602B3
S3150800A57069462046FFF7FAFE0028F4D102B010BD5E
S3150800A58010B50446436803B1984723689B6920467B
S3150800A590984710BD70477047704708B50022427546
S3150800A5A080F82520026180F82A200368DB6998472D
S3150800A5B008BD10B582B004468189027D0132D2B247
S3150800A5C0027500F12803009300F118038068FFF76D
S3150800A5D010FC23689B6820469847092384F82A308C
S3150800A5E002B010BD90F82A30002B4FD1F0B583B0D9
S3150800A5F00446806890F8463033B1437A23B9637DC0
S3150800A60013B994F825302BB1236913F0010F15D12E
S3150800A61003B0F0BD0123437284F82530A068418B4E
S3150800A620A1810022226122751123009304F12603D9
S3150800A630FFF733FB022384F82A30E9E704F12607FB
S3150800A64004F11605227DA1890126019600953B464F
S3150800A650FFF747FB304604F083FB227DA1890023E0
S3150800A660019300953B46A068FFF73BFB237D3344E7
S3150800A6702375304604F074FB2B46227DA189A06819
S3150800A680FFF75DFB042384F82A30C1E77047000012
S3150800A69070B5064618483060B16089B1486E58B141
S3150800A6A00120044601EB84056D6E35B10130C0B258
S3150800A6B004460328F6DD03E0002401EB84014E6618
S3150800A6C00E493160002186F82410F1613162B068C4
S3150800A6D080F84820B2681361702386F8263086F819
S3150800A6E02710712386F8283086F829103046FFF798
S3150800A6F054FF304670BD00BFAC76030884F70208E5
S3150800A70010B584B0034690F82420012A84BF00229D
S3150800A71080F8242090F8241041F0700104AA02F869
S3150800A720011D81898068DC7D01949B7D009301234E
S3150800A730FFF770FA04B010BDF0B583B0044690F880
S3150800A7402A30023B072B09D8DFE803F03D4F04A364
S3150800A75010687A8D036913F0020F01D103B0F0BDBA
S3150800A760FFF7CEFF062384F82A30F7E7036913F0CC
S3150800A770100FF3D000F1280700F11805027D818932
S3150800A7800126019600953B468068FFF7AAFA3046EF
S3150800A79004F0E6FA227DA1890023019300953B4641
S3150800A7A0A068FFF79EFA237D33442375304604F0EC
S3150800A7B0D7FA2B46227DA189A068FFF7C0FA08239D
S3150800A7C084F82A30CAE7036913F0040FC6D0027D5D
S3150800A7D00132D2B2027500F1160381898068FFF74B
S3150800A7E0AEFA032384F82A30B8E7036913F0020F98
S3150800A7F0B4D0FFF785FF012004F0B2FA227D0132BA
S3150800A800D2B22275A1891323009304F12803A06804
S3150800A810FFF743FA072384F82A309FE7036913F002
S3150800A820400F9BD0027D0132D2B2027500F11803A7
S3150800A83081898068FFF783FA082384F82A308DE730
S3150800A840036913F0200F89D08268002382F8463006
S3150800A850826882F848300125457503681B69984760
S3150800A86084F82A507AE7036913F0800F3FF476AF2D
S3150800A870027D0132D2B20275818900F12603009366
S3150800A88000F116038068FFF7B4FA052384F82A3026
S3150800A89064E7036913F0080F3FF460AF81898068A5
S3150800A8A0FEF7ACFF4FF6FF73A3810023236184F8FC
S3150800A8B02A3053E770B582B083685A7A52B993F84A
S3150800A8C047203AB1427D2AB990F8252012B90A7A6A
S3150800A8D0022A06D086890A78F3B29A4215D002B0BF
S3150800A8E070BD4C7B0A7B42EA0422112AF2D100226F
S3150800A8F083F8472084680123637280F825308368CB
S3150800A9005B8B838180F82A20E4E74A78331243F088
S3150800A91020039A42E3D10D4604468B79CA7943EA65
S3150800A9200221012908D094F82810994200F00781DD
S3150800A9302046FFF701FFD2E72B7A012BF8D0032B2D
S3150800A9401ED0022B4FD0052B6BD0042B00F0918024
S3150800A950062B00F0B380072BEAD12B7BA27D9A4207
S3150800A96000F0E180227E9A42E2D16A7B637E9A42B7
S3150800A970DED16B7A2375236943F080032361D7E719
S3150800A9806A7C2B7C53EA0223D2D1EA7CAB7C53EA5D
S3150800A9900223CDD1AB7B94F826209A4213D094F8A3
S3150800A9A028209A42C4D1EA7B94F829309A42BFD12A
S3150800A9B06B7A23752B7B23766B7B6376236943F04F
S3150800A9C040032361B4E7E97B94F827209142E6D156
S3150800A9D06B7A23752B7BA3756B7BE375236943F031
S3150800A9E004032361A4E76A7B2B7B43EA0223112B2A
S3150800A9F00CD0132B9CD16B7A2375AB7B2376EB7B20
S3150800AA006376236943F01003236191E76B7A237514
S3150800AA10AB7BA375EB7BE375236943F001032361E5
S3150800AA2086E76A7C2B7C53EA022381D12B7B94F838
S3150800AA3026209A4211D094F828209A427FF478AFBB
S3150800AA406A7B94F829309A427FF472AF6B7A237541
S3150800AA50236943F0200323616AE7697B94F827207A
S3150800AA609142E8D16B7A2375236943F00203236187
S3150800AA705EE72B7B94F826209A4212D094F8282079
S3150800AA809A427FF455AF6A7B94F829309A427FF44C
S3150800AA904FAF04F118036A7A3146A068FFF77AF9CE
S3150800AAA046E7697B94F827209142E7D104F116031B
S3150800AAB06A7A3146A068FFF76DF939E72B7B94F877
S3150800AAC026209A421AD094F828209A427FF430AF6A
S3150800AAD06A7B94F829309A427FF42AAF6A7A2275FB
S3150800AAE004F11803009304F128033146A068FFF720
S3150800AAF0A4F923689B682046984719E7697B94F868
S3150800AB0027209142DFD16A7A227504F11603009351
S3150800AB1004F126033146A068FFF78FF923689B687E
S3150800AB202046984704E7697BE27D91427FF41AAF95
S3150800AB306B7A2375236943F008032361F8E694F8D2
S3150800AB40293093427FF4F4AE2B7AA12B7FF4F0AE32
S3150800AB502E79711E23685B6905F10902C9B2204680
S3150800AB6098476B7A012B10D0022B7FF4E1AE206A4E
S3150800AB7000283FF4DDAEB31E02680A350095156855
S3150800AB80DBB200222146A847D2E6E06900283FF456
S3150800AB90CFAEB31E02680A3500951568DBB20022EF
S3150800ABA02146A847C4E603292CD8DFE801F0020DA0
S3150800ABB01721007A00F00F00072825D030B30128A6
S3150800ABC014BF002001207047007A00F00F000138FA
S3150800ABD0C0B202288CBF002001207047007A00F01E
S3150800ABE00F000338C0B202288CBF0020012070472E
S3150800ABF0007A00F00F000538C0B202288CBF00208A
S3150800AC0001207047002070470120704701207047D7
S3150800AC1008B5032908DD8068C0F31700044B5B5CA0
S3150800AC20D84000F0010008BDFFF7BDFF08BD00BF12
S3150800AC30A4F702080A4B5B5C01229A4090F843305D
S3150800AC40B0F8441043EA012323EA020180F84310CE
S3150800AC50090AA0F844101A4214BF012000207047C0
S3150800AC60A4F70208082904D009290CBF007B002094
S3150800AC707047C07A704701440879704770B5044632
S3150800AC8001295BDD1346002A58D01278012A0DD017
S3150800AC90112A56D1032954DDCA1ED2B23C2A28BF2E
S3150800ACA03C22D91C043022F065FB08E04A1ED2B2C9
S3150800ACB03C2A28BF3C22591C043022F05BFBA268C0
S3150800ACC0C2F31702236CC3F317039A4236D022EA5B
S3150800ACD0030384F843301B0AA4F84430236C62F358
S3150800ACE01703236400212046FFF75DFF0646054645
S3150800ACF001212046FFF757FF10B146F00205EDB2D5
S3150800AD0002212046FFF74FFF10B145F00405EDB2CA
S3150800AD1003212046FFF747FF10B145F00805EDB2BD
S3150800AD2094F84E309D4209D025EA030394F843204F
S3150800AD3063F3030284F8432084F84E5094F84D30A8
S3150800AD4003B970BD23681B6804F14601204698477D
S3150800AD50F7E799B110B40C46C37C8B4218D002228F
S3150800AD601346C3EBC30303441B7BA34208D001323B
S3150800AD70D2B213460F2AF4DD002006E008307047E9
S3150800AD8042B10830C2EBC20210445DF8044B70476A
S3150800AD900122F6E70020F8E711F0800F49D130B418
S3150800ADA00546072B47DC7AB9EC7C14B30220044627
S3150800ADB0C4EBC4042C44247B5CB1441CE0B20446B6
S3150800ADC00F28F5DD002037E0C0790728ECD10020F0
S3150800ADD032E088B3A9B972B1C0EBC0032B44412253
S3150800ADE01A73EB790133EB71C0EBC0002844007B82
S3150800ADF022E00120EEE7C0EBC0032B4401221A73C0
S3150800AE00F2E74FF0000461F3C5046AB144F0400468
S3150800AE10EB790133DBB2EB7163F30204C0EBC000DC
S3150800AE2028440473E0B207E06FF3861463F3020460
S3150800AE30F4E700207047002030BC704770B4134B0D
S3150800AE4003600022C2710273012343738273051DD6
S3150800AE5085600271082141710F2161F387028271B1
S3150800AE60024600241E46D47416755475C3EBC301F6
S3150800AE7001448D6001330732102BF4D1002380F88A
S3150800AE80B8301122024B1A7070BC7047C876030896
S3150800AE903C0A002010B491B10C46C37C8B4228D0E2
S3150800AEA002210B46C3EBC30303441B7BA3421AD000
S3150800AEB00131C9B20B460F29F4DD00201CE000F170
S3150800AEC00801F1B10868B8B14C79E4B10378934246
S3150800AED012D0002303300133DBB2A3420BDA017828
S3150800AEE09142F7D108E051B10830C1EBC1010144E4
S3150800AEF0E7E70121F8E700205DF8044B70470020DA
S3150800AF00FAE70020F8E70020F6E723B330B41D4639
S3150800AF1089B1C37C8B421CD002242346C3EBC303EE
S3150800AF2003441B7B8B420ED00134E4B223460F2C1C
S3150800AF30F4DDD62005E0083088B10171056042715C
S3150800AF40002030BC704744B10830C4EBC404204428
S3150800AF50F2E70124F8E7D8207047D620F1E7D62093
S3150800AF60EFE7000070B582B00C4616460C4D00227D
S3150800AF701021284604F0B2FD44F002048DF804407E
S3150800AF808DF805604FF0FF33022201A9054807F046
S3150800AF90C4F901221021284604F0A0FD02B070BDB4
S3150800AFA00010024098D300202DE9F04F83B0824666
S3150800AFB0174601939DF83090012500EB810802F1B0
S3150800AFC01E0B19E057BB0122E8215046FFF7CAFFBE
S3150800AFD0662003F0C5FED8F8780003681C684B465F
S3150800AFE0019A3946A0470D282AD1022E2CDC642066
S3150800AFF003F0B6FE0135EDB26E1EF6B2D8F878004B
S3150800B00003685C684B46019A3946A047E028D9D0C0
S3150800B0100D280AD00028DED0044609E05AF82B008D
S3150800B02003685B6901999847D5E7022E04DD044653
S3150800B030204603B0BDE8F08F642003F091FED9E7FF
S3150800B04004460028F4D000E004463FB11E375AF8FB
S3150800B050270003685B6901999847E9E70122E82117
S3150800B0605046FFF77FFF662003F07AFEE0E7000010
S3150800B07070B584B004AC04F8091D104D00221021E7
S3150800B080284604F02BFD0E4E4FF0FF3301222146D1
S3150800B090304607F042F904A9002301F8013D4FF0B4
S3150800B0A0FF330122304607F023FB012210212846F0
S3150800B0B004F014FD9DF80F0004B070BD00100240A6
S3150800B0C098D300202DE9F84F04468A4617469B4632
S3150800B0D003F040FE00F59C5508350026B146B046FB
S3150800B0E04AEA07074FF0F00A03F034FE401B00282F
S3150800B0F020DA3A4651462046FFF734FFC82603F0C1
S3150800B10029FE401B00280BDA31462046FFF7B0FF20
S3150800B11010F0800FF3D08022C8212046FFF722FFC7
S3150800B120F8212046FFF7A4FF00F00F06042E04D0EE
S3150800B1300E2E0CD03046BDE8F88F09F101091FFA2A
S3150800B14089F9BBF1000FCFD0D945CDD1F2E708F187
S3150800B15001085FFA88F8B8F1030FC5D1EAE70000DD
S3150800B1602DE9F04F87B000908B4601929A46109EC3
S3150800B1709DF844300393BAF800904B780293002365
S3150800B180AAF800308B7813F0020F14BF2022102281
S3150800B190E821FFF7E7FE17E0F821009C2046FFF7B5
S3150800B1A067FF80F01000C0F300109BF8023060F3D0
S3150800B1B041038BF8023013F0020F14BF202210222D
S3150800B1C0E8212046FFF7CEFE019B9BF800200021D0
S3150800B1D00098FFF777FF05460628DDD000286AD1D4
S3150800B1E0C821009C2046FFF743FF10F0040F5FD0EC
S3150800B1F030212046FFF73CFF04464845C8BF5FFAA2
S3150800B20089F4BAF80020A9EB020212B222EAE27225
S3150800B210A242A8BF224617460DF11808082308F8C7
S3150800B220013D00221021254804F058FC4FF0FF3359
S3150800B23001224146224807F070F8FFB23A4600213B
S3150800B240304622F0BCF84FF0FF333A4631461C48E8
S3150800B25007F04EFA3E4401221021184804F03EFC3D
S3150800B2600422C8210098FFF77DFEBAF8003023446F
S3150800B2709BB2AAF80030029A944208DB994506DD8B
S3150800B280039B002BA0D0184603F06AFD9CE7A8464E
S3150800B290F8210098FFF7ECFEC0F300109BF8023087
S3150800B2A060F341038BF80230404607B0BDE8F08FE3
S3150800B2B04FF0F008F8E78046F6E700BF00100240B6
S3150800B2C098D30020F8B50E4689B1C17CB14244D066
S3150800B2D002252C46C4EBC4040444247BB44235D06E
S3150800B2E00135EDB22C460F2DF4DDD620F8BD00F160
S3150800B2F00805002D38D02968002937D01C4607468E
S3150800B3003146FFF7C7FD206090B383789A080F2A65
S3150800B310A8BF0F2201239340013B069A13803246A9
S3150800B320E0213846FFF71EFED8213846FFF7A0FE73
S3150800B330AB79A3B197F8B82042F002020243D2B221
S3150800B340D8213846FFF70EFE0020F8BD55B100F1AA
S3150800B3500801C5EBC5050D44CBE70125F7E700F065
S3150800B360F902EDE7D620F8BDD620F8BDD720F8BDFE
S3150800B370DB20F8BD30B585B004461D46002303938F
S3150800B380ADF80A300DF10A03009303ABFFF79AFFF5
S3150800B390034610B1184605B030BDBDF80A209DF821
S3150800B3A024300193089B00932B4603992046FFF708
S3150800B3B0D7FE0346EEE70000F0B583B00D46174604
S3150800B3C01C46114E00221021304604F087FB45F03A
S3150800B3D0020502A901F8015D0C4D4FF0FF33012269
S3150800B3E0284606F09AFF4FF0FF333A46214628468C
S3150800B3F006F093FF3C4401221021304604F06EFB10
S3150800B400204603B0F0BD00BF0010024098D30020CC
S3150800B4102DE9F04F85B00192009391F8018008F16B
S3150800B420FF33DBB23F2B04D9DA25284605B0BDE841
S3150800B430F08F04460E4603F08DFC00F59C5A0AF17F
S3150800B440080AB37803F00103002B14BF80224022B8
S3150800B450E8212046FFF786FD009B002B00F0A98017
S3150800B4604FF0C80BCDF80880BDF80830009A934213
S3150800B47028BF134603935FFA83F80E9B42461021B2
S3150800B4802046FFF799FF424638212046FFF76AFD16
S3150800B490327842F02002F0212046FFF763FD594634
S3150800B4A02046FFF7E5FD10F0800FF8D080225946B8
S3150800B4B02046FFF757FDF8212046FFF7D9FD00F093
S3150800B4C00F054FF000094F4663E003F043FCA0EB7D
S3150800B4D00A0000285FDA062D1CD00E2D15D0042D83
S3150800B4E00AD0F8212046FFF7C3FDC0F34010B37811
S3150800B4F060F30003B37098E709F101091FFA89F9A7
S3150800B500019BEBB199451BD1EBE70137FFB2032F3E
S3150800B51016D1E6E7F8212046FFF7AAFD80F02000BD
S3150800B520C0F34010B37860F30003B37003F001036F
S3150800B530002B14BF80224022E8212046FFF712FD87
S3150800B540002238212046FFF70DFD0E9B1A781021A0
S3150800B5502046FFF707FD424638212046FFF702FD41
S3150800B560327842F02002F0212046FFF7FBFC5946CC
S3150800B5702046FFF77DFD10F0800FF8D0802259464F
S3150800B5802046FFF7EFFCF8212046FFF771FD00F093
S3150800B5900F05002D99D10099039A8B1A9BB219466B
S3150800B5A000930E9B184610440E9000297FF45CAF5A
S3150800B5B097E7002595E730B585B004461D46002374
S3150800B5C00393ADF80A300DF10A03009303ABFFF7B6
S3150800B5D079FE034610B1184605B030BDBDF80A20FD
S3150800B5E0089B00932B4603992046FFF711FF034655
S3150800B5F0F1E72DE9F04F8BB0029003921C46BDF897
S3150800B6006090BDF86470DDF868801B9E0023069381
S3150800B610ADF816300DF11603009306ABFFF752FE90
S3150800B620054618B128460BB0BDE8F08F8DF81C40CA
S3150800B6309DF850308DF81D309DF854308DF81E3029
S3150800B6409DF858308DF81F30BDF85C30ADF82030C5
S3150800B650ADF8229007AB08222021029D2846FFF765
S3150800B660ABFEBDF81630039A10212846FFF72AFDCF
S3150800B67005460028D6D104F08004B8F1000F5DD045
S3150800B680002C47D0069A937843F002039370B9F1D9
S3150800B690000F58D04C464FF0000B26E0DDF818A0F6
S3150800B6A0F8210298FFF7E4FC80F02000C0F3401070
S3150800B6B09AF8023060F341038AF8023013E03368DF
S3150800B6C0D3F800A0BDF81410A9EB0403ADF8263092
S3150800B6D00DF1260342463046D047BDF81430E41A29
S3150800B6E0A4B2BB422FDB002C36D0ADF81470BDF8DF
S3150800B6F01620CDF804B0CDF8008005AB069902985F
S3150800B700FFF72EFD05460628C8D000288AD1002E48
S3150800B710D5D1E2E7069A937843F001039370BDF812
S3150800B7201620CDF800803B4606990298FFF770FE72
S3150800B730054600287FF476AF802105E0002CCCBFB3
S3150800B740A021802100E0A021BDF81630039A0298B6
S3150800B750FFF7B8FC054665E7A021002D7FF462AF28
S3150800B760F2E730B589B0002407940C9D0695059339
S3150800B77004930394012302930194062300938023E0
S3150800B780FFF737FF09B030BD30B589B000240794FC
S3150800B7900D9D0695059304930394022302939DF841
S3150800B7A030300193062300938023FFF722FF09B068
S3150800B7B030BDF0B599B005460E4617461C4608AB8F
S3150800B7C0019300940923FFF7DFFF034610B11846DB
S3150800B7D019B0F0BD1E9B079308AB0693402305934B
S3150800B7E0BDF82230049300230393022302930194A5
S3150800B7F00623009380233A4631462846FFF7F9FE8A
S3150800B8000346E4E710B588B0002407940694059427
S3150800B8100494039402940193052300932346FFF7A7
S3150800B820E8FE04464FF4967003F09AFA204608B0EC
S3150800B83010BD10B588B000240794069405940494A6
S3150800B840039402940193092300932346FFF7D1FE3C
S3150800B85008B010BD002900F01E832DE9F04F99B0FD
S3150800B86017918346C1EBC10303441B7B03F0070210
S3150800B870099213F0400F5FD0012303930F930193AE
S3150800B880039A531EDBB20E2B00F21E820F2A4ADCE5
S3150800B890C2EBC2035B441B7BC3F3C203099A934200
S3150800B8A059D1039B002B3ED0039B1193C3EBC303D3
S3150800B8B05B441B7B03F007020A9213F0400F67D024
S3150800B8C001230493049A531EDBB20E2B00F2068260
S3150800B8D00F2A54DCC2EBC2035B441B7BC3F3C203CF
S3150800B8E00A9A934262D1049B002B48D0049B129378
S3150800B8F0C3EBC3035B441B7B03F007020B9213F0F5
S3150800B900400F00F0D3810F9B059396E1C3EBC3026A
S3150800B9105A44127BC2F3C20209998A421DD00133E6
S3150800B920DBB20F2BF2DD9BF80730099A934204BF6E
S3150800B93003F1FF338BF80730179BC3EBC3025A4456
S3150800B940002313730121517393730BF1040393605E
S3150800B95019B0BDE8F08F039BE1E70393A1E7012344
S3150800B9600393A1E7C3EBC3025A44127BC2F3C20294
S3150800B9700A998A421CD00133DBB20F2BF2DD9BF801
S3150800B98007300A9A934204BF03F1FF338BF8073056
S3150800B990119BC3EBC3035B4400221A734FF00101EA
S3150800B9A059739A730BF104029A6069E7049BE2E7FC
S3150800B9B0049398E70F9B049398E7019B05935DE131
S3150800B9C0019B069314E1019B0793C5E0DDF80490FB
S3150800B9D0CAE1DDF820909BF80730169A934204BF17
S3150800B9E003F1FF338BF80730109BC3EBC3035B44AB
S3150800B9F000221A734FF0010159739A730BF104026E
S3150800BA009A6009F1FF33DBB20E2B00F28F81B9F190
S3150800BA100F0F69DCC9EBC9035B441B7BC3F3C20385
S3150800BA200E9A934200F09C810E9A89E1DDF82090E7
S3150800BA30D1E7019FC8E1019DF0E1019C17E29BF85F
S3150800BA400730B34204BF03F1FF338BF80730C9EB65
S3150800BA50C909D9444FF0000389F80C304FF00103A7
S3150800BA6089F80D304FF0000389F80E300BF1040306
S3150800BA70C9F808306B1EDBB20E2B00F2B7810F2D0A
S3150800BA8009DCC5EBC5035B441B7BC3F3C203434513
S3150800BA9040F0B481BFE19BF80730434504BF03F18A
S3150800BAA0FF338BF80730029BC3EBC3035B440022CA
S3150800BAB01A734FF0010159739A730BF104029A60D5
S3150800BAC07B1EDBB20E2B00F267810F2F09DCC7EB5A
S3150800BAD0C7035B441B7BC3F3C203534540F0648131
S3150800BAE06FE1DDF8209076E79BF807300E9A9342CF
S3150800BAF004BF03F1FF338BF80730159BC3EBC30371
S3150800BB005B4400221A734FF0010159739A730BF1C3
S3150800BB1004029A60079A531EDBB20E2B00F2FC80D1
S3150800BB200F2A2DDCC2EBC2035B441B7BC3F3C203A3
S3150800BB300D9A93420ED00D99079B0133DBB20F2B5A
S3150800BB401EDCC3EBC3025A44127BC2F3C2028A420A
S3150800BB50F3D10793079B9BB1079A1592C2EBC203D1
S3150800BB605B441B7B13F0400FC7D0C2EBC2035B4498
S3150800BB701B7B03F007030E93DDF804A0D14640E7CC
S3150800BB809BF807300D9A934204BF03F1FF338BF8F5
S3150800BB900730149BC3EBC3035B4400221A734FF0B0
S3150800BBA0010159739A730BF104029A60069A531E9F
S3150800BBB0DBB20E2B00F2A6800F2A28DCC2EBC203EA
S3150800BBC05B441B7BC3F3C2030C9A93420ED00C99B9
S3150800BBD0069B0133DBB20F2B19DCC3EBC3025A44B5
S3150800BBE0127BC2F3C2028A42F3D10693069B73B153
S3150800BBF0069B1493C3EBC3035B441B7B03F007024A
S3150800BC000D9213F0400FC4D0019B079382E79BF86F
S3150800BC1007300C9A934204BF03F1FF338BF80730C1
S3150800BC20139BC3EBC3035B4400221A734FF0010155
S3150800BC3059739A730BF104029A60059A531EDBB284
S3150800BC400E2B55D80F2A28DCC2EBC2035B441B7B9C
S3150800BC50C3F3C2030B9A93420ED0059B0133DBB2A2
S3150800BC600F2B1ADCC3EBC3025A44127BC2F3C2027F
S3150800BC700B998A42F2D10593059B73B1059B1393E1
S3150800BC80C3EBC3035B441B7B03F007020C9213F060
S3150800BC90400FC5D0019B069388E79BF807300B9A9F
S3150800BCA0934204BF03F1FF338BF80730129BC3EBB3
S3150800BCB0C3035B4400221A734FF0010159739A7348
S3150800BCC00BF104029A60FDE59BF81330C3F3C20337
S3150800BCD0099A93423FF443AE012320E69BF81330BA
S3150800BCE0C3F3C2030A9A93423FF464AE0F9B42E63B
S3150800BCF09BF81330C3F3C2030B9A93423FF45DAE2D
S3150800BD00019BABE79BF81330C3F3C2030C998B4234
S3150800BD103FF456AE019B5CE79BF81330C3F3C203AE
S3150800BD200D998B423FF44FAE019B06E79BF8133003
S3150800BD30C3F3C2030E9A93423FF448AEDDF804906B
S3150800BD4009F101095FFA89F9B9F10F0F3FF7CCAE8E
S3150800BD50C9EBC9035B441B7BC3F3C2039342EFD110
S3150800BD60B9F1000F3FF4C0AECDF84090C9EBC90356
S3150800BD705B441B7B13F0400F3FF436AEC9EBC90397
S3150800BD805B441B7B03F007031693DDF804A0CDF88C
S3150800BD90209057469A4693E69BF81330C3F3C2039E
S3150800BDA053453FF446AE019F0137FFB20F2F3FF7C9
S3150800BDB010AEC7EBC7035B441B7BC3F3C2035345F3
S3150800BDC0F2D1002F3FF432AE0297C7EBC7035B44AC
S3150800BDD01B7B13F0400F3FF466AEC7EBC7035B440B
S3150800BDE093F80C8008F00708019D43E69BF813308A
S3150800BDF0C3F3C20343453FF41EAE019D0135EDB2C0
S3150800BE000F2D3FF748AEC5EBC5035B441B7BC3F359
S3150800BE10C2034345F2D1002D3FF43DAEA946C5EB1A
S3150800BE20C5035B441B7B13F0400F3FF410AEC5EB14
S3150800BE30C5035B441E7B06F00706019C1BE09BF8C6
S3150800BE401330C3F3C203B3423FF4F7AD019C013488
S3150800BE50E4B20F2C3FF7F3ADC4EBC4035B441B7B82
S3150800BE60C3F3C203B342F2D1002C3FF4E8AD214636
S3150800BE705846FFF7EFFC631EDBB20E2BDFD80F2CFC
S3150800BE803FF7DDADC4EBC4035B441B7BC3F3C203BE
S3150800BE90B342DCD1E8E770472DE9F041412911D0DA
S3150800BEA0C37C8B4237D002221346C3EBC303034439
S3150800BEB01B7B8B421AD00132D2B213460F2AF4DD0D
S3150800BEC0BDE8F0810246012300241E46051DD474F0
S3150800BED016755475C3EBC30101448D6001330732EF
S3150800BEE0102BF4D10023C371BDE8F0818AB1054651
S3150800BEF01746C2EBC20303441B7B13F0400F14D052
S3150800BF00C2EBC20283181E7B06F007060124A04670
S3150800BF102FE0BDE8F0810122E9E7444625E0EB7908
S3150800BF20B34204BF03F1FF33EB71C7EBC707EB1945
S3150800BF3000221A73012159739A7304359D60BDE86E
S3150800BF40F081EB7CC3F3C203B342E6D04446013426
S3150800BF50E4B20F2CE3DCC4EBC4032B441B7BC3F312
S3150800BF60C203B342F3D1002CD9D021462846FFF7A5
S3150800BF7071FC631EDBB20E2BE3D80F2CCFDCC4EBAF
S3150800BF80C4032B441B7BC3F3C203B342DFD1EAE7E6
S3150800BF902DE9F84310F1080600F0AA808468002C01
S3150800BFA000F0A880837311F0800F40F0AB80072A59
S3150800BFB000F3A880C47C44B302252C46C4EBC40411
S3150800BFC00444247B34B10135EDB22C460F2DF5DD42
S3150800BFD0D42590E0002D00F09580C1B9C5EBC505C4
S3150800BFE0054401242C73C27CA24244D002210A468D
S3150800BFF0C2EBC2020244127BA24219D00131C9B275
S3150800C0000A460F29F4DDD62575E00125E5E7002760
S3150800C0103C4661F3C50467F3861462F30204C5EB74
S3150800C020C50505442C73E4B2002CDCD1D42562E0A6
S3150800C030002963D0C1EBC101711861D007468B7125
S3150800C040234600221146FFF7DDFB0546002852D09D
S3150800C050412C12D0FB7CA34234D002221346C3EBF8
S3150800C060C3033B441B7BA3421AD00132D2B2134608
S3150800C0700F2AF4DD3FE00121DCE73A4601230020E0
S3150800C0801E463C1DD07416755075C3EBC301394462
S3150800C0908C6001330732102BF4D10023FB712AE0A0
S3150800C0A04AB39046C2EBC2033B441B7B13F0400FD6
S3150800C0B012D0C2EBC202BB181E7B06F0070601248B
S3150800C0C0A14639E00122ECE74C4631E0FB79B34260
S3150800C0D004BF03F1FF33FB71C8EBC80807EB08037D
S3150800C0E000221A73012159739A73381D986002E069
S3150800C0F0D62500E0D7252846BDE8F883D625FAE7F1
S3150800C100D625F8E7D425F6E7FB7CC3F3C203B3428A
S3150800C110DAD04C460134E4B20F2CD7DCC4EBC403A6
S3150800C1203B441B7BC3F3C203B342F3D1002CCDD0EF
S3150800C13021463846FFF78EFB631EDBB20E2BE3D88B
S3150800C1400F2CC3DCC4EBC4033B441B7BC3F3C20301
S3150800C150B342DFD1EAE72DE9F04F8DB005460291EB
S3150800C1600392994600218DF8181008238DF8193086
S3150800C1700B460F2262F387038DF81A3003681B6893
S3150800C1809847002800F092800446066806AB0360CC
S3150800C19080F8069007AB0093122300221146284622
S3150800C1A0FFF7DFFA26608046002840F08180BDF858
S3150800C1B024300493BDF826B09DF8203005939DF8E9
S3150800C1C021A0044600270EE0CDF80090039B029AB2
S3150800C1D021462846FEF7E8FED12825D10134E4B2E7
S3150800C1E027460F2C24DC05EB8706B06F0028F5D010
S3150800C1F003681B6998470028F0D1B06F03681B6A6B
S3150800C200514698470028E9D0B06F03689B695A469B
S3150800C210049998470028D7D1B06F0368DB69059958
S3150800C22098470028D0D1D9E70F2FD8BF80463FDDE1
S3150800C230444600264F460BE0B06F03689B695A4692
S3150800C2400499984710B30134E4B226460F2C25DC2E
S3150800C25005EB8606B06F0028F5D003681B6998477A
S3150800C2600028F0D1B06F03681B6A5146984700282A
S3150800C270E2D10097039B029A21462846FEF794FED0
S3150800C28000F0F703D12BDED0804611E0B06F0368CB
S3150800C290DB69059998470028D5D1EAE73B46039A12
S3150800C2A002992846FFF774FE804601E04FF0D6084B
S3150800C2B040460DB0BDE8F08F10B50446F821FEF7EC
S3150800C2C0D7FE00F0C00040282DD007D9802811D00D
S3150800C2D0C0280ED10122204B1A7010BD40B9D122B8
S3150800C2E0D8212046FEF73EFE00221B4B1A7010BDD1
S3150800C2F010BD10BDD8212046FEF7BAFE10F0020F79
S3150800C30008D1C922D8212046FEF72CFE0222124B5C
S3150800C3101A7010BDCB22D8212046FEF723FE032231
S3150800C3200D4B1A7010BDD8212046FEF7A1FE10F05D
S3150800C330020F08D1CB22D8212046FEF713FE03228E
S3150800C340054B1A7010BDC922D8212046FEF70AFEF1
S3150800C3500222014B1A7010BD40DA00202DE9F04187
S3150800C36007464FF400516B4803F0B2FB38B16A4BED
S3150800C3701B78032B40D8DFE803F01A142926C821B6
S3150800C3803846FEF775FE10F0200F05D10022C821A9
S3150800C3903846FEF7E7FDEAE73846FFF78DFF202225
S3150800C3A0F5E713225D4B1A704FF0000816E05B4B59
S3150800C3B01B7803F0F003102B21D01122574B1A706B
S3150800C3C04FF000080AE04FF0010801E04FF00008BE
S3150800C3D0524B1B7803F0F003102B05D007F17406B7
S3150800C3E007F1B40534460FE002F0B4FC4B4BC830F5
S3150800C3F0586020221A70F1E74FF00008EEE74FF078
S3150800C4000008EBE7AC4207D054F8040F0028F9D02F
S3150800C4100368DB689847F5E7404B1B78402B45D007
S3150800C42007D8202B2ED0302B36D0112B17D0BDE8AD
S3150800C430F081512B51D0802B59D0502BF7D1C821E0
S3150800C4403846FEF715FE10F0400FF0D0334C512356
S3150800C450237002F07FFC14306060BDE8F081002391
S3150800C46087F8B83004E003689B689847A64204D06A
S3150800C47056F8040F0028F6D1F8E71222274B1A704F
S3150800C480BDE8F08102F066FC244B5B68C31A002BFA
S3150800C490CDDB3022214B1A700122E8213846FEF7FF
S3150800C4A061FD40221D4B1A70BDE8F081E82138462F
S3150800C4B0FEF7DEFD10F0010FB9D1D8213846FEF798
S3150800C4C0D7FD40F00802D2B2D8213846FEF74AFD19
S3150800C4D05022124B1A70BDE8F08102F03BFC0F4B5C
S3150800C4E05B68C31A002BA2DB80220C4B1A704346EA
S3150800C4F0002211463846FFF72EFE30B1D22896D0D4
S3150800C500A022064B1A70BDE8F0819022034B1A70E0
S3150800C5108DE700BF0008024040DA00203C0A0020F0
S3150800C5200368D3B130B40479CCB113889BB10B68D6
S3150800C5301D7843791B1B0468E5540379013B037195
S3150800C5401388013B13800B6801330B60047934B1FF
S3150800C5501388002BEBD1002004E0002070474379B4
S3150800C5600371012030BC70477F281BD981B942F27C
S3150800C570AC03984213D00C4A012332F8021F8142B9
S3150800C58003D001339BB2802BF7D18033D8B27047E2
S3150800C590FF2806D88038044B33F81000704700236C
S3150800C5A0F3E70020704700BFB8F70208612812D0E9
S3150800C5B00A4901226223984205D0013231F8023F26
S3150800C5C0002BF8D105E028B1054B03EB4202B2F87F
S3150800C5D0E002704770470022F6E700BFBAF8020883
S3150800C5E0B8F7020808B520F0A3FE08BD08B520F084
S3150800C5F0A7FE08BD08B5044B1A1803EB80035B6851
S3150800C6005B68107A984708BD640A002008B5084B8D
S3150800C6101B5C0BB1002008BD054B01221A541A18E1
S3150800C62003EB800043681B68107A984708BD00BF73
S3150800C630640A002038B5044C251804EB80046068A9
S3150800C6408468287AA04738BD640A002038B5044CA7
S3150800C650251804EB80046068C468287AA04738BDAA
S3150800C660640A002010B5044B1C1803EB80035B68B2
S3150800C6701B69207A984710BD640A0020002070477D
S3150800C6803AB101388A1811F8013B00F8013F914286
S3150800C690F9D1704722B1821800F8011B8242FBD1FA
S3150800C6A070470000F0B51A4B002632464FF0010ECF
S3150800C6B01C68E4B1D0F80052AC4209D001320C3300
S3150800C6C0022AF5D10EBB02290CBF00201220F0BDAC
S3150800C6D05D68D0F80842A542F0D11D89B0F8064237
S3150800C6E0A542EBD1022AEDD019B11020F0BD76464D
S3150800C6F0E4E702EB4202064B03EB82025389B3F5E9
S3150800C700807F0CBF10200020F0BD0020F0BD00BFC8
S3150800C710440A0020F0B4D0F80052284A00231468CE
S3150800C720AC420CD001330C32022BF8D1234B1B68D8
S3150800C730002B3BD0214BDB68BBB1002034E05768A7
S3150800C740D0F80842A742EDD11689B0F80642A642AB
S3150800C750E8D1022BEAD0C1B103EB4302174901EB3A
S3150800C7608202528922B300201EE00123134E03EBF6
S3150800C77043029200B418B550D0F808226260B0F8A7
S3150800C7800622228100226281A9B903EB43020B49E2
S3150800C79001EB82025189013189B203EB4300074A52
S3150800C7A002EB80025181581CF0BC70470023DDE77C
S3150800C7B04FF48071F1E74FF48071EEE7440A0020E8
S3150800C7C00138012801D90220704700EB4003104ABE
S3150800C7D002EB83035B89B3F5807F0BD08BB1013BFA
S3150800C7E09BB200EB40020A4901EB8202538143B136
S3150800C7F00020704700EB4003054A02EB8303002242
S3150800C8005A8100EB400083000020014AD05070474F
S3150800C810440A0020D0F82422131D490AD0F8000241
S3150800C82090F80202B1FBF0F1506848B1814205D395
S3150800C830091A53F8080F20B18842F9D958680844EC
S3150800C84070477047CA7E8B7E43EA022390F800221F
S3150800C850032A01D018467047487D0A7D42EA00221D
S3150800C86043EA0243F6E7024600F10B010020C30142
S3150800C87043EA500312F8010B50FA83F3D8B28A42FE
S3150800C880F5D170470168F1B110B40C781F2C11D995
S3150800C8903A2C21D00A4612F8013F1F2B0CD93A2B05
S3150800C8A0F9D14B1C9A4211D1302C12D102310160B8
S3150800C8B0002005E023460A463A2B18BF0020F0D090
S3150800C8C05DF8044B70474FF0FF3070474FF0FF306C
S3150800C8D0F6E74FF0FF30F3E70A46E2E790F804324E
S3150800C8E00BB9002070472DE9F0410446D0F83052C4
S3150800C8F0074601232A46014690F80102FFF7A6FEDD
S3150800C900F8B9002384F80432D4F82432EB1AD4F8A0
S3150800C9101C22934218D294F80362012E17D94FF0BD
S3150800C9200108D4F81C321D4443462A46394694F871
S3150800C9300102FFF78BFE013E012EF2D10020BDE871
S3150800C940F0810120BDE8F0810020BDE8F0810020DB
S3150800C950BDE8F08170B5D0F830328B4216D0044667
S3150800C9600D46FFF7BBFF064608B1304670BD0123EA
S3150800C9702A46214694F80102FFF75CFE00281CBFF0
S3150800C98001264FF0FF35C4F83052EEE70026ECE7F3
S3150800C99010B50446002380F804324FF0FF33C0F880
S3150800C9A03032FFF7D7FF08B1032010BD94F8FF21F6
S3150800C9B094F8FE3143EA02231BB2174A934201D088
S3150800C9C0022010BD94F8392094F838301B0443EA45
S3150800C9D0026394F83620134394F8372043EA022377
S3150800C9E023F07F430D4A934213D094F8553094F8B8
S3150800C9F05400000440EA036094F85230184394F84F
S3150800CA00533040EA032020F07F40801A18BF0120E7
S3150800CA1010BD002010BD00BF55AAFFFF46415400B7
S3150800CA20D8B108B5D0F80032CBB193F8001209B9DD
S3150800CA30092008BDB3F80612B0F80422914201D0C5
S3150800CA40092008BD93F80102FFF7D4FD00F00100A4
S3150800CA5000280CBF0020092008BD092070470920BE
S3150800CA6008BD00002DE9F04184B0064617460023AC
S3150800CA7003600846FFF706FF051EC0F2B4819E4B09
S3150800CA8003EB85039C69002C00F0B181346094F8AF
S3150800CA90003283B194F80102FFF7ACFD10F0010FE4
S3150800CAA009D1002F00F0A58100F0040000280CBF72
S3150800CAB000200A2098E1002384F80032E8B284F8BE
S3150800CAC00102FFF7A3FD10F0010F01D003208BE14F
S3150800CAD027B110F0040F01D00A2085E10021204675
S3150800CAE0FFF756FF0346012806D00026032B00F061
S3150800CAF082819BB30D2077E123466D4604F1400001
S3150800CB006946002705E03A4641F8042B103383426C
S3150800CB1012D093F8C221002AF5D093F8C96193F888
S3150800CB20C821120442EA066293F8C661324393F8B2
S3150800CB30C76142EA0622E7E704AF4FF0020807E0BA
S3150800CB4031462046FFF724FF034638B1AF42CDD021
S3150800CB5055F8046B002EF3D14346F7E7227BE37AB8
S3150800CB6043EA02231BB2B3F5007F01D00D203BE157
S3150800CB70E37DA27D52EA03220DD194F8273094F87A
S3150800CB802620120442EA036294F824301A4394F8E1
S3150800CB90253042EA0322C4F81C22217C84F80312B9
S3150800CBA04B1EDBB2012B01D90D201DE1677B84F8F2
S3150800CBB002720FB90D2017E17B1E3B4201D00D20F2
S3150800CBC012E1A37C607C40EA0320A4F8080210F076
S3150800CBD00F0F40F01281257DE37C53EA05230DD122
S3150800CBE094F8235094F822301B0443EA056394F81A
S3150800CBF020502B4394F8215043EA052394F80FE07C
S3150800CC00A57B55EA0E2500F0FA8002FB01FC05EB30
S3150800CC10101101EB0C0E7345C0F0F380A3EB0E0365
S3150800CC20B3FBF7F3002B00F0EE8040F6F5718B426C
S3150800CC3094BF012102214FF6F577BB4200F2ED8041
S3150800CC400233C4F81832C4F820623544C4F82452B2
S3150800CC500EEB0607C4F82C7203292DD1002840F0E4
S3150800CC60D48094F82F0094F82E10090441EA006144
S3150800CC7094F82C00014394F82D0041EA0021C4F8E9
S3150800CC8028129B0003F2FF13B2EB532FC0F0BF80AC
S3150800CC904FF0FF33C4F81032C4F80C32802384F8FE
S3150800CCA0053294F8312094F8303043EA02231BB257
S3150800CCB0012B23D0032173E0002800F0AA806544E5
S3150800CCC0C4F8285202290FBF5B0003EB430003F0A8
S3150800CCD0010303EB500303F2FF13B2EB532FC0F02B
S3150800CCE09A804FF0FF33C4F81032C4F80C32802310
S3150800CCF084F8053254E000BF440A0020711C20461F
S3150800CD00FFF728FE002866D1002384F8053294F838
S3150800CD10FF2194F8FE3143EA02231BB2454A9342A7
S3150800CD205BD1E278A3781B0443EA026322781343B3
S3150800CD30627843EA0223404A934250D194F8E721A5
S3150800CD4094F8E6311B0443EA026394F8E42113439A
S3150800CD5094F8E52143EA0223384A934241D194F8EC
S3150800CD60EB2194F8EA311B0443EA026394F8E821BC
S3150800CD70134394F8E92143EA0223C4F8103294F8DD
S3150800CD80EF2194F8EE311B0443EA026394F8EC2190
S3150800CD90134394F8ED2143EA0223C4F80C32032125
S3150800CDA084F80012264A938B01339BB29383A4F826
S3150800CDB006320023C4F814321368A34202D10022B3
S3150800CDC01F4B1A601E4BDB689C4202D100221C4B8B
S3150800CDD0DA60002008E00321E2E70321E0E7032107
S3150800CDE0DEE70321DCE70B2004B0BDE8F0810C2068
S3150800CDF0FAE70020F8E70120F6E70D20F4E70D2012
S3150800CE00F2E70D20F0E70D20EEE70D20ECE70D2008
S3150800CE10EAE70D20E8E70D20E6E70233C4F8183202
S3150800CE20C4F820623544C4F824520EEB0601C4F84F
S3150800CE302C1213E755AAFFFF5252614172724161E3
S3150800CE40440A00202DE9F84301F10904D0F810320C
S3150800CE50002B4DD0D0F814727D1E00224FF02E08FC
S3150800CE604FF0E50C4FF0100914E0661C84F80080BA
S3150800CE70A3F14104E4B2192C21D897F80CE0344602
S3150800CE804E4616EA0E0F1CBF2033DBB22370013460
S3150800CE900B2A16D0013215F8013F202BF8D0052BA6
S3150800CEA05BD0092AE1D0A3F14106F6B2192EEDD8D6
S3150800CEB097F80CE0082A8CBF10260826E1E73446C6
S3150800CEC0E4E7FB7A0B72FA7FBB7F1B0443EA026333
S3150800CED03A7F13437A7F43EA02230B607A7E3B7ECE
S3150800CEE043EA02238B80FA7DBB7D43EA0223CB808B
S3150800CEF0002323708F69CFB3D0F8103203B3CC69FF
S3150800CF00FCB1B0F824224FF6FF739A421DD0D0F830
S3150800CF102082B8F80000D0B10D467E1E0024A14636
S3150800CF204946FFF721FBA0B1EB69013BA34212D9A1
S3150800CF30013406F8010F38F814000028F0D100E093
S3150800CF40002400233B55BDE8F8830024F9E70024B4
S3150800CF50F7E70024F5E70024F3E7092A01D063463A
S3150800CF6094E784F80080013463468FE7BDE8F883C8
S3150800CF7010B50446FFF7B2FC034660B994F80032D0
S3150800CF80032B0AD00022114694F80102FFF76AFB28
S3150800CF90031C18BF0123184610BD94F80532012B4F
S3150800CFA0F0D14FF4007200212046FFF773FB55239A
S3150800CFB084F8FE31AA2384F8FF3152232370637064
S3150800CFC06123A3704122E270722184F8E41184F887
S3150800CFD0E51184F8E62184F8E731D4F8103284F8AC
S3150800CFE0E831C3F3072284F8E9211A0C84F8EA2108
S3150800CFF01B0E84F8EB31D4F80C3284F8EC31C3F309
S3150800D000072284F8ED211A0C84F8EE211B0E84F809
S3150800D010EF31D4F820220132C4F830220123214608
S3150800D02094F80102FFF712FB002384F80532A9E7FA
S3150800D0300239D0F81832023B99423DBF90F80232C5
S3150800D040D0F82C0201FB030000207047012965D99E
S3150800D050F8B5D0F81832994262D20C46064690F8CE
S3150800D0600032022B2CD0032B3DD0012B01D00120FE
S3150800D070F8BD01EB5105D0F8241201EB5521FFF755
S3150800D08069FC10B14FF0FF30F8BD6F1CC5F30805F9
S3150800D090755DD6F8241201EB57213046FFF75AFC86
S3150800D0A010B14FF0FF30F8BDC7F30807F05D45EA49
S3150800D0B0002014F0010F14BF0009C0F30B00F8BDDF
S3150800D0C0D0F8241201EB1421FFF744FC10B14FF0FD
S3150800D0D0FF30F8BD610001F4FF7173185B78705C6E
S3150800D0E040EA0320F8BDD0F8241201EBD411FFF76B
S3150800D0F031FC10B14FF0FF30F8BDA10001F4FE710C
S3150800D1007218D07893781B0443EA0063705C18435E
S3150800D110537840EA032020F07040F8BD012070479C
S3150800D1200120F8BDF8B50546A0F80612D0F8084261
S3150800D130012C4FD00E46D0F80032D3F8182294426C
S3150800D14001D30220F8BD74B993F80022032A05D04A
S3150800D150B3F8082296420DD30220F8BDD3F8282248
S3150800D160002AF5D0144693F802723F01BE421DD339
S3150800D170F61B07E0D3F82802C5F80C42E0B90220EE
S3150800D180F8BD1E462146D5F80002FFF75FFF0446A4
S3150800D190B0F1FF3F20D0012820D9D5F80032D3F8C6
S3150800D1A0183298421CD2F31BBE42EAD22146D5F861
S3150800D1B00002FFF73DFFDFE700EB1610C5F8100287
S3150800D1C006F00F06D5F8003203EB4616C5F81462CA
S3150800D1D00020F8BD0220F8BD0120F8BD0220F8BDE8
S3150800D1E00220F8BD2DE9F843012940F28C80D0F8D9
S3150800D1F01832994201D3022786E016460C460546A0
S3150800D20090F80032022B4DD0032B5FD0012B01D0B2
S3150800D210022779E001EB5108D0F8241201EB5821D6
S3150800D220FFF798FB074600286ED108F10109C8F3F5
S3150800D230080814F0010F1DD015F8083003F00F0385
S3150800D24043EA061305F80830012385F80432D5F8B1
S3150800D250241201EB59212846FFF77CFB002856D1FA
S3150800D260C9F30809C6F3071205F80920012385F84A
S3150800D270043249E005F80860012385F80432D5F838
S3150800D280241201EB59212846FFF764FB002840D1F8
S3150800D290C9F3080915F8093023F00F03C6F303226A
S3150800D2A01A43E1E7D0F8241201EB1421FFF752FBE9
S3150800D2B0074648BB610001F4FF716E542944C6F362
S3150800D2C007224A70012385F804321DE0D0F824129B
S3150800D2D001EBD411FFF73EFB0746A8B9A10001F4FC
S3150800D2E0FE716B18DA78120602F0704232436A54FD
S3150800D2F0C2F307215970110C9970120EDA700123C6
S3150800D30085F8043200E002273846BDE8F883074668
S3150800D310FAE70746F8E7F8B505460F4649B9D0F8DB
S3150800D3200C62A6B1D0F818329E4228BF01263446B0
S3150800D3301CE0FFF78BFE0346012849D9B0F1FF3FF1
S3150800D3404BD0D5F81822904247D33E46EFE7012640
S3150800D350EDE721462846FFF779FE034678B1B0F196
S3150800D360FF3F3AD0012838D0B44235D00134D5F839
S3150800D37018329C42EDD3012E2CD90224E9E76FF02E
S3150800D380704221462846FFF72DFF0346D0B98FB9CC
S3150800D390C5F80C42D5F81032B3F1FF3F1FD0013B58
S3150800D3A0C5F8103295F8053243F0010385F80532C1
S3150800D3B0234612E0224639462846FFF713FF03465E
S3150800D3C00028E5D0012B0CBF4FF0FF33012304E002
S3150800D3D0012302E0002300E000231846F8BD234697
S3150800D3E0FBE72DE9F843B0F806420134A3B213B9B6
S3150800D3F00420BDE8F883D0F8103213B90420BDE83C
S3150800D400F8830E46054614F00F0716D10133C0F807
S3150800D4101032D0F80C1241B9D0F80032B3F80832FD
S3150800D4209C420AD30420BDE8F883D0F8000290F89D
S3150800D4300232013B13EA14180AD0A5F80642D5F8B9
S3150800D440003203EB4713C5F814320020BDE8F88311
S3150800D450FFF7FCFD8146012857D9B0F1FF3F57D0A9
S3150800D460D5F80002D0F81832994544D316B90420E5
S3150800D470BDE8F883D5F80C12FFF74DFF814610B9C1
S3150800D4800720BDE8F883012845D0B0F1FF3F45D015
S3150800D490D5F80002FFF722FA002842D14FF40072AD
S3150800D4A00021D5F80002FFF7F5F8D5F800624946DD
S3150800D4B03046FFF7BDFDC6F830020126D5F8003222
S3150800D4C093F80222904510D283F80462D5F8000238
S3150800D4D0FFF704FA40BBD5F80022D2F83032013300
S3150800D4E0C2F8303208F10108E8E7D3F83022A2EB97
S3150800D4F00802C3F83022C5F80C924946D5F800024E
S3150800D500FFF796FDC5F8100297E70220BDE8F883F5
S3150800D5100120BDE8F8830220BDE8F8830120BDE8B4
S3150800D520F8830120BDE8F8830120BDE8F8830000F0
S3150800D5302DE9F04F85B005460021FFF7F3FD834638
S3150800D54000285AD14FF6FF73A5F824324FF0FF0A88
S3150800D55057469946D04609E0A5F824924746002141
S3150800D5602846FFF73EFF8346002846D1D5F8101215
S3150800D570D5F80002FFF7EEF9834600283DD1D5F825
S3150800D58014422678002E00F08380E52EE4D0E37A54
S3150800D59003F03F0213F0080F17D00F2ADCD1D5F895
S3150800D5A020B2BBF1000FDAD016F0400F29D094F85C
S3150800D5B00DA006F0BF06B5F80632A5F82432637B3F
S3150800D5C00193534522D04746C9E70F2AE7D027B922
S3150800D5D02046FFF748F982450FD0D5F81832DA7A8F
S3150800D5E012F0010F50D104F10B0014F8011B13F8C7
S3150800D5F0012B914248D1A042F7D1584605B0BDE863
S3150800D600F08FB74218BF4746A9D1D8E7237823F049
S3150800D6104003013B03EB430203EB820302931E4FD5
S3150800D62007F10D0A012011E01846FEF7BFFF039027
S3150800D630029BFE2B15D85A1C02923BF81300FEF7E4
S3150800D640B5FF039B83420CD157450ED017F8012B23
S3150800D650A3185978A35C43EA01230028E4D14B4573
S3150800D660F2D0DDF804A0474679E7237813F0400F97
S3150800D67005D020B1029B3BF81330002BF1D1013EB7
S3150800D680F7B2DDF804A06AE7A5F82492474666E7EC
S3150800D6904FF0040BB1E700BF78FC02082DE9F04F04
S3150800D6A083B005468A460B782F2B14D05C2B12D0F4
S3150800D6B0D0F80032D3F81432C0F808329AF800309D
S3150800D6C01F2B0FD800212846FFF72CFD0346002202
S3150800D6D0C5F8142276E00AF1010A0023C5F80832D3
S3150800D6E0ECE79A46D046534613F8010B2F28F8D094
S3150800D6F05C2808BF9A46F5D0D5F8206280B21F2864
S3150800D70040F254812F2800F057815C2800F064818C
S3150800D710B71E0124A1464FF02A0B13E0002B50D167
S3150800D72027F8022F631C1AF8010F1F2840F24081C0
S3150800D7302F2800F043815C2800F04081B3F5807FF4
S3150800D7403FD01C464946FEF70FFF0246002838D050
S3150800D7507F28E5D8222800F00F815B46A84998B2B1
S3150800D7609042DBD011F8013F002BF8D1D8E7338877
S3150800D7702E2B40F02E81002326F81430D5F81822D7
S3150800D780A34234BF2E212021D15401330B2BF5D1CE
S3150800D790D5F8183247F02007DF729DE073882E2BE4
S3150800D7A040F0178133882E2B40F01381E3E7013CC4
S3150800D7B000F0E28032F8023D202BF8D02E2BF6D06E
S3150800D7C024B90623184603B0BDE8F08F4FEA44088B
S3150800D7D04FF0000926F814900B222021D5F81802DC
S3150800D7E0FEF758FFB11E4B4600E0013331F8022F11
S3150800D7F0202AFAD02E2AF8D00BB147F00307A8F151
S3150800D800020806EB080236F808102E2905D0013C56
S3150800D81003D032F8021D2E29F9D14FF0080B002249
S3150800D8200192914605E0A04500F0D98047F003072C
S3150800D830434603F1010836F8130040B32028F5D013
S3150800D8402E28F0D0019B5B4517D2A04500F0C78073
S3150800D8507F2867D82B2873D02C236A4A99B281422D
S3150800D8607AD012F8013F002BF8D1A0F141039BB200
S3150800D870192B74D849F0020965E0BBF10B0F45D0A6
S3150800D880A04500F0AF8047F0030740F2AB80D5F81B
S3150800D89018321A78E52A42D0BBF1080F04BF4FEABE
S3150800D8A089095FFA89F909F00C030C2B61D009F094
S3150800D8B00302032A5DD017F0020F0AD109F0030903
S3150800D8C0B9F1010F08BF47F01007042B08BF47F04E
S3150800D8D00807D5F81832DF722846FFF729FED5F86B
S3150800D8E01832DA7A0346002848D112F0040F7FF47A
S3150800D8F069AFD5F81412CB7A13F0100F54D0D5F8B7
S3150800D9000002FEF79FFFC5F80802EBE647F003079B
S3150800D910D5F818321A78E52AC5D14FF00B0B05222F
S3150800D9201A70B9E70021FEF71FFE0346002863D0E8
S3150800D930354A134413F8700C47F00207002889D1BA
S3150800D94047F003075F20D5F8183201990A4658545C
S3150800D9504346013201926CE7002BF1D185E7A0F12D
S3150800D96061039BB2192BEED849F00109203880B221
S3150800D970E9E747F002079EE7062323E7042B7FF42F
S3150800D98021AF12F0200F09D00023C5F80832C5F8D8
S3150800D990143212F0040F3FF4A5AE13E702F00402A6
S3150800D9A0002A08BF05230DE705230BE701230024FA
S3150800D9B008EB030A042704E00123002408EB030A02
S3150800D9C00027012C3FF4D3AE022C3FF4E7AE002C1F
S3150800D9D0D2D006EB4402EDE601230024EEE7BBF1C4
S3150800D9E00B0F93D04FEA89095FFA89F923464FF05E
S3150800D9F00B0B082201921CE747F00207A0E700BFBD
S3150800DA00D5760308E176030878FC02082DE9F04F7D
S3150800DA1089B00446D0F81852D0F820920C2229462C
S3150800DA2005A8FEF72DFE9DF81F3013F0200F04D031
S3150800DA300626304609B0BDE8F08F13F0010F7AD0FC
S3150800DA400023EB72C4F820320B2205A92846FEF7FC
S3150800DA5017FE4FF0010843464FF07E0A202700E0E4
S3150800DA6043460DF11306072203F00F0000F13001BB
S3150800DA70392988BF00F13701013A06F801191B094F
S3150800DA80F2D108A9114401F814AC5AB12978202911
S3150800DA900BD0294601339A4206D011F8010F2028E7
S3150800DAA0F8D102E0134600E013462B4405E0394658
S3150800DAB003F8011B591B072907D8072AF7D808A90D
S3150800DAC0114411F8141C0132F2E72046FFF730FD25
S3150800DAD0064628BB08F10108B8F1640F1ED00B22D0
S3150800DAE005A92846FEF7CCFDB8F1050FB8D9A9F166
S3150800DAF00206434636F8022F002AB2D0102102F059
S3150800DB00010000EB4303520813F4803F1CBF83F463
S3150800DB10883383F021030139F1D1EBE7072688E73B
S3150800DB20B8F1640F00F09F80042882D19DF81F3059
S3150800DB30EB72C4F820929DF81F3013F0020F1CD028
S3150800DB40B9F80030BBB10023013339F8022F002A97
S3150800DB50FAD103F11905684BA3FB0535AD08002179
S3150800DB602046FFF7DFFA0646002840F09A8000278D
S3150800DB704FF001080FE00023EBE70125EFE7013737
S3150800DB80BD4200F0928041462046FFF72AFC064631
S3150800DB90002840F08680D4F81012D4F80002FEF768
S3150800DBA0D9FE064600287CD1D4F814321B78E52B1A
S3150800DBB0E5D0002BE3D00027E5E7B4F80612491BA9
S3150800DBC02046FFF7AFFA064600287FF432AFD4F8AE
S3150800DBD01802FEF748FE0090002701971BE07146E1
S3150800DBE04AE04FF6FF72934202D038F811300BB96B
S3150800DBF049F0400980F80090D4F80032012283F8F1
S3150800DC00042239462046FFF7ECFB064600287FF437
S3150800DC1010AF013D4BD0D4F81012D4F80002FEF72D
S3150800DC2099FE064600287FF404AFD4F82082D4F87B
S3150800DC3014025FFA85F99DF8003043734FF00F031D
S3150800DC40C37207738776C77609F1FF3101EB410383
S3150800DC5001EB8301294A02F10D0C019B4FF6FF7671
S3150800DC604FF0FF0A0BE00726E3E692F800E000F81B
S3150800DC700EA086448EF801A001326245B1D0B342A7
S3150800DC80F3D001F1010E38F81130117843540144EC
S3150800DC904FEA132B81F801B0002BA0D17146334609
S3150800DCA0EAE7042E08BF0726C3E6013D85D1D4F866
S3150800DCB01012D4F80002FEF74DFE064600287FF43F
S3150800DCC0B8AE20220021D4F81402FEF7E3FC0B229A
S3150800DCD0D4F81812D4F81402FEF7D2FCD4F8142299
S3150800DCE0D4F81832DB7A03F018031373D4F8003229
S3150800DCF0012283F804229CE64FECC44E78FC020805
S3150800DD00012932D9F8B504460E46D0F81832994298
S3150800DD1002D302221046F8BD002704E02E46D4F8A6
S3150800DD201832AB42F6D931462046FFF78FF9054639
S3150800DD30F0B101281ED0B0F1FF3F1DD03A4631465A
S3150800DD402046FFF74FFA02460028E3D1D4F81032EE
S3150800DD50B3F1FF3FE2D00133C4F8103294F805322C
S3150800DD6043F0010384F80532D8E7022210467047CB
S3150800DD700022CFE70222CDE70122CBE710B584B017
S3150800DD8001900091144604A840F8041DFEF77AFD98
S3150800DD9000282ADB194B03EB80039B6953B1174A0A
S3150800DDA01268934213D0154AD268934213D00022C0
S3150800DDB083F80022019BDBB1002283F800220F4A78
S3150800DDC002EB80008361012C09D000200EE00021BF
S3150800DDD00A4A1160E7E70021084AD160E7E700220E
S3150800DDE0694601A8FEF73EFE00E00B2004B010BD10
S3150800DDF0024B03EB800300209861F7E7440A0020F2
S3150800DE002DE9F047ADF5107D0191002800F0B980A5
S3150800DE10044615460023C0F8003202F01E0201A986
S3150800DE2086A8FEF71FFE0646002840F0AB804FF492
S3150800DE300070FEF7D7FB8046002800F0A88005F0A2
S3150800DE401F098E9003AB8C93019906A8FFF726FC51
S3150800DE508B9F8246002840F09C80002F00F0C980E6
S3150800DE6039F0010314BF0121002106A8FEF71AFCA8
S3150800DE70824615F01C0F5CD048B9FB7A13F0110FD7
S3150800DE8040F0CA8015F0040F0AD00826BAE0BAF1A5
S3150800DE90040F30D049F008098B9FBAF1000F38D12A
S3150800DEA019F0080F56D0FEF7E9FBB873C0F307233D
S3150800DEB0FB73030C3B74000E78740025FD723D77E6
S3150800DEC07D77BD77FD7739468698FEF7BBFCBD762C
S3150800DED0FD763D757D75869B012283F804220546ED
S3150800DEE0002835D0D3F830A201461846FFF708FFB8
S3150800DEF088B1064695E04E4B1B682BB14C4BDB6848
S3150800DF004FF0120A002BC5D106A8FFF77FFD8246FF
S3150800DF10C0E7564685E08698013DC0F80C52514642
S3150800DF20FEF718FD054698B14046FEF75FFB2E46FC
S3150800DF3028E0002872D1FB7A13F0100F70D115F083
S3150800DF40020F02D013F0010F6FD115F0080F01D0A0
S3150800DF5049F02009869BD3F83032C4F81C32C4F83D
S3150800DF60207239F0010314BF0121002106A8FEF72B
S3150800DF70D1FBC4F82802002843D04046FEF736FBFA
S3150800DF8011E0092630460DF5107DBDE8F08711260B
S3150800DF90F8E715F01C0F7FF47AAF4046FEF726FB2C
S3150800DFA0BAF1000F2BD184F80692002584F807529F
S3150800DFB0DDF8188239464046FEF744FCC4F81002DC
S3150800DFC0FA7FBB7F1B0443EA02633A7F13437A7FD7
S3150800DFD043EA0223C4F80C32C4F80852C4F81852AB
S3150800DFE0C4F82452C4F80082B8F80632A4F80432F9
S3150800DFF0C8E715F01C0F09D14FF0060ACDE75646BB
S3150800E000C0E702264046FEF7F1FABBE749F00809E1
S3150800E0108B9F4FF0060AC0E70726F3E7064600E09F
S3150800E02004264046FEF7E2FAACE70726F9E700BF02
S3150800E030440A00202DE9F04F83B004468846164668
S3150800E04099460023C9F80030FEF7EAFC019058B952
S3150800E05094F80732002B40F0F88094F8063213F053
S3150800E060020F05D107230193019803B0BDE8F08F8D
S3150800E070D4F80832F34202D2002E40F0BB80D4F81E
S3150800E0800832D4F80C22934288BFC4F80C3294F8AC
S3150800E090063243F0200384F80632E5E7D4F8243242
S3150800E0A0DBB32046FEF7B6FB0028E8D001283AD0B5
S3150800E0B0B0F1FF3F3CD0C4F81402D4F810320BB9C3
S3150800E0C0C4F8100294F8063213F0400F35D1D4F88C
S3150800E0D000A2D4F814125046FEF7AAFF05460028F7
S3150800E0E042D03D445FEA562B56D09AF8023207EBE7
S3150800E0F00B029A4288BFA3EB070B5B462A464146AA
S3150800E1009AF80102FEF7A2FA98BBD4F81812491B2E
S3150800E1108B4533D84FEA4B255EE0D4F814121046E7
S3150800E120FFF7F9F8C0E7022384F8073201939BE763
S3150800E130012384F80732019396E7D4F800020123F5
S3150800E140D4F81822214690F80102FEF77FFA30B972
S3150800E15094F8063223F0400384F80632B7E7012321
S3150800E16084F8073201937FE7022384F80732019384
S3150800E1707AE7012384F80732019375E74FF40072B2
S3150800E18008EB41212046FEF77BFA94F8063223F085
S3150800E190400384F80632BDE7D4F818329D4205D00C
S3150800E1A0D4F80822D4F80C329A4240D3C4F818524C
S3150800E1B0D4F80802C0F30800C0F50075B54228BFB8
S3150800E1C035462A4641462044FEF75AFA94F806325E
S3150800E1D043F0400384F80632A844D4F808322B44A6
S3150800E1E0C4F80832D9F800302B44C9F80030761B39
S3150800E1F03FF445AFD4F80812C1F30803002BD7D172
S3150800E200D4F8002292F80232013B03EA512313F0B4
S3150800E210FF077FF457AF00297FF440AFD4F8100208
S3150800E22000287FF443AF1046FFF775F83CE7012353
S3150800E2302A4621469AF80102FEF7FCF90028B5D0CD
S3150800E240012384F8073201930EE701930CE738B5EA
S3150800E2500446FEF7E5FB034608BB94F8062212F0CF
S3150800E260200F1CD012F0400F11D0D4F80002012361
S3150800E270D4F81822214690F80102FEF7E7F900289B
S3150800E2804AD194F8063223F0400384F80632D4F8CB
S3150800E2901C12D4F80002FEF75DFB034608B11846C7
S3150800E2A038BDD4F82052EB7A43F02003EB72D4F849
S3150800E2B00C322B77B4F80C321B0A6B77B4F80E3293
S3150800E2C0AB7794F80F32EB77D4F81032AB76C3F30A
S3150800E2D00722EA761B0C2B751B0A6B75FEF7CEF91F
S3150800E2E0A875C0F30723EB75030C2B76000E68762A
S3150800E2F00023AB74EB7494F8063223F0200384F8F9
S3150800E3000632D4F80032012283F80422D4F8000237
S3150800E310FEF72EFE0346C2E70123C0E710B5044602
S3150800E320FFF795FF034608B1184610BD2046FEF7CD
S3150800E33077FB03460028F7D1D4F82802FEF740FAFF
S3150800E34003460028F0D10022C4F80022ECE770B595
S3150800E350ADF5107D01900D46002201A986A8FEF7AD
S3150800E36081FB044618B120460DF5107D70BD4FF4AB
S3150800E3700070FEF737F90646A8B18E9003AB8C936A
S3150800E380019906A8FFF78AF9044630B98B9B43B171
S3150800E3901DB1294606A8FEF755FD3046FEF726F9B3
S3150800E3A0E1E70624F9E71124DDE72DE9F04FADF59D
S3150800E3B0117D0190FEF762F90546012201A986A89A
S3150800E3C0FEF750FB044620B120460DF5117DBDE849
S3150800E3D0F08F4FF40070FEF705F90646002800F0A6
S3150800E3E0C7808E9003AB8C93019906A8FFF756F960
S3150800E3F00346002800F0B780042840F0BC808C9BB8
S3150800E400DB7A13F0200F40F0B58000218698FEF7DE
S3150800E41082FF804648B1012801D1022406E0B0F106
S3150800E420FF3F08BF012476D000E0072424B1414607
S3150800E4308698FFF765FC97E08698FEF74FFA04463C
S3150800E4400028F4D1869F41463846FEF7F1FD04467A
S3150800E45000974FF4007200213846FEF71BF90B228D
S3150800E46020213846FEF716F94FF02E0987F8009056
S3150800E4701023FB72BD75C5F30723FB752B0C3B7682
S3150800E4802B0E7B7687F81A80C8F30723FB764FEAAC
S3150800E49018433B751B0A7B7520223946B818FEF7C8
S3150800E4A0EFF887F82190889B869A92F8001203293C
S3150800E4B053D087F83A30C3F3072287F83B201B0C62
S3150800E4C087F834301B0A87F83530869B93F8023272
S3150800E4D0EBB103F1FF395FFA89F909F10109A144A2
S3150800E4E04FF0010A4FF4007B8698671CC0F830424B
S3150800E4F080F804A2FEF7F2F90446002897D15A4696
S3150800E50000210098FEF7C6F83C464F45ECD106A810
S3150800E510FFF77CFA0446002C89D18B9B1022DA720D
S3150800E5209D75C5F30722DA752A0C1A762D0E5D76C7
S3150800E53083F81A80C8F30722DA764FEA184883F870
S3150800E54014804FEA182883F815808698012380F8E6
S3150800E5500432FEF70DFD044606E0D2F8282293425F
S3150800E56008BF0023A5E708243046FEF73FF82BE747
S3150800E570112429E706231C46F6E700002DE9F04F8B
S3150800E58089B00590012988BF132002D909B0BDE8D2
S3150800E590F08F0C46174605A8FEF774F90028C0F256
S3150800E5A08C82D54B03EB80039D69002D00F0878292
S3150800E5B0002385F80032C6B23046FEF727F810F079
S3150800E5C0010F01D00320E1E710F0040F01D00A2063
S3150800E5D0DCE706AA01213046FEF744F8002840F099
S3150800E5E07082069A7F2A40F26E82002C14BF4FF082
S3150800E5F000094FF03F09A2EB090206927B1E3B4237
S3150800E60004D11FB1B7F5007F16D219E04FF4FA61AD
S3150800E610B2FBF1F1B1F5806F29D2B8480023013376
S3150800E62030F8027FB942FAD3B54901EB4303B3F890
S3150800E630A870B7F5007F00D37F0A002F08BF01270F
S3150800E640802F28BF80270197B2FBF7F340F6F571B4
S3150800E6508B4200F246824FF6F5718B420AD803EBDD
S3150800E660430301335B0803334FF0010842E24FF4DA
S3150800E6700047E1E79F0007F207277F0A4FF00308E4
S3150800E680002300934FF0200A3BE207AA03213046F5
S3150800E690FDF7E8FF20B9079B013BB3F5004F01D30F
S3150800E6A001230793079A531E5B4452421340A3EB78
S3150800E6B00B030793B8F1030F19D01F44069AA2EB70
S3150800E6C00A03DB1B00995B1A0199B3FBF1F3039369
S3150800E6D0B8F1020F00F0F180B8F1010F40F0F380B5
S3150800E6E0B2F5803F34BFC3464FF0060B15E09A4497
S3150800E6F0029A1A440292069BA3EB0A03DB1B009AB2
S3150800E7009B1A019AB3FBF2F31A4603934FF6F57375
S3150800E7109A4240F2DA814FF00C0B002C40F0DB8075
S3150800E7204FF4007200212846FDF7B4FF012385F84F
S3150800E730BF3185F8C031002285F8C12185F8C2B1FC
S3150800E740FE2185F8C311069909EB010043F6C16459
S3150800E750B0FBF4F00790840844F03F0485F8C44100
S3150800E76085F8C5013F2085F8C60185F8C72185F8D3
S3150800E770C82185F8C92185F8CA11C1F3072085F88B
S3150800E780CB01080C85F8CC01090E85F8CD11552169
S3150800E79085F8FE11AA2185F8FF1129463046FDF7AE
S3150800E7A055FF002840F095814FF0F80B04954FF47B
S3150800E7B0007200212846FDF76DFF0B2251492846B5
S3150800E7C0FDF75EFF0023EB7202232B739DF80430DE
S3150800E7D06B7385F80EA0CAF3072A85F80FA00123E4
S3150800E7E02B74B8F1030F4FF000036B7418BF0223A4
S3150800E7F0AB74069BB3F5803F70D2EB74C3F3072363
S3150800E8002B7585F815B03F232B7600236B76FF22F0
S3150800E810AA76EB7685F81C906B77AB77EB77FDF7E6
S3150800E8202DFF0790B8F1030F70D185F84300C0F3A8
S3150800E830072385F84430030C85F84530000E85F823
S3150800E840460085F82470C7F3072385F825303B0C66
S3150800E85085F826303B0E85F82730022385F82C30BC
S3150800E860002385F82D3085F82E3085F82F300124C1
S3150800E87085F8304085F83130062285F8322085F84B
S3150800E8803330802385F84030292385F84230132217
S3150800E8901D4905F14700FDF7F3FE552385F8FE31BE
S3150800E8A0AA2385F8FF3123464A4629463046FDF70E
S3150800E8B0CDFE002857D0012068E640F6F573039987
S3150800E8C0994240F20481B2F5803F34BF4FF0040B01
S3150800E8D04FF0060B21E74FF0F00B67E785F820307D
S3150800E8E0C3F3072285F821201A0C85F822201B0E6F
S3150800E8F085F8233085E700BF440A002008FD020892
S3150800E90078FC0208E8760308F476030885F82700F9
S3150800E910C0F3072385F82830030C85F82930000E44
S3150800E92085F82A00AF75C7F30723EB75802385F8AA
S3150800E9302430292385F826301322874905F12B0030
S3150800E940FDF79EFE552385F8FE31AA2385F8FF318B
S3150800E95001234A4629463046FDF778FE002800F08E
S3150800E960E080012012E6012309F106022946304615
S3150800E970FDF76CFE4FF4007200212846FDF78AFE6B
S3150800E9806BF0FF0307932B70BDF81C301B0A6B70E6
S3150800E990BDF81E30AB709DF81F30EB70FF232B714E
S3150800E9A06B71AB71EB712B726B72AB720F23EB72DF
S3150800E9B0029A541C012329463046FDF747FE0028D3
S3150800E9C040F089804FF4007200212846FDF762FE68
S3150800E9D0012307939B462246079BBB420DD202F1B1
S3150800E9E0010A5B4604993046FDF730FE002874D1CB
S3150800E9F0079B013307935246EEE71446019B009A9C
S3150800EA00B8F1030F18BF1346224601271C4402F12A
S3150800EA10010A3B4604993046FDF718FE00285ED1E8
S3150800EA205246A245F3D1B8F1030F3DD152232B70BC
S3150800EA306B706123AB704122EA70722185F8E4118C
S3150800EA4085F8E51185F8E62185F8E731039A531E1E
S3150800EA5085F8E831531EC3F3072385F8E931531EB9
S3150800EA601A0C85F8EA211B0E85F8EB31022385F886
S3150800EA70EC31002385F8ED3185F8EE3185F8EF3174
S3150800EA80552385F8FE31AA2385F8FF31012309EBC2
S3150800EA90030229463046FDF7D9FD012309F107028D
S3150800EAA029463046FDF7D2FD002211463046FDF7CD
S3150800EAB0D9FD003018BF012068E50B2066E50C205B
S3150800EAC064E5012062E5012060E50E205EE50E2082
S3150800EAD05CE501205AE5012058E5012056E50120AC
S3150800EAE054E54FF6F5718B423FF6C4AD02335B0031
S3150800EAF04FF0020803F2FF135F0A202300934FF03A
S3150800EB00010A0AEB09030293009907EB010B9B44E0
S3150800EB10019BA3EB09035B449A42BFF4B6AD0E20F2
S3150800EB2034E54FF4007200212846FDF7B3FDB8F12D
S3150800EB30010F0A4B18BF6FF0FF0343EA0B03079355
S3150800EB402B70BDF81C301B0A6B70BDF81E30AB70FD
S3150800EB509DF81F30EB702BE70877030800FFFF00CE
S3150800EB60114B5B7ADBB2012B01D90120704730B417
S3150800EB700D4C657AEDB200236355657A04EB85057D
S3150800EB806860607A20440272627AD2B2501CC0B2BF
S3150800EB90607230320A703A224A702F228A70CB701D
S3150800EBA0184630BC704700BF640A002008B500222A
S3150800EBB0FFF7D6FF08BD00000D4B5B7A9BB10378C3
S3150800EBC0303BDBB20A4A02EB830252686AB1084A52
S3150800EBD002EB83010020486013441872537A013B04
S3150800EBE0DBB253727047012070470120704700BF9F
S3150800EBF0640A002008B50021FFF7DEFF08BD000003
S3150800EC0008B50122064B1A7006F072FC20B9044AB0
S3150800EC10137803F0FE031370014B187808BD00BF84
S3150800EC200000002008B50122064B1A7006F0A6FC63
S3150800EC3020B9044A137803F0FE031370014B1878C1
S3150800EC4008BD00BF0000002000B583B001934FF453
S3150800EC500073009352020023084606F03DFB00307D
S3150800EC6018BF012003B05DF804FB00B583B001931B
S3150800EC704FF40073009352020023084606F03EFB49
S3150800EC80003018BF012003B05DF804FB144B1B7855
S3150800EC9013F0010F01D003207047032903D8DFE8DA
S3150800ECA001F01D0413180420704710B596B01446D9
S3150800ECB0684606F06BFC129B5B0A139A43EAC2533A
S3150800ECC02360002016B010BD4FF400731380002097
S3150800ECD070474FF400731360012070470020704797
S3150800ECE00000002010B50446074B1868074BA3FB25
S3150800ECF00030800900F00CFB002221464FF0FF305F
S3150800ED0000F0BCFA002010BD04000020D34D6210AC
S3150800ED1008B50B4B1A6842F400721A601A6842F476
S3150800ED2080621A601A6842F480721A60032000F042
S3150800ED3093FA0020FFF7D6FF1CF040FD002008BD1F
S3150800ED40003C0240024A136801331360704700BF53
S3150800ED5074DA0020014B1868704700BF74DA002087
S3150800ED6010B582B00190FFF7F5FF0446FFF7F2FFF2
S3150800ED70019B001B9842F9D302B010BD70470000F2
S3150800ED80002800F0BC8010B50446036C43B1236C20
S3150800ED9013F0100F0AD00120002384F83C3010BD70
S3150800EDA0436480F83C30FFF7E9FFF0E7236C23F46F
S3150800EDB0885323F0020343F002032364514B5A6835
S3150800EDC022F440325A605A6861680A435A602268D7
S3150800EDD0536823F48073536022685368216943EAB1
S3150800EDE0012353602268536823F0407353602268F6
S3150800EDF05368A1680B4353602268936823F4006341
S3150800EE00936022689368E1680B439360A26A3E4B5D
S3150800EE109A4251D02268936823F0706393602268FF
S3150800EE209368A16A0B4393602268936823F0405362
S3150800EE30936022689368E16A0B439360226893683B
S3150800EE4023F00203936022689368A16943EA4103A9
S3150800EE509360236A002B3AD12268536823F400632F
S3150800EE6053602268D36A23F47003D3622168CB6A9D
S3150800EE70E269013A43EA0253CB622268936823F4B3
S3150800EE800073936022689368216B43EA4123936079
S3150800EE902268936823F480639360226893686169A3
S3150800EEA043EA8123936000206064236C23F0030304
S3150800EEB043F0010323646FE72268936823F07063C5
S3150800EEC093602268936823F040539360B6E72268FC
S3150800EED0536843F4006353602268536823F460431D
S3150800EEE053604FF4604393FAA3F3B3FA83F22168AD
S3150800EEF04868636A013B934003434B60B1E70120CE
S3150800EF00704700BF002301400100000F82B00023B4
S3150800EF10019390F83C30012B63D0012380F83C30F4
S3150800EF2003689A6812F0010F14D19A6842F0010238
S3150800EF309A60304B1B68304AA2FB03239B0C03EBF9
S3150800EF4043030193019B2BB1019B013B0193019B59
S3150800EF50002BF9D10268936813F0010F44D0036CB3
S3150800EF6023F4E06323F0010343F4807303645368D6
S3150800EF7013F4806F05D0036C23F4405343F4805395
S3150800EF800364036C13F4805F1ABF436C23F0060313
S3150800EF9000234364002380F83C306FF0220313609B
S3150800EFA0164B5B6813F01F0F0AD103689A6812F0B4
S3150800EFB0405F1BD19A6842F080429A60002011E0B7
S3150800EFC002680F4B9A4201D000200BE09B6813F0B1
S3150800EFD0405F0DD10A4A936843F08043936000204E
S3150800EFE000E0022002B070470020FBE70020F9E7A6
S3150800EFF00020F7E70400002083DE1B4300230140BE
S3150800F0000020014003689A6812F4806F03D09B6859
S3150800F01013F4807F1CD170B50C460546FFF79AFE9F
S3150800F02006462A68136813F0020F1AD1B4F1FF3F97
S3150800F030F8D024B1FFF78EFE801B8442F1D22B6CE8
S3150800F04043F004032B64002385F83C30032070BD8D
S3150800F050036C43F020030364002380F83C3001204E
S3150800F06070476FF0120313602B6C43F400732B6424
S3150800F0702B689A6812F0405F17D1AA69BAB9DA6A9A
S3150800F08012F4700F03D09B6813F4806F11D12B6CA8
S3150800F09023F480732B642B6C13F4805F0BD12B6CD9
S3150800F0A043F001032B64002070BD002070BD0020D2
S3150800F0B070BD002070BD002070BD0368D86C704715
S3150800F0C030B482B00023019390F83C30012B00F055
S3150800F0D0B680012380F83C300B68092B3AD90568BD
S3150800F0E0EA689BB203EB43031E3B072404FA03F3C7
S3150800F0F022EA0303EB600468E5680B8803EB430325
S3150800F1001E3B8A6802FA03F32B43E3604B68062B1F
S3150800F11035D805686A6B03EB8303053B1F2404FA9D
S3150800F12003F322EA03036B630468656B0A884B687A
S3150800F13003EB8303053B02FA03F32B43636302687D
S3150800F140404B9A424BD0002380F83C30184602B018
S3150800F15030BC704705682A699BB203EB4303072452
S3150800F16004FA03F322EA03032B61046825690B8872
S3150800F17003EB43028B6893402B432361C6E70C2BB2
S3150800F18016D805682A6B03EB8303233B1F2404FA6E
S3150800F19003F322EA03032B630468256B0A884B688A
S3150800F1A003EB8303233B02FA03F32B432363C6E7EC
S3150800F1B00568EA6A03EB8303413B1F2404FA03F359
S3150800F1C022EA0303EB620468E56A0A884B6803EBE4
S3150800F1D08303413B02FA03F32B43E362AFE70B6871
S3150800F1E0122B22D00B68184A934201D0112BAAD1B0
S3150800F1F0164A536843F4000353600A68124B9A424E
S3150800F200A1D1134B1B68134AA2FB03239B0C03EBE8
S3150800F21083035B000193019B002B94D0019B013B68
S3150800F2200193019B002BF9D18DE7084A536843F4F3
S3150800F230800353600268034B9A42D3D083E70220C7
S3150800F24085E700BF0020014012000010002301409E
S3150800F2500400002083DE1B43074AD36823F4E063D7
S3150800F2601B041B0C43F0BF6343F40033000200F495
S3150800F270E0600343D360704700ED00E030B4154BFF
S3150800F280DC68C4F30224C4F10703042B28BF042353
S3150800F290251D062D8CBFE51E0025012404FA03F35F
S3150800F2A0013B1940A940AC40013C224011430028CB
S3150800F2B009DB0901C9B200F1604000F5614080F838
S3150800F2C0001330BC704700F00F000901C9B2024BA9
S3150800F2D01954F6E700ED00E014ED00E0420900F0ED
S3150800F2E01F00012303FA00F0014B43F82200704780
S3150800F2F000E100E0430900F01F00012202FA00F0D5
S3150800F3002033024A42F82300704700BF00E100E0BC
S3150800F3100138B0F1807F0AD2064B5860F021064AC0
S3150800F32082F823100020986007221A60704701208F
S3150800F330704700BF10E000E000ED00E0430900F070
S3150800F3401F00012202FA00F06033024A42F8230045
S3150800F350704700BF00E100E00428044A13680CBFA8
S3150800F36043F0040323F004031360704710E000E041
S3150800F370704708B5FFF7FCFF08BD00000268D3B266
S3150800F380103B0849A1FB03131B090749C95CC16562
S3150800F390032B22F47F7222F0030288BF04328265AF
S3150800F3A0806D7047ABAAAAAA4CFD020838B5044678
S3150800F3B0FFF7D0FC002C00F094800546002384F863
S3150800F3C03430022384F835302268136823F00103A9
S3150800F3D0136023681A6812F0010F0AD0FFF7BAFC07
S3150800F3E0401B0528F5D920236365032084F83500DA
S3150800F3F038BD1A683C4810406168A2680A43E1684B
S3150800F4000A4321690A4361690A43A1690A43E16912
S3150800F4100A43216A0A430243616A042916D01A601C
S3150800F42021684B6923F00703626A1343042A12D042
S3150800F4304B612046FFF7A2FFE26D3F2393408360AE
S3150800F44000206065012384F8353038BDE16A206BF9
S3150800F45001430A43E3E7A26AA069D0B9012A0CD09E
S3150800F46032B1022A10D00020002834D11343DFE736
S3150800F47094F82F0000F00100F6E7E06AB0F1C07FCB
S3150800F48014BF00200120EFE794F82F0000F00100D8
S3150800F490EAE7B0F5005F08D0022A1CD9032A18D17A
S3150800F4A094F82F0000F00100DEE7032A0FD8DFE802
S3150800F4B002F01202120794F82F0000F00100D3E7B9
S3150800F4C0E06AB0F1C07F14BF00200120CCE700201D
S3150800F4D0CAE70020C8E740236365012084F83500A1
S3150800F4E038BD012038BD00BF3F8010F040B338B5A5
S3150800F4F0044690F83530DBB2022B01D1022038BD24
S3150800F5000268136823F001031360036800251D6071
S3150800F51003685D6003689D600368DD6003681D61BC
S3150800F520036821225A61FFF729FFE26D3F239340C2
S3150800F5308360656584F8355084F83450284638BDAC
S3150800F5400120704770B490F83440012C42D0856D84
S3150800F550012480F8344090F83540E4B2012C05D0F7
S3150800F560002380F83430022070BC7047022480F8EB
S3150800F5703540002444650668346824F480243460E1
S3150800F580046863608368402B1FD00368996003682A
S3150800F590DA60C26D3F239340AB600268136843F09C
S3150800F5A0160313600268536943F080035361036CC2
S3150800F5B023B10268136843F00803136002681368EE
S3150800F5C043F0010313600020CEE703689A600368DE
S3150800F5D0D960DEE70220C7E790F83530DBB2022BA8
S3150800F5E003D08023436501207047052380F8353012
S3150800F5F00268136823F001031360002070470000B7
S3150800F600F0B583B0044600230193724B1E68876DDC
S3150800F6103D68C26D082393402B4210D003681A68D0
S3150800F62012F0040F0BD01A6822F004021A60C26D99
S3150800F63008239340BB60436D43F001034365E26DC5
S3150800F640654B93401D4209D02268526912F0800F1B
S3150800F65004D0BB60636D43F002036365E26D5F4BE4
S3150800F66093401D4209D02268126812F0020F04D096
S3150800F670BB60636D43F004036365E26D102393403A
S3150800F6801D4224D02268126812F0080F1FD0BB60F2
S3150800F69023681A6812F4802F0DD01B6813F4002F04
S3150800F6A004D1236C9BB12046984710E0A36C73B134
S3150800F6B0204698470BE01A6812F4807F03D11A682F
S3150800F6C022F008021A60236C0BB120469847E26DB7
S3150800F6D0202393401D4255D02268126812F0100F5D
S3150800F6E050D0BB6094F83530DBB2052B0ED02368BA
S3150800F6F01A6812F4802F33D01B6813F4002F2AD10E
S3150800F700636C002B3ED0204698473BE0226813687E
S3150800F71023F0160313602268536923F080035361AC
S3150800F720236CA3B12268136823F008031360E26D03
S3150800F7303F239340BB60002384F83430012384F8C8
S3150800F7403530236D002B43D02046984740E0A36C04
S3150800F750002BE7D1EBE7E36BA3B12046984711E00E
S3150800F7601A6812F4807F09D11A6822F010021A600A
S3150800F770002384F83430012384F83530E36B0BB169
S3150800F78020469847636D1BB3636D13F0010F1BD0BA
S3150800F790052384F835302268136823F001031360C3
S3150800F7A00F4AA2FB0632920A019B013301939A4241
S3150800F7B004D323681B6813F0010FF5D1002384F8DE
S3150800F7C03430012384F83530E36C0BB12046984772
S3150800F7D003B0F0BD04000020010080000400800092
S3150800F7E0B5814E1B2DE9F04F83B00025664FDFF833
S3150800F7F0A4E1664EDFF8A091DFF8A0A156E0EC0878
S3150800F80000EB8404D4F820C005F007024FEA820B07
S3150800F8100F2202FA0BF22CEA020C0A6902FA0BF220
S3150800F82042EA0C0222624DE0846802EA040BCC68C4
S3150800F83004FA0CF444EA0B048460446824EA030BD3
S3150800F8404C68C4F30013AB4043EA0B03436050E033
S3150800F8500022A24042EA0C029A6033686FEA080462
S3150800F8604A6812F4803F0CBF234048EA030333601A
S3150800F87073684A6812F4003F0CBF234048EA030342
S3150800F8807360B2684B6813F4801F0CBF224048EAC5
S3150800F8900202B260F3684A6812F4001F0CBF2340E4
S3150800F8A048EA0303F3600135102D6AD00123AB4003
S3150800F8B00A6803EA02084345F5D14A6822F01002AD
S3150800F8C0022A9CD004684FEA450C032202FA0CF27D
S3150800F8D0D24304EA020B4C6804F0030404FA0CF45D
S3150800F8E044EA0B0404604C6824F01004013C012C23
S3150800F8F09AD9C3681A408B6803FA0CF31343C3609A
S3150800F9004B6813F0805FCED0002301937B6C43F4E1
S3150800F91080437B647B6C03F480430193019B25F051
S3150800F920030303F1804303F59C339A6805F0030447
S3150800F930A4004FF00F0C0CFA04FC22EA0C0C7045DC
S3150800F94086D0484513D0504513D0114A904212D05C
S3150800F95002F58062904210D002F5806290420ED085
S3150800F96002F5806290420CBF0622072271E7012247
S3150800F9706FE702226DE703226BE7042269E7052297
S3150800F98067E703B0BDE8F08F00380240003C01404D
S3150800F990000C024000000240000402400008024039
S3150800F9A02DE9F04F00234FF00108DFF818A1DFF822
S3150800F9B01891DFF818B108E04FF0000E0EFA04F4BB
S3150800F9C0A44560D00133102B77D008FA03F202EA77
S3150800F9D00105AA42F6D106685F000324BC40E44349
S3150800F9E0264006604FEAD30E00EB8E0EDEF820C0E6
S3150800F9F003F00706B6000F2707FA06F62CEA0606EE
S3150800FA00CEF82060866826408660466826EA0202A6
S3150800FA104260C2681440C46023F0030202F18042C7
S3150800FA2002F59C32966803F00304A400A74006EA90
S3150800FA30070C5045C0D0584517D0214EB04216D0B5
S3150800FA4006F58066B04215D006F58066B04214D039
S3150800FA5006F58066B04213D006F58066B0420CBF44
S3150800FA604FF0060E4FF0070EA8E7C646A6E74FF07A
S3150800FA70020EA3E74FF0030EA0E74FF0040E9DE732
S3150800FA804FF0050E9AE7946824EA07079760D9F8B5
S3150800FA900020ED432A40C9F80020D9F804202A405E
S3150800FAA0C9F80420D9F808202A40C9F80820D9F846
S3150800FAB00C201540C9F80C5084E7BDE8F08F00BF4C
S3150800FAC00008024000000240003C014000040240D9
S3150800FAD00369194214BF01200020704712B90904AE
S3150800FAE081617047816170477047000008B5054B12
S3150800FAF05B69034200D108BD024B5861FFF7F4FF6A
S3150800FB00F9E700BF003C014003685A6912F4806FA8
S3150800FB100DD06FF480625A610423036400230363E3
S3150800FB20202280F83D2080F83C30012070470020D4
S3150800FB3070472DE9F041064690461D46C1F3074732
S3150800FB408CB2012F33680CBF5B699B6934EA0303E7
S3150800FB500CBF01230023434513D1B5F1FF3FF0D075
S3150800FB602DB1FFF7F7F8069BC01A8542E9D20023A4
S3150800FB703363202286F83D2086F83C300320BDE812
S3150800FB80F0810020BDE8F0812DE9F04104461746D2
S3150800FB909846C1F307468DB2012E23680CBF5B69F0
S3150800FBA09B6935EA030314BF0123002363B3236863
S3150800FBB05A6912F4806F13D1B7F1FF3FECD02FB119
S3150800FBC0FFF7C8F8A0EB08008742E5D200232363B5
S3150800FBD0202284F83D2084F83C300320BDE8F081DB
S3150800FBE01A6842F400721A6023686FF480625A61D8
S3150800FBF00423236400232363202284F83D2084F809
S3150800FC003C300120BDE8F0810020BDE8F08170B5E8
S3150800FC1004460D46164623685B6913F0800F19D112
S3150800FC202046FFF771FFB8B9B5F1FF3FF3D025B10C
S3150800FC30FFF790F8801B8542EDD2236C43F0200332
S3150800FC40236400232363202284F83D2084F83C3073
S3150800FC50032070BD002070BD012070BD2DE9F04164
S3150800FC6084B00546884616461F460B9C02681368EC
S3150800FC7043F48073136000940A9B00224FF001112D
S3150800FC80FFF757FF20B10323184604B0BDE8F081FB
S3150800FC902A6808F0FE03136123460A9A2249284671
S3150800FCA0FFF772FF28B12B6C042B0CBF012303232B
S3150800FCB0EAE7002303932B685A6903929B69039327
S3150800FCC0039B22460A992846FFF7A1FF034658B127
S3150800FCD02B6C042B01D00323D6E72A68136843F458
S3150800FCE0007313600123CFE7012F0ED02B68320A69
S3150800FCF01A6122460A992846FFF789FF034678B112
S3150800FD002B6C042B05D00323BEE72A68F6B21661CE
S3150800FD10BAE72A68136843F4007313600123B3E74C
S3150800FD202A68F6B21661AFE7020001002DE9F04134
S3150800FD3084B005460E46174698460B9C026813681B
S3150800FD4043F4806313600268136843F48073136096
S3150800FD5000940A9B00224FF00111FFF7EAFE20B13A
S3150800FD600323184604B0BDE8F0812B68F6B206F006
S3150800FD70FE021A6123460A9A3C492846FFF704FF01
S3150800FD8028B12B6C042B0CBF01230323E9E70023BE
S3150800FD9003932B685A6903929B690393039B224634
S3150800FDA00A992846FFF733FF58B12B6C042B01D06C
S3150800FDB00323D6E72A68136843F400731360012304
S3150800FDC0CFE7B8F1010F0DD02B683A0A1A6122461F
S3150800FDD00A992846FFF71BFFC8B12B6C042B0FD0D6
S3150800FDE00323BEE72B68FFB21F6122460A992846FD
S3150800FDF0FFF70DFFB0B12B6C042B0CD00323B0E733
S3150800FE002A68136843F4007313600123A9E72B6873
S3150800FE10FFB21F61E9E72A68136843F400731360A9
S3150800FE2001239EE72A68136843F4807313600094DD
S3150800FE300A9B00224FF001112846FFF77AFE08B107
S3150800FE4003238EE72B6846F001061E6123460A9AAD
S3150800FE5006492846FFF798FE0346002881D02B6CF2
S3150800FE60042B0CBF012303237BE700BF020001001C
S3150800FE7070B504460D46164623685B6913F0040FF1
S3150800FE8019D12046FFF740FEB8B9B5F1FF3FF3D0C8
S3150800FE9025B1FEF75FFF801B8542EDD2236C43F048
S3150800FEA02003236400232363202284F83D2084F85A
S3150800FEB03C30032070BD002070BD012070BD70B5B8
S3150800FEC005460C4616462B685A6912F0400F22D191
S3150800FED05A6912F0100F11D124B1FEF73BFF801BAF
S3150800FEE08442F0D22B6C43F020032B64202385F840
S3150800FEF03D30002385F83C30032070BD6FF01002BA
S3150800FF005A6100232B642B63202285F83D2085F84F
S3150800FF103C30012070BD002070BD0000002872D062
S3150800FF2038B5044690F83D30002B41D0242384F898
S3150800FF303D302268136823F00103136000F0B0FB1C
S3150800FF40324BA3FB00239B0C22685360216865682B
S3150800FF502F4A954231D801330B62226863682C49CF
S3150800FF608B4234D85B00B0FBF3F0C0F30B03032BD2
S3150800FF7098BF0420D0612268E369216A0B431360A5
S3150800FF8022682369E1680B43936022686369A16963
S3150800FF900B43D3602268136843F001031360002003
S3150800FFA02064202384F83D30206384F83E0038BD61
S3150800FFB080F83C301BF032FCB8E74FF4967202FB2F
S3150800FFC003F3144AA2FB03239B090133C4E7A16880
S3150800FFD049B903EB4303B0FBF3F0C0F30B0373B16A
S3150800FFE040F40040C6E703EB830303EB8303B0FB4F
S3150800FFF0F3F0C0F30B0323B140F44040BAE7012005
S31508010000B8E70120B6E70120704700BF83DE1B432E
S31508010010A0860100D34D62102DE9F04383B0044652
S315080100200F4690469946BDF82C50FEF793FE94F874
S315080100303D30DBB2202B18BF022303D0184603B08C
S31508010040BDE8F0830646009019230122434920465C
S31508010050FFF76FFD08B10223F0E794F83C30012B56
S3150801006001D10223EAE7012384F83C3022681368A8
S3150801007023F400631360212384F83D30402384F878
S315080100803E3000232364A3F58033E36201960C9B7B
S3150801009000934B46424639462046FFF7DFFD70B9C5
S315080100A0002D2ED132460C992046FFF7E1FE034674
S315080100B0002844D0236C042B3AD00323BEE7236CD3
S315080100C0042B4FF0000384F83C300CBF01230323B3
S315080100D0B4E7236C042B01D00323AFE72268136826
S315080100E043F4007313600123A8E7002BDAD00A9BB7
S315080100F05B781361023DADB20A9B02330A93002D68
S31508010100D0D032460C992046FFF781FD0028E0D170
S3150801011023680A9A12781A616B1E9BB22268516982
S3150801012011F0040FE1D10A9A01320A921D46E6E757
S315080101302268136843F40073136001237EE721687C
S315080101400A6842F400720A60202284F83D200022DF
S3150801015084F83E2084F83C2070E700BF02001000B6
S315080101602DE9F04387B004460D4690469946BDF8F9
S315080101703C60FEF7EFFD94F83D30DBB2202B18BF4B
S31508010180022503D0284607B0BDE8F083074600904C
S315080101901923012282492046FFF7CBFC08B1022523
S315080101A0F0E794F83C30012B01D10225EAE7012357
S315080101B084F83C302268136823F400631360222311
S315080101C084F83D30402384F83E3000232364A3F5A8
S315080101D08033E3620197109B00934B4642462946BA
S315080101E02046FFF7A3FD054648B1236C042B4FF0C3
S315080101F0000384F83C300CBF01250325C2E766B924
S315080102000023029323685A6902929A690292029A12
S315080102101A6842F400721A6054E0012E0ED0022EBA
S3150801022029D00023059323685A6905929B6905938A
S31508010230059BDFF870914FF0000869E022681368A2
S3150801024023F4806313600023039323685A69039296
S315080102509A690392039A1A6842F400721A603A4636
S3150801026010992046FFF72BFE002834D123681B6915
S315080102700E9A137026E02268136823F480631360CC
S315080102802268136843F40063136000230493236808
S315080102905A6904929B690493049B0097109B002258
S315080102A040492046FFF745FC002872D122681368A9
S315080102B043F40073136023681B690E9A137023684D
S315080102C01B695370202384F83D30002384F83E309F
S315080102D084F83C3056E7236C202B0CBF03250125F7
S315080102E050E73A4610992046FFF7E9FD002841D123
S315080102F023681B690E9A137023685A6912F0040F52
S315080103003ED10E9B01330E93013EB6B2002ED9D0D3
S31508010310032EE6D8012EA2D0022EBED00097109B3E
S31508010320424649462046FFF704FC002833D1226895
S31508010330136823F48063136023681B690E9A13708C
S315080103400097109B424649462046FFF7F2FB20BB21
S315080103502268136843F40073136023681B690E9AB5
S31508010360537023681B699370033EB6B21346033371
S315080103700E93CBE7236C202B0CBF0325012501E740
S315080103801B690E9A5370023EB6B2134602330E9398
S31508010390BCE70325F6E60325F4E60325F2E600BFE6
S315080103A0020010000400010030B583B00023019358
S315080103B0234B1A6C42F080521A641B6C03F080536B
S315080103C00193019B4FF4803393FAA3F3B3FA83F3B2
S315080103D003F1845303F560339B0001221A60FEF78B
S315080103E0B9FC0546174C636813F4803F08D1FEF73C
S315080103F0B1FC401BB0F57A7FF5D9032003B030BDB7
S315080104004FF4003393FAA3F3B3FA83F303F1845356
S3150801041003F560339B0001221A60FEF79BFC054633
S31508010420084C636813F4003F07D1FEF793FC401BA1
S31508010430B0F57A7FF5D90320E0E70020DEE700BFB3
S31508010440003802400070004070B588B00C46164668
S3150801045008B300230293204D2A6B42F004022A6353
S315080104602A6B02F004020292029A4FF40072039276
S3150801047002220492032206920593079303A91748B9
S31508010480FFF7B0F9AB6844EAC60423F078431C4386
S31508010490AC6008B070BD002301930F4D2A6B42F082
S315080104A001022A632A6B02F001020192019A4FF4B2
S315080104B080720392022204920322069205930793FD
S315080104C003A90748FFF78EF9AA6822F0EC623243BE
S315080104D01443AC60DDE700BF003802400008024063
S315080104E000000240674B1B6803F00F038B4209D2D9
S315080104F0CBB2644A1370136803F00F03994201D013
S31508010500012070472DE9F041036813F0020F06D068
S315080105105D4A936823F0F0038468234393600D468C
S315080105200446036813F0010F6AD04268012A27D0EE
S31508010530931E012B2CD9544B1B6813F0020F00F0A4
S315080105409E8051498B6823F0030313438B60FEF7A2
S3150801055001FC06466368012B22D0022B30D0032BFF
S315080105603ED0494F41F28838BB6813F00C0F47D08B
S31508010570FEF7F0FB801B4045F6D90320BDE8F08164
S31508010580414B1B6813F4003FDBD10120BDE8F08124
S315080105903D4B1B6813F0007FD3D10120BDE8F081E4
S315080105A0394F41F28838BB6803F00C03042B27D076
S315080105B0FEF7D0FB801B4045F5D90320BDE8F08145
S315080105C0314F41F28838BB6803F00C03082B17D06A
S315080105D0FEF7C0FB801B4045F5D90320BDE8F08135
S315080105E0294F41F28838BB6803F00C030C2B07D05E
S315080105F0FEF7B0FB801B4045F5D90320BDE8F08125
S31508010600204B1B6803F00F039D420AD2EAB21D4B29
S315080106101A701B6803F00F039D4202D00120BDE842
S31508010620F081236813F0040F06D0174A936823F460
S31508010630E053E1680B439360236813F0080F07D072
S31508010640114A9368216923F4604343EAC10393601D
S3150801065000F030FD0C4B9B68F02292FAA2F2B2FA36
S3150801066082F203F0F003D340084AD35CD840084B22
S3150801067018600020FEF736FB0020BDE8F081012056
S31508010680BDE8F081003C02400038024054FD0208F2
S3150801069004000020014B1868704700BF04000020C1
S315080106A0084B9B684FF4E05292FAA2F2B2FA82F230
S315080106B003F4E053D340044AD35C044A1068D84093
S315080106C0704700BF0038024054FD020804000020AC
S315080106D0084B9B684FF4604292FAA2F2B2FA82F290
S315080106E003F46043D340044AD35C044A1068D840F3
S315080106F0704700BF0038024054FD0208040000207C
S315080107002DE9F04383B00446036813F0010F00F0A6
S31508010710AB80964AD2F88C3023F0C063816B0B43C9
S31508010720C2F88C30856BB5FA85F56D09236813F027
S31508010730020F0CD08D4AD2F88C3023F0C053E16BEE
S315080107400B43C2F88C30E36B002B08BF01252368E5
S3150801075013F0040F00F08A80844AD2F88C3023F40F
S315080107604013216B0B43C2F88C30266BB6F5801FFC
S3150801077008BF0125B6FA86F67609236813F0080F2D
S315080107800FD07A4AD2F88C3023F44003616B0B43BD
S31508010790C2F88C30636BB3F5800F69D0002B08BFA4
S315080107A00126236813F0200F64D1236813F0100F74
S315080107B003D094F858206E4B1A60236813F0800F03
S315080107C008D06A4AD2F8943023F44003E16C0B430B
S315080107D0C2F89430236813F0400F08D0634AD2F860
S315080107E0943023F08063A16C0B43C2F894302368DC
S315080107F013F4807F0DD05D4AD2F8943023F000635C
S31508010800616D0B43C2F89430636DB3F1006F08BF95
S315080108100126236813F4007F08D0544AD2F894308D
S3150801082023F08053616C0B43C2F89430236813F4A8
S31508010830806F0CD04D4AD2F8943023F00053216DC5
S315080108400B43C2F89430236DB3F1005F7BD0012DC1
S3150801085079D02368B3F5006F75D0012E00F0C781F2
S31508010860002003B0BDE8F08300255FE7002684E792
S31508010870012596E7002301933C4B1A6C42F08052FE
S315080108801A641B6C03F080530193019B394A136860
S3150801089043F480731360FEF75DFA8046354F3B6873
S315080108A013F4807F07D1FEF755FAA0EB080002285A
S315080108B0F5D90320D5E72D4B1B6F13F4407312D0DE
S315080108C0226C02F4407293420DD0284B1A6F22F41F
S315080108D04072294901200860002008601A671B6FC9
S315080108E013F0010F12D1236C03F44072B2F5407F65
S315080108F01ED01E4A936823F4F81393601B4A116F9E
S31508010900236CC3F30B030B4313674EE7FEF722FA77
S315080109108146164F41F288383B6F13F0020FE2D138
S31508010920FEF718FAA0EB09004045F5D9032098E728
S315080109300E498A6822F4F81223F0704323F44073AF
S3150801094013438B60DAE700220C4B1A60FEF702FAB2
S315080109500746064D2B6813F0006F11D0FEF7FAF91A
S31508010960C01B0228F6D903207BE700BF00380240E6
S31508010970E011474200700040400E47426800474276
S31508010980236813F0010F01D0A26B2AB113F0020FED
S3150801099043D0E36B002B40D1CB49D1F884304FF4D7
S315080109A0403090FAA0FEBEFA8EFED1F884504FF080
S315080109B0706C9CFAACF8B8FA88F847F6C07292FAE5
S315080109C0A2F2B2FA82F790FAA0F0B0FA80F09CFA95
S315080109D0ACFCBCFA8CFC4FF0E04999FAA9F9B9FAD2
S315080109E089F9A268BA40676907FA09F73A43676855
S315080109F03A4305F0706525FA08F808FA0CFC42EA4C
S31508010A000C0203F4403323FA0EF3013323F00043B7
S31508010A10013B83401343C1F88430236813F0040F64
S31508010A2003D0226BB2F5801F53D013F0080F03D001
S31508010A30636BB3F5800F4CD0236813F4806F04D031
S31508010A40236DB3F1005F00F08F80236813F4006F04
S31508010A502CD047F6C07090FAA0F0B0FA80F04FF4A7
S31508010A60403393FAA3F3B3FA83F54FF0706191FA21
S31508010A70A1F1B1FA81F14FF0E04292FAA2F2B2FA8B
S31508010A8082F2E3685B08013BAB40A56805FA00F012
S31508010A90034360680343206900FA01F10B43616966
S31508010AA001FA02F21343884AC2F884300122874BBD
S31508010AB01A60FEF74FF90746834D2B6813F0006F4E
S31508010AC07FF4CBAEFEF746F9C01B0228F5D9032001
S31508010AD0C7E67D49D1F884304FF4403090FAA0FE3C
S31508010AE0BEFA8EFED1F884504FF0E04C9CFAACF871
S31508010AF0B8FA88F847F6C07292FAA2F2B2FA82F701
S31508010B0090FAA0F0B0FA80F04FF0706999FAA9F955
S31508010B10B9FA89F99CFAACFCBCFA8CFCA268BA4011
S31508010B20276907FA09F73A4367683A4305F0E04542
S31508010B3025FA08F808FA0CFC42EA0C0203F44033D9
S31508010B4023FA0EF3013323F00043013B8340134399
S31508010B50C1F88430D1F88C20A36A013B22F01F0228
S31508010B601343C1F88C3067E7DFF85CE1DEF88420CF
S31508010B704FF4403393FAA3FCBCFA8CFCDEF88410DC
S31508010B804FF0E04090FAA0F8B8FA88F847F6C0792D
S31508010B9099FAA9F9B9FA89F993FAA3F3B3FA83F792
S31508010BA04FF0706595FAA5F5B5FA85F590FAA0F0B6
S31508010BB0B0FA80F0E3685B08013BBB40A76807FA17
S31508010BC009F73B4367683B4301F0E04121FA08F81E
S31508010BD008FA00F0034302F4403222FA0CF2013219
S31508010BE0520002FA05F52B43CEF884302DE7002290
S31508010BF0374B1A60FEF7AEF80646334D2B6813F0ED
S31508010C00005F06D0FEF7A6F8801B0228F6D9032056
S31508010C1027E6236813F0040F01D0226B22B113F0E3
S31508010C20080F37D0636BABBB2749D1F888304FF42F
S31508010C30403090FAA0F7B7FA87F747F6C07292FAEA
S31508010C40A2F2B2FA82F690FAA0F0B0FA80F04FF06A
S31508010C50706595FAA5F5B5FA85F5E269B240666A51
S31508010C6006FA05F52A43A5692A4303F44033FB40EE
S31508010C70013323F00043013B83401343C1F8883015
S31508010C80D1F88C30E26A013A23F4F85343EA022395
S31508010C90C1F88C30236813F4807F03D0636DB3F1F8
S31508010CA0006F17D001220A4B1A60FEF753F8054662
S31508010CB0054C236813F0005F37D1FEF74BF8401B4C
S31508010CC00228F6D90320CCE50038024068004742DD
S31508010CD0700047421648D0F888204FF0706191FAA3
S31508010CE0A1F7B7FA87F747F6C07595FAA5F5B5FAE4
S31508010CF085F54FF4403393FAA3F3B3FA83F691FAE1
S31508010D00A1F1B1FA81F1236A5B08013BB340E669B7
S31508010D1006FA05F52B43A469234302F07062FA40EB
S31508010D208A401343C0F88830BCE7002099E500BF24
S31508010D3000380240F0B583B00446036813F0010F8A
S31508010D4034D0AE4B9B6803F00C03042B25D0AB4B78
S31508010D509B6803F00C03082B1AD0A84B9B6803F079
S31508010D600C030C2B4CD02279A54B1A706368002B07
S31508010D704CD0FDF7EFFF0646A04D2B6813F4003F54
S31508010D8014D1FDF7E7FF801B6428F6D9032088E113
S31508010D909A4B5B6813F4800FDFD0984B1B6813F4EA
S31508010DA0003F03D06368002B00F07881236813F0B5
S31508010DB0020F5CD0914B9B6813F00C0F3AD08F4B06
S31508010DC09B6803F00C03082B2FD08C4B9B6803F010
S31508010DD00C030C2B38D0E368002B6ED00122894B0B
S31508010DE01A60FDF7B7FF0646844D2B6813F0020F0C
S31508010DF055D1FDF7AFFF801B0228F6D9032050E134
S31508010E007E4B5B6813F4800FADD0C6E7FDF7A2FFF2
S31508010E1006467A4D2B6813F4003FC7D0FDF79AFFB3
S31508010E20801B6428F6D903203BE1744B5B6813F4F5
S31508010E30800FCAD1714B1B6813F0020F0AD0E36801
S31508010E40012B07D001202CE16C4B5B6813F4800F52
S31508010E50C1D1EFE769480168F82393FAA3F3B3FA16
S31508010E6083F22369934021F0F80213430360236850
S31508010E7013F0080F45D063698BB30122624B1A60E0
S31508010E80FDF768FF06465D4D6B6F13F0020F38D10B
S31508010E90FDF760FF801B0228F6D9032001E15748B8
S31508010EA00168F82393FAA3F3B3FA83F2236993400B
S31508010EB021F0F80213430360D9E70022514B1A6067
S31508010EC0FDF748FF06464D4D2B6813F0020FCED0AD
S31508010ED0FDF740FF801B0228F6D90320E1E0002236
S31508010EE0494B1A60FDF736FF0646444D6B6F13F002
S31508010EF0020F06D0FDF72EFF801B0228F6D9032024
S31508010F00CFE0236813F0040F1FD1A369002B00F06B
S31508010F10C7803A4A926802F00C02082A00F0C38098
S31508010F20022B59D00022394B1A60FDF713FF0546EB
S31508010F30324C236813F0007F00F0AE80FDF70AFFFC
S31508010F40401B0228F5D90320ABE0002301932B4B64
S31508010F501A6C42F080521A641B6C03F08053019399
S31508010F60019B2B4A136843F480731360FDF7F2FE65
S31508010F700646274D2B6813F4807F06D1FDF7EAFE56
S31508010F80801B0228F6D903208BE0227A214B1A709E
S31508010F90A36883B1FDF7DEFE0746184D41F2883690
S31508010FA02B6F13F0020FB0D1FDF7D4FEC01BB04270
S31508010FB0F6D9032075E0FDF7CDFE07460F4D41F240
S31508010FC088362B6F13F0020F9FD0FDF7C3FEC01BA7
S31508010FD0B042F6D9032064E000220C4B1A60FDF7F3
S31508010FE0B9FE0646054D2B6813F0007F14D0FDF7B0
S31508010FF0B1FE801B0228F6D9032052E000380240D0
S315080110000238024000004742800E474260004742CC
S31508011010007000407038024047F6C07696FAA6F688
S31508011020B6FA86F64FF4403292FAA2F2B2FA82F58D
S315080110304FF0706090FAA0F0B0FA80F04FF0E041FE
S3150801104091FAA1F1B1FA81F1E369226A1343626A5D
S31508011050B2401343A26A5208013AAA401343E26A0C
S3150801106082401343226B02FA01F10B430F4A536084
S3150801107001220F4B1A60FDF76DFE05460B4C2368DE
S3150801108013F0007F06D1FDF765FE401B0228F6D94D
S31508011090032006E0002004E0002002E0012000E031
S315080110A0002003B0F0BD0120FBE700BF0038024075
S315080110B060004742274B9B6803F00C03082B03D0BB
S315080110C00C2B25D024487047224B5A6802F03F0260
S315080110D05B68204B5B6847F6C07191FAA1F0B0FADC
S315080110E080F00B40C3401C48B0FBF2F000FB03F054
S315080110F0184B5B684FF4403292FAA2F2B2FA82F2C6
S3150801110003F44033D34001335B00B0FBF3F070477F
S31508011110104B5A6802F03F025B680E4B5B6847F654
S31508011120C07191FAA1F0B0FA80F00B40C3400A48A9
S31508011130B0FBF2F000FB03F0064B5B684FF0E042B0
S3150801114092FAA2F2B2FA82F203F0E043D340B0FB7C
S31508011150F3F07047003802400024F4000268536B2C
S3150801116013F0450FFBD0536B13F0040F03D0042380
S31508011170936303207047536B13F0010F04D140F2B8
S31508011180FF53936300207047012090637047000066
S3150801119038B50268536B13F0450FFBD0536B13F048
S315080111A0040F03D004239363032038BD536B13F054
S315080111B0010F02D00120906338BD0D460446104642
S315080111C002F0EFF9A84201D0102038BD236840F299
S315080111D0FF529A63002002F0E7F9334B0340002BD4
S315080111E03FD000283FDB10F0804F01D0092038BDE1
S315080111F010F0005F01D00A2038BD10F0805F34D1AD
S3150801120010F0006F33D110F0806F32D110F0807F6B
S3150801121031D110F4000F30D110F4800F2FD110F412
S31508011220001F2ED110F4801F2DD110F4002F2CD1C0
S3150801123010F4802F2BD110F4003F2AD110F4803FEF
S3150801124029D110F4004F28D110F4804F27D110F47A
S31508011250005F26D100F00800002814BF1A200020DC
S3150801126038BD002038BD1C2038BD0B2038BD0C20E8
S3150801127038BD0D2038BD0E2038BD0F2038BD1020D1
S3150801128038BD112038BD122038BD132038BD1420B1
S3150801129038BD152038BD162038BD172038BD182091
S315080112A038BD192038BD00BF08E0FFFD30B587B04D
S315080112B004460D4600220092436A1B0401930D233E
S315080112C002934023039304924FF48063059301A983
S315080112D0006802F051F92068436B13F0450FFBD003
S315080112E0436B13F0040F04D004238363032007B070
S315080112F030BD436B13F0010F03D0012383631846F6
S31508011300F5E702F04EF90D2818BF1020EFD1236832
S3150801131040F2FF529A63002002F046F90090009BC2
S31508011320C3F343232B70009A3C4B1340002B52D036
S31508011330009B002B51DB009B13F0804F01D0092045
S31508011340D5E7009B13F0005F01D00A20CFE7009B89
S3150801135013F0805F43D1009B13F0006F41D1009BCE
S3150801136013F0806F3FD1009B13F0807F3DD1009B26
S3150801137013F4000F3BD1009B13F4800F39D1009B66
S3150801138013F4001F37D1009B13F4801F35D1009B3E
S3150801139013F4002F33D1009B13F4802F31D1009B16
S315080113A013F4003F2FD1009B13F4803F2DD1009BEE
S315080113B013F4004F2BD1009B13F4804F29D1009BC6
S315080113C013F4005F27D1009B03F00803002B14BF19
S315080113D01A2000208BE7002089E71C2087E70B20CD
S315080113E085E70C2083E70D2081E70E207FE70F2094
S315080113F07DE710207BE7112079E7122077E7132094
S3150801140075E7142073E7152071E716206FE7172093
S315080114106DE718206BE7192069E700BF08E0FFFDB3
S315080114202DE9F0418EB004460E460023019302933E
S315080114300822099210250A9540220B920C934FF423
S3150801144080630D9309A9006802F096F8294620469B
S31508011450FFF79EFE054618B128460EB0BDE8F08195
S31508011460636A1B04099337250A9509A9206802F0BE
S3150801147083F829462046FFF78BFE05460028EBD15F
S315080114804FF0FF3303930823049330230593022374
S315080114900693002507950123089303A9206802F0FE
S315080114A08FF8099533250A9509A9206802F064F889
S315080114B029462046FFF76CFE05460028CCD10DF1DA
S315080114C0040840F22A472068436B3B4208D1436B24
S315080114D013F4001FF8D002F03FF848F8040BF2E7BE
S315080114E0436B13F0080F03D0082383630425B3E77E
S315080114F0436B13F0020F02D002258563ACE7436BF9
S3150801150013F0200F03D0202383630625A4E740F2B6
S31508011510FF538363019B1A0E42EA0362190201F41F
S315080115207F010A431B0A03F47F4313437360029B3B
S315080115301A0E42EA0362190201F47F010A431B0AE1
S3150801154003F47F431343336086E770477047704758
S3150801155010B5044603685A6B12F4807F17D15A6B8B
S3150801156012F0020F1DD15A6B12F0080F1FD15A6BD8
S3150801157012F0200F22D15A6B12F0100F25D12268D2
S31508011580D36B23F4414323F03A03D36310BD4FF4DD
S3150801159080729A63012383640023C364FFF7D6FF2D
S315080115A0EDE702229A63C264FFF7D1FFE7E7082253
S315080115B09A630423C364FFF7CAFFE0E720229A630C
S315080115C00623C364FFF7C3FFD9E710229A630523ED
S315080115D0C364FFF7BCFFD2E7F0B40346026A81F899
S315080115E05620426AA1F85420826A900F0870C2F305
S315080115F083604870C2F301628A7093F82A20CA7020
S3150801160093F829200A7193F828204A7193F82F2014
S315080116101201CA80D86ACA8892B2C0F30354224317
S31508011620CA80C0F30340087293F82D20D009487286
S31508011630C2F380108872C2F34010C872C2F3001058
S31508011640087300204873186A012840F2AE80022800
S3150801165000F0EA802920C2F380144C76520002F089
S315080116607E028A761A6B8C7EC2F3C0152C438C7661
S3150801167002F07F02CA765A6BD40F0C77C2F3417413
S315080116804C77C2F382648C77920D02F00C02CA770A
S315080116905A6BCC7FC2F381552C43CC77C2F34054A5
S315080116A081F82040002481F82140C2F3004281F8E4
S315080116B022205A6BC2F3C03481F82340C2F3803426
S315080116C081F82440C2F3403481F82540C2F300343E
S315080116D081F82640C2F3812481F82740C2F301220A
S315080116E081F828205A6BC2F3460281F82920012481
S315080116F081F82A4093F83B2081F82C2093F83A2068
S315080117001202CA85CA8D92B293F839502A43CA85FC
S315080117109A6B12060A630A6B93F83F5042EA05422E
S315080117200A630D6BDA8F120292B22A430A630D6BB2
S3150801173093F83D202A430A6393F83C2081F8342024
S3150801174093F8432081F83520B3F8422012068A63BC
S315080117508D6B1A6C120202F47F022A438A638D6B1F
S315080117601A6C120292B22A438A638D6B93F8472048
S315080117702A438A635A6C91F83C50C2F3035635439F
S3150801178081F83C50120A02F47062CA87CA8F92B273
S3150801179093F845502A43CA875B6CC3F3460381F81D
S315080117A0403081F84140F0BC7047920202F4406231
S315080117B00A610869DA6A920002F47F7202430A61D1
S315080117C01A6B086940EA92700861C2F3C26008752B
S315080117D0C2F302624A751A6BC2F342508875C2F3A4
S315080117E08240C875D20B02F006020A76186BC0F35E
S315080117F007220C7EC0F3C030204308760C690F7EA1
S31508011800087AC0B2012606FA00F008653444A4FB3A
S315080118100045B81C06FA00F0A4FB006700FB057733
S31508011820C1E91267002016E7DA6A120402F47C128B
S315080118300A610A6993F8330042EA00220A610869D3
S3150801184093F8322002430A6193F831200C69002586
S31508011850013445F10005E80440EA5430E4048C6497
S31508011860C8644FF4007008650020F4E62DE9F043DA
S3150801187093B00446894600268DF847600677FFF738
S3150801188064FE0B960C960D960E960F96762310937C
S315080118900EAB93E807008DE807000BAB0ECB20686B
S315080118A001F03EFE8DF81760AB4F3E60206801F0EF
S315080118B05BFE0120FDF754FA01233B600696079665
S315080118C0089609964FF480630A9306A9206801F0E1
S315080118D053FE21684B6B13F0800F40F099814B6BD7
S315080118E0C3F3C0134FF6FF72002B40F091814B6B87
S315080118F0C3F3C013013AF7D103238DE14FF4D5732E
S315080119000693082307934023089306A9206801F044
S3150801191033FE21684B6B13F0450F40F094814FF469
S3150801192080334A6B013B12F0450F03D1002BF8D1E6
S315080119304B6B01E04A6B2BBB04238B6303238DF8A6
S3150801194017309DF8173053BB012323624FF08045AA
S31508011950002306933726079606A9206801F00CFE90
S3150801196031462046FFF714FC8DF817009DF817300D
S31508011970002B6DD14FF00008464645F0004545F469
S31508011980801527E002F00402002AD5D14B6B13F02B
S31508011990400F1DBF40238B6300232923CFE7002572
S315080119A0D6E79DF81730DBB240E140F2FF53936367
S315080119B033468DF817309DF81730002B3BD130464A
S315080119C001F0F2FD08F10108002838DB4FF6FF7334
S315080119D0984541D0069637270797402308930996D5
S315080119E04FF480630A9306A9206801F0C5FD3946BC
S315080119F02046FFF7CDFB8DF817009DF81730002B11
S31508011A00CFD10695292307934023089309964FF4C6
S31508011A1080630A9306A9206801F0AEFD2268536B1C
S31508011A2013F0450FFBD0536B13F0040FBDD00423FD
S31508011A3093630323BDE79DF81730DBB2F6E04FF653
S31508011A40FE73984508D810F0804F1CBF0223236205
S31508011A509DF81730DBB2E9E01B238DF817309DF8A6
S31508011A601730DBB2E2E0206801F082FD58B925267D
S31508011A708DF847609DF84730002B00F097809DF858
S31508011A804700C0B2DCE0236A042B00F08D800023F6
S31508011A90069302220792C022089209934FF48063A3
S31508011AA00A9306A9206801F067FD2046FFF756FB51
S31508011AB006460028DCD101F077FDA063042001F079
S31508011AC073FDE063082001F06FFD20640C2001F02E
S31508011AD06BFD6064236A022B01D9062B3ED10323D1
S31508011AE007934023089306A9206801F045FD20685D
S31508011AF0436B13F0450FFBD0436B13F0040F03D070
S31508011B00042383630326B3E7436B13F0010F02D063
S31508011B1001268663ACE701F044FD032818BF1026A9
S31508011B20A6D1236840F2FF529A63002001F03CFDDA
S31508011B3010F4604F01D1000C11E010F4005F40F081
S31508011B40868010F4804F40F0848010F4004F40F0F6
S31508011B508280012003E000BFA08025420120236A7C
S31508011B60042B85D060620004069009230793C023DD
S31508011B70089306A9206801F0FFFC2046FFF7EEFA54
S31508011B80064600287FF474AF01F00EFDA06204201A
S31508011B9001F00AFDE062082001F006FD20630C2031
S31508011BA001F002FD606363E7002661E749462046C6
S31508011BB0FFF712FD8DF847009DF8473083B123469C
S31508011BC053F8105B93E807008DE80700043494E89E
S31508011BD00E00284601F0A4FC9DF84700C0B22FE08C
S31508011BE0B9F854301B040693072507954023089333
S31508011BF0002309934FF480630A9306A9206801F02C
S31508011C00BBFC29462046FFF7C3FA8DF84700D6E7FD
S31508011C1040F2FF538B6300238DF817309DF8173078
S31508011C20002B3FF46BAE9DF81730DBB28DF84730C9
S31508011C309DF84730002B3FF416AF9DF84700C0B218
S31508011C4013B0BDE8F0834A6B02F004029CE6132642
S31508011C500EE710260CE70F260AE700BF70B592B00B
S31508011C60036A032B00F09F80022B00F2A080B1F5D6
S31508011C70805F00F09E800D460446B1F5006F03D0E3
S31508011C8000293CD026268FE000200590069001F019
S31508011C908BFC10F0007F01D00E2639E005A92046FD
S31508011CA0FFF7BEFB0646002832D1069B13F4802FA8
S31508011CB001D125262CE0636A1B040793372608966B
S31508011CC04023099300230A934FF480630B9307A9D2
S31508011CD0206801F051FC31462046FFF759FA0646BD
S31508011CE0B0B9022307930626089607A9206801F0CA
S31508011CF043FC31462046FFF74BFA064608E000202A
S31508011D000590069001F050FC10F0007F19D00E26C0
S31508011D10002E49D163680C93A3680D93E3680E936B
S31508011D200F9563691093A3691193246812AB13E99C
S31508011D3007008DE807000CAB0ECB204601F0F0FB3F
S31508011D4032E005A92046FFF76BFB06460028DFD1DE
S31508011D50069B13F4803F01D12526D9E7636A1B0444
S31508011D600793372608964023099300230A934FF4CD
S31508011D7080630B9307A9206801F0FEFB31462046D4
S31508011D80FFF706FA06460028C2D10023079306265E
S31508011D90089607A9206801F0EFFB31462046FFF7B0
S31508011DA0F7F90646B4E72726304612B070BD002675
S31508011DB0FAE72726F8E730B587B0044600230193EA
S31508011DC00C2502954022039204934FF480630593F0
S31508011DD001A9006801F0D0FB29462046FFF7D8F98A
S31508011DE007B030BD2DE9F0438DB004460E46904646
S31508011DF0149D02680021D162026A022A17D007954A
S31508011E00102708974023099300230A934FF4806308
S31508011E100B9307A9206801F0AFFB39462046FFF767
S31508011E20B7F9074650B138460DB0BDE8F0834FEA19
S31508011E30582848EAC3584FF40075E0E74FF0FF33D6
S31508011E400193159B03FB05F5029590230393022342
S31508011E500493002305930123069301A9206801F041
S31508011E60AFFB159B012B23D9122508950CA941F81F
S31508011E70148D206801F080FB29462046FFF788F972
S31508011E8007460028CFD123685A6B12F4957F64D18F
S31508011E905A6B12F4004FF7D0351F06F11C0820685B
S31508011EA001F05AFB45F8040FA845F8D12036EAE7B0
S31508011EB0112508950CA941F8148D206801F05CFBE1
S31508011EC029462046FFF764F907460028ABD140F2B8
S31508011ED02A4823685A6B12EA080F34D15A6B12F44E
S31508011EE0004FF7D0351F06F11C09206801F034FBB5
S31508011EF045F8040F4D45F8D12036EAE7436B13F050
S31508011F00020F02D0022787638DE7436B13F0200F78
S31508011F1003D020238363062785E7436B13F4001F49
S31508011F2018BF4FF0FF350AD001F016FB46F8040B2F
S31508011F302068436B13F4001F01D0013DF4D140F230
S31508011F40FF5383636FE75B6B2068436B13F0080FDE
S31508011F50D4D008238363042765E75B6B13F4807F7A
S31508011F60F2D0236A022BEFD82046FFF724FF074653
S31508011F70EAE72DE9F04F8DB004460F461646169D41
S31508011F8000228DF803200168CA62026A022A2ED04D
S31508011F9007954FF01008CDF82080402309930023B8
S31508011FA00A934FF480630B9307A9206801F0E4FABA
S31508011FB041462046FFF7ECF80346A0B9179B012BCB
S31508011FC08CBF4FF019084FF01808CDF820800CA9DE
S31508011FD041F8146D206801F0CFFA41462046FFF713
S31508011FE0D7F8034650B118460DB0BDE8F08F4FEA51
S31508011FF0562949EAC3564FF40075C9E7179B03FBEF
S3150801200005F54FF0FF3301930295902303930023BF
S31508012010049305930123069301A9206801F0D0FAD8
S31508012020179B012B29D94FF0000823685A6B12F424
S315080120308D7F40F0A4805A6B12F4804FF6D0A5EB41
S31508012040080ABAF11F0F46D81AF0030F4FEA9A0A7F
S3150801205018BF0AF1010ABAF1000FE6D0B9460026FF
S315080120604946206801F07BFA09F104090136B245AF
S31508012070F6D1B6003744B044D7E74FF0000840F22E
S315080120801A4623685A6B324240F086805A6B12F41C
S31508012090804FF7D0A5EB080BBBF11F0F28D81BF013
S315080120A0030F4FEA9B0B18BF0BF1010BBBF1000F96
S315080120B0E7D0BA464FF000095146206801F04FFAB9
S315080120C00AF1040A09F10109CB45F5D14FEA890953
S315080120D04F44C844D5E73E462037B94631462068BD
S315080120E001F03DFA04364E45F8D108F120089CE77F
S315080120F0B9462037BA464946206801F030FA09F14F
S315080121000409D145F7D108F12008BAE7236A022B59
S3150801211039D82046FFF74FFE35E0536B13F0020F0F
S3150801212002D0022393635EE7536B13F0100F03D0BB
S3150801213010239363052356E740F2FF5393630DF18A
S3150801214003012046FFF7B2F8034600287FF44BAF98
S315080121509DF80320063AD2B2012A3FF644AF0DF1A3
S3150801216003012046FFF7A2F8034600287FF43BAF98
S315080121709DF80320063AD2B2012AF0D933E75B6B00
S3150801218013F4807FC2D12268536B13F0080FC4D0B1
S3150801219008239363042326E75B6BF4E730B587B01E
S315080121A00446436A1B0401930D25029540230393B4
S315080121B0002304934FF48063059301A9006801F095
S315080121C0DBF929462046FEF7E3FF10B1022007B0E6
S315080121D030BD01F0E9F9C0F34320043818BF0120E6
S315080121E0F5E7F8B507460E4615461C463A6893685C
S315080121F036EA03030CBF012300239D4238D0B4F10C
S31508012200FF3FF4D02CB1FCF7A5FD069BC01A84420A
S31508012210ECD83A68536823F0E00353607B68B3F55A
S31508012220827F0BD0BB6AB3F5005F14D0012387F810
S315080122305130002387F850300320F8BDBB68B3F549
S31508012240004F02D0B3F5806FECD13A68136823F0DA
S3150801225040031360E6E73A68136823F400531B0446
S315080122601B0C13603A68136843F400531360DDE7E7
S315080122700020F8BD10B582B0044600920B46002234
S315080122808021FFF7AEFF034620B1636D43F02003BB
S3150801229063650323184602B010BD00283BD010B56C
S315080122A004460023836290F85130002B2ED0022376
S315080122B084F851302268136823F0400313602268BA
S315080122C06368A1680B43E1680B4321690B436169A4
S315080122D00B43E1690B43216A0B43A16A0B43A169CD
S315080122E001F400710B4313602268638B03F0040346
S315080122F0616A0B4353602268D36923F40063D3618F
S3150801230000206065012384F8513010BD80F85030F3
S3150801231019F0B0FACBE7012070472DE9F04184B0F6
S315080123201D4690F85030012B03D1022004B0BDE8B8
S31508012330F08104460E469046012380F85030FCF79A
S3150801234009FD074694F85130DBB2012B07D002206C
S31508012350012384F85130002384F85030E6E7002E33
S3150801236000F09E80B8F1000F00F09C80032384F8EA
S315080123705130002363652663A4F83480A4F83680B7
S31508012380A363A387E38763642364A368B3F5004F54
S315080123901BD023681A6812F0400F03D11A6842F05D
S315080123A040021A60E368B3F5006F14D063681BB185
S315080123B0E38E9BB2012B41D1236816F8012B1A73C0
S315080123C0E38E013B9BB2E38638E02268136843F447
S315080123D080431360DDE763681BB1E38E9BB2012B73
S315080123E012D1236836F8022BDA60E38E013B9BB2E1
S315080123F0E38609E0002D57D0B5F1FF3F04D0FCF77D
S31508012400A9FCC01B854251D9E38E9BB233B323681D
S315080124109A6812F0020FEDD036F8022BDA60E38ED5
S31508012420013B9BB2E386EFE7002D41D0B5F1FF3FB3
S3150801243004D0FCF78FFCC01B85423BD9E38E9BB2C7
S3150801244063B123689A6812F0020FEDD016F8012BD2
S315080124501A73E38E013B9BB2E386EFE700972B469F
S31508012460012202212046FFF7BCFE08B103206FE7CF
S315080124703A4629462046FFF7FDFE18B12023636533
S31508012480012065E7A36833B903932368DA680392E1
S315080124909B680393039B606D003018BF012057E7C3
S315080124A0012055E7012053E7032051E703204FE7B1
S315080124B003204DE703204BE72DE9F04F85B09846F9
S315080124C00E9D90F85030012B04D10223184605B011
S315080124D0BDE8F08F04460F461646012380F85030B2
S315080124E0FCF738FC814694F85130DBB2012B13D046
S315080124F06268B2F5827F07D00223012284F851204F
S31508012500002284F85020E1E7A268002A40F0E4801E
S31508012510042B01D00223F0E7002F00F0DF80002E04
S3150801252000F0DE80B8F1000F00F0DC8094F851303D
S31508012530DBB2012B04BF052384F851300023636500
S31508012540A663A4F83E80A4F83C802763A4F83680E5
S31508012550A4F834802364636423681A6812F0400F70
S3150801256003D11A6842F040021A60E368B3F5006FB6
S3150801257013D063681BB1E38E9BB2012B07D1236885
S3150801258017F8012B1A73E38E013B9BB2E3864FF0D2
S3150801259001084FF0000BC24661E063681BB1E38E88
S315080125A09BB2012B07D1236837F8022BDA60E38E39
S315080125B0013B9BB2E3864FF001084FF0000BC24680
S315080125C018E0E38F9BB263B123689A6812F0010F92
S315080125D007D0DB6826F8023BE38F013B9BB2E38712
S315080125E0D046B5F1FF3F05D0FCF7B4FBA0EB0900D7
S315080125F0854279D9E38E9BB21BB9E38F9BB2002B37
S3150801260048D0B8F1000FDCD0E38E9BB2002BD8D0AE
S3150801261023689A6812F0020FD3D037F8022BDA60D2
S31508012620E38E013B9BB2E386D846CAE7E38F9BB2AA
S3150801263063B123689A6812F0010F07D0DB6833701B
S31508012640E38F013B9BB2E3870136D046B5F1FF3FE5
S3150801265005D0FCF77FFBA0EB0900854246D9E38E3E
S315080126609BB213B9E38F9BB2A3B1B8F1000FDDD0CA
S31508012670E38E9BB2002BD9D023689A6812F0020F19
S31508012680D4D03A781A73E38E013B9BB2E3860137BD
S31508012690D846CBE7CDF800902B46012202212046E9
S315080126A0FFF79FFD08B1032327E74A462946204637
S315080126B0FFF7E0FD034618B12023636501231CE7F4
S315080126C0A268002A7FF419AF03922268D1680391A0
S315080126D092680392039A10E702230EE701230CE797
S315080126E001230AE7012308E7032306E7032304E78F
S315080126F02DE9F04182B004460D4690461E464368D0
S31508012700B3F5827F07D094F85030012B0FD1022000
S3150801271002B0BDE8F0818368002BF4D1042380F868
S315080127205130009613460A46FFF7C6FEF0E7012325
S3150801273084F85030FCF70EFB074694F85130DBB2AB
S31508012740012B07D00220012384F85130002384F895
S315080127505030DDE7002D71D0B8F1000F70D0042399
S3150801276084F8513000236365A563A4F83C80A4F876
S315080127703E802363A386E38623646364A368B3F573
S31508012780004F0BD023681A6812F0400F03D11A685C
S3150801279042F040021A60E36883B129E022681368AF
S315080127A023F480431360EDE7002E4BD0B6F1FF3FCB
S315080127B004D0FCF7CFFAC01B864245D9E38F9BB2FA
S315080127C033B323689A6812F0010FEDD01B7B05F825
S315080127D0013BE38F013B9BB2E387EFE7002E35D040
S315080127E0B6F1FF3F04D0FCF7B5FAC01B86422FD9D4
S315080127F0E38F9BB263B123689A6812F0010FEDD09B
S31508012800DB6825F8023BE38F013B9BB2E387EFE7E1
S315080128106368B3F5827F04D0606D003018BF01206C
S3150801282091E7A368B3F5004F02D0B3F5806FF3D1F2
S315080128302268136823F040031360EDE7012082E75D
S31508012840012080E703207EE703207CE703207AE75F
S31508012850032078E77047022380F839300268136845
S3150801286043F001031360012380F8393000207047D3
S315080128707047704770477047704710B5044603683C
S315080128801A6912F0020F11D0DA6812F0020F0DD090
S315080128906FF002021A610123037603689B6913F03C
S315080128A0030F70D0FFF7E6FF0023237623681A6922
S315080128B012F0040F12D0DA6812F0040F0ED06FF07E
S315080128C004021A610223237623689B6913F4407F65
S315080128D05FD02046FFF7CEFF0023237623681A69C7
S315080128E012F0080F12D0DA6812F0080F0ED06FF046
S315080128F008021A61042323762368DB6913F0030FA0
S315080129004ED02046FFF7B6FF0023237623681A69BF
S3150801291012F0100F12D0DA6812F0100F0ED06FF005
S3150801292010021A61082323762368DB6913F4407FB2
S315080129303DD02046FFF79EFF0023237623681A69B8
S3150801294012F0010F03D0DA6812F0010F36D12368AD
S315080129501A6912F0800F03D0DA6812F0800F34D1A9
S3150801296023681A6912F0400F03D0DA6812F0400F93
S3150801297032D123681A6912F0200F03D0DA6812F0EF
S31508012980200F30D110BDFFF774FF2046FFF773FF04
S315080129908AE72046FFF76DFF2046FFF76CFF9BE7A6
S315080129A02046FFF766FF2046FFF765FFACE720469E
S315080129B0FFF75FFF2046FFF75EFFBDE76FF00102F5
S315080129C01A612046FFF754FFC1E76FF080021A61CA
S315080129D0204600F093F8C3E76FF040021A612046DB
S315080129E0FFF74AFFC5E76FF020021A61204600F09B
S315080129F084F8C7E70368314A90422FD0B0F1804F77
S31508012A002CD0A2F57C42904228D002F580629042F1
S31508012A1024D002F58062904220D002F57842904295
S31508012A201CD0274A90422FD002F5806290422BD0C3
S31508012A3002F58062904227D0A2F59832904223D0BF
S31508012A4002F5806290421FD002F5806290421BD047
S31508012A5003608B68C3620B68836221E023F070030D
S31508012A604A681343154A90420ED0B0F1804F0BD0F5
S31508012A70A2F57C42904207D002F58062904203D0CB
S31508012A8002F58062904213D123F44073CA68134356
S31508012A9003608B68C3620B688362084B984202D055
S31508012AA0084B984201D10B690363012343617047BF
S31508012AB002F578429042E7D0B3E700BF0000014033
S31508012AC00040014000040140A8B110B5044690F841
S31508012AD039305BB1022384F83930211D2068FFF7AC
S31508012AE089FF012384F83930002010BD80F8383079
S31508012AF0FFF7B0FEEEE7012070477047704702689E
S31508012B00D36823F49073D3600268536923F00103F1
S31508012B105361202380F83A30704700002DE9F047C9
S31508012B2004460268136923F44053C1680B431361D1
S31508012B300168CA6822F4164222F00C028368006909
S31508012B40034360690343E06903431343CB60226887
S31508012B50536923F44073A1690B435361E369B3F5E0
S31508012B60004F5FD02568B64B9D4200F0128103F5F0
S31508012B7080639D4200F00D81FDF792FD00EB800018
S31508012B8000EB800063689B00B0FBF3F3DFF8B482C7
S31508012B90A8FB03235B091E01FDF782FD00EB8000FC
S31508012BA000EB800063689B00B0FBF3F7FDF778FD47
S31508012BB000EB800000EB800063689B00B0FBF3F339
S31508012BC0A8FB03235B094FF0640A0AFB13731B0175
S31508012BD03233A8FB03235B0903F0F007FDF760FD19
S31508012BE000EB800000EB800063689B00B0FBF3F903
S31508012BF0FDF756FD00EB800000EB800063689B0043
S31508012C00B0FBF3F3A8FB03235B090AFB13931B0130
S31508012C103233A8FB0323C3F343133B433344AB606B
S31508012C20BDE8F087256803F1804303F510439D420B
S31508012C3059D003F580639D4255D0FDF731FD00EB70
S31508012C40800000EB800063685B00B0FBF3F3DFF8FC
S31508012C50F481A8FB03235B091F01FDF721FD00EBA6
S31508012C60800000EB800063685B00B0FBF3F6FDF7BC
S31508012C7017FD00EB800000EB800063685B00B0FB8A
S31508012C80F3F3A8FB03235B094FF0640A0AFB1363FA
S31508012C90DB003233A8FB03231B0903F4F876FDF79F
S31508012CA0FFFC00EB800000EB800063685B00B0FB73
S31508012CB0F3F9FDF7F5FC00EB800000EB8000636893
S31508012CC05B00B0FBF3F3A8FB03235B090AFB139331
S31508012CD0DB003233A8FB0323C3F342133B443344DB
S31508012CE0AB60BDE8F087FDF7F3FC00EB800000EB75
S31508012CF0800063685B00B0FBF3F3DFF84881A8FB4B
S31508012D0003235B091F01FDF7E3FC00EB800000EBE1
S31508012D10800063685B00B0FBF3F6FDF7D9FC00EBB6
S31508012D20800000EB800063685B00B0FBF3F3A8FB4F
S31508012D3003235B094FF0640A0AFB1363DB00323392
S31508012D40A8FB03231B0903F4F876FDF7C1FC00EB86
S31508012D50800000EB800063685B00B0FBF3F9FDF7C8
S31508012D60B7FC00EB800000EB800063685B00B0FBFA
S31508012D70F3F3A8FB03235B090AFB1393DB00323346
S31508012D80A8FB0323C3F342133B443344AB60BDE8BA
S31508012D90F087FDF79DFC00EB800000EB800063687F
S31508012DA09B00B0FBF3F3DFF89C80A8FB03235B09C8
S31508012DB01E01FDF78DFC00EB800000EB80006368C7
S31508012DC09B00B0FBF3F7FDF783FC00EB800000EBFB
S31508012DD0800063689B00B0FBF3F3A8FB03235B0940
S31508012DE04FF0640A0AFB13731B013233A8FB032352
S31508012DF05B0903F0F007FDF76BFC00EB800000EBC5
S31508012E00800063689B00B0FBF3F9FDF761FC00EBFA
S31508012E10800000EB800063689B00B0FBF3F3A8FB1E
S31508012E2003235B090AFB13931B013233A8FB032314
S31508012E30C3F343133B433344AB60BDE8F08700BF9C
S31508012E40001001401F85EB512DE9F04107460E465A
S31508012E5015469846069C3A68136836EA03030CBF7A
S31508012E6001230023AB421ED1B4F1FF3FF4D02CB1AC
S31508012E70FBF770FFA0EB08008442ECD23A68D368EE
S31508012E8023F4D073D3603A68536923F0010353617D
S31508012E90202387F8393087F83A30002387F8383005
S31508012EA00320BDE8F0810020BDE8F08158B310B5D4
S31508012EB0044690F839300BB3242384F83930226854
S31508012EC0D36823F40053D3602046FFF727FE226810
S31508012ED0136923F4904313612268536923F02A0383
S31508012EE053612268D36843F40053D3600020E0633A
S31508012EF0202384F8393084F83A3010BD80F8383008
S31508012F0018F03CFDD8E7012070472DE9F04782B05B
S31508012F101F4690F83930DBB2202B04D0022318461D
S31508012F2002B0BDE8F08704460E461546002952D080
S31508012F30002A52D090F83830012B01D10223EEE74E
S31508012F40012380F838300023C363212380F8393000
S31508012F50FBF700FF8046A5844FF0000A4FF0800971
S31508012F6012E000974346524649462046FFF76CFF52
S31508012F70002834D122683388C3F3080353602369D0
S31508012F80ABB90236E58CA5B1013DE584A368B3F575
S31508012F90805FE6D000974346524649462046FFF7EA
S31508012FA053FFF0B9236832785A600136EAE70136E9
S31508012FB0E8E700974346002240212046FFF744FFF1
S31508012FC0034608B10323AAE7202284F83920002200
S31508012FD084F83820A3E70123A1E701239FE7032308
S31508012FE09DE703239BE72DE9F04782B01F4690F83A
S31508012FF03A30DBB2202B03D0022002B0BDE8F087BD
S3150801300004460E461546002955D0002A55D090F893
S315080130103830012B01D10220EFE7012380F838303F
S315080130200023C363222380F83A30FBF793FE8246D6
S31508013030A5854FF000094FF020081FE00097534679
S315080130404A4641462046FFF7FFFE002837D1236945
S3150801305033B923685B68C3F3080326F8023B0BE020
S3150801306023685B68DBB226F8013B05E023685B68E9
S3150801307003F07F0333700136E58DADB1013DE5857A
S31508013080A368B3F5805FD9D0009753464A464146AF
S315080130902046FFF7D9FEA0B92369002BE6D123689C
S315080130A05B6833700136E7E7202384F83A3000205D
S315080130B084F83800A1E701209FE701209DE7032056
S315080130C09BE7032099E7000038B590F83940E4B248
S315080130D0202C01D0022038BD002931D0002A31D058
S315080130E090F83830012B01D1022038BD1346044629
S315080130F0012280F8382001628384C3840025C563D0
S31508013100212280F83920026B0F48D063226B0F48C1
S315080131101064226B0E48D064226B1565226804324E
S31508013120206BFCF70FFA23686FF040021A6084F8E7
S3150801313038502268536943F080035361284638BDE5
S31508013140012038BD012038BDED31010825320108BD
S315080131500D33010838B590F83A40E4B2202C01D075
S31508013160022038BD002937D0002A37D090F83830E8
S31508013170012B01D1022038BD13460A460546012115
S3150801318080F83810826283850024C463222180F87E
S315080131903A10416B1248C863696B12480864696B37
S315080131A01148C864696B0C6529680431686BFCF7BA
S315080131B0C9F92A68D36843F48073D3602A685369C6
S315080131C043F0010353612A68536943F0400353618D
S315080131D085F83840204638BD012038BD012038BD64
S315080131E02F320108013301080D33010808B5836B35
S315080131F00268126812F4807F0FD10022DA841968F6
S315080132004A6922F080024A611968CA6842F0400296
S31508013210CA60202283F8392008BD184611F002FE3B
S3150801322008BD704708B5806BFFF7FBFF08BD08B5F9
S31508013230836B0268126812F4807F13D10022DA8543
S315080132401968CA6822F48072CA6019684A6922F044
S3150801325001024A6119684A6922F040024A6120223C
S3150801326083F83A20184615F06DFA08BD08B590F8A6
S315080132703A30DBB2222B01D0022008BD8368B3F5B0
S31508013280805F0ED0036903BB836A5A1C8262026897
S3150801329052681A70C38D013B9BB2C385F3B10020F6
S315080132A008BD826A036943B903685B68C3F3080307
S315080132B01380836A02338362ECE703685B68DBB2D7
S315080132C01380836A01338362E4E7826A531C83624B
S315080132D003685B6803F07F031370DBE70268D36852
S315080132E023F49073D3600268536923F00103536191
S315080132F0202380F83A3015F025FA002008BD7047DA
S3150801330008B5806BFFF7FBFF08BD704710B5846BE6
S315080133102268516994F83930DBB2212B0ED0236823
S315080133205A6994F83A30DBB2222B14D0E36B43F096
S315080133301003E3632046FFF7E8FF10BD11F0800F85
S31508013340EDD00023E384D36823F0C003D3602023A0
S3150801335084F83930E3E712F0400FE7D00023E3851C
S315080133602046FFF7CCFBE1E710B50446026813686F
S31508013370D068516913F00F0F17D113F0200F02D03F
S3150801338010F0200F0DD113F0800F02D010F0800F2E
S3150801339079D113F0400F03D010F0400F40F0A2800E
S315080133A010BD2046FFF762FF10BD11F0010102D1E1
S315080133B010F4907FE7D013F0010F06D010F4807F48
S315080133C003D0E26B42F00102E26313F0040F0DD061
S315080133D0002900F09280E26B42F00202E26313F0E8
S315080133E0020F08D113F0080F0CD10FE013F0020FEA
S315080133F000F0868051B1E26B42F00402E26313F0F9
S31508013400080F03D0E26B42F00802E263E26B002A7E
S31508013410C6D013F0200F02D010F0200F21D1236857
S315080134205A69E36B13F0080F02D112F0400F24D04A
S315080134302046FFF764FB23685A6912F0400F18D03B
S315080134405A6922F040025A61636B73B12F4A1A65B1
S31508013450606BFCF7C1F80028A2D0606B036D984732
S3150801346010BD2046FFF702FFD9E72046FFF74DFFBB
S3150801347010BD2046FFF749FF10BD2046FFF745FF5F
S315080134800023E36310BD94F83930DBB2212B87D1D1
S31508013490A368B3F5805F16D0236A591C21621B788D
S315080134A05360E38C013B9BB2E384002B7FF478AF36
S315080134B02268D36823F08003D3602268D36843F077
S315080134C04003D36010BD236A1B88C3F30803536006
S315080134D023691BB9236A02332362E2E7236A0133AC
S315080134E02362DEE7D36823F04003D360202384F800
S315080134F03930204611F096FC10BD13F0020F85D124
S3150801350013F0080F82D0002980D07BE71135010816
S3150801351008B5806B0023C385C384FFF7F6FE08BD93
S3150801352084B010B402AC84E80E0042680399029B89
S315080135300B4304990B4305990B4306990B430799CA
S315080135400B4322F4FD4222F07F021343436000201D
S315080135505DF8044B04B07047D0F8800070470B68DB
S31508013560C0F88030002070470323036000207047AD
S31508013570006800F00300704710B40B688360C268E6
S315080135804B688C682343CC68234309690B4322F4AF
S315080135907F6222F00F021343C36000205DF8044BDB
S315080135A070470069C0B2704782B000230193034B8C
S315080135B003440193019B186802B07047142C01401B
S315080135C010B40B6843624B688362C26A8B68CC6825
S315080135D023430C69234349690B4322F0F70213433A
S315080135E0C36200205DF8044B704700000E49D1F80C
S315080135F0883043F47003C1F888300C4B1A6842F0DE
S3150801360001021A60002098601A6822F0847222F476
S3150801361080321A60064A5A601A6822F480221A60B1
S31508013620D860044B8B60704700ED00E0003802401B
S31508013630103000240080000810B582B002AB03F8F0
S31508013640011D0268546801221946A04702B010BD3F
S315080136504FF0FF3070474FF0FF307047704710B595
S3150801366014464FF0FF3392B20069FFF74EFC20462D
S3150801367010BD00B583B04FF0FF3301220DF10701EC
S315080136800069FFF7B0FC9DF8070003B05DF804FB7D
S31508013690FEE70120704700001622024B1A604FF020
S315080136A0FF307047C0DA002010B51446012807D04C
S315080136B002280DD009220A4B1A604FF0FF3010BDBF
S315080136C04FF0FF3392B20748FFF71FFC204610BDA3
S315080136D04FF0FF3392B20348FFF717FC204610BD9F
S315080136E0C0DA0020ECD4002008B503460A4A10685F
S315080136F0EFF308820344934202D8074A136008BDD0
S31508013700192206490220FFF7CFFF0C22044B1A6043
S315080137104FF0FF3008BD00BF080000201C770308E2
S31508013720C0DA002010B50446FCF7B4FF054BA3FB2D
S315080137300030000D04FB00F00A380138B0F1FF3FF4
S31508013740FBD110BD83DE1B4308B5FBF709FB08BD9A
S3150801375008B50120FFF7E6FF08BD08B50A20FFF7FF
S31508013760E1FF08BD10B582B018468DF8072001396A
S31508013770062919D8DFE801F0041B2A3B4C565600E6
S315080137802D4C002210212046FCF7A8F90120FBF751
S31508013790E7FA012210212046FCF7A0F901224FF48D
S315080137A000412648FCF79AF9012002B010BD9DF8A0
S315080137B007302BB9002220211F48FCF78FF9F3E7C0
S315080137C0012220211C48FCF789F9EDE79DF807300D
S315080137D033B901224FF400411848FCF77FF9E3E7B2
S315080137E000224FF400411548FCF778F9DCE79DF80B
S315080137F007303BB9002210210F48FCF76FF9FFF794
S31508013800ACFFD1E7012210210B48FCF767F9F6E76F
S315080138104FF47A7301220DF1070109480068FEF792
S315080138207CFDC1E74FF47A739DF8072001460448E9
S315080138300068FEF772FDB7E7000402400000024087
S31508013840740A002008B5084B186001224FF400419C
S315080138500648FCF743F90A20FBF782FA044A0549A8
S31508013860054800F0D3FC08BD740A00200000024098
S31508013870653701081000002078DA00202DE9F04F9D
S3150801388089B007460D46039116469B46BDF8484042
S31508013890DDF84CA0009400F05CF8002856D0002C06
S315080138A054D00BF10703C3F3CC0304933444A3B2F6
S315080138B00593ABF108039BB2DA080132069223F0AD
S315080138C007032A460F321344079318E05B46554609
S315080138D032E00135ADB24FEA5808AC4208D018F0CB
S315080138E0010FF6D032462946384600F0DCFCF0E7EF
S315080138F0049B9A440136B6B2059B9E4226D0039B89
S31508013900DC1DA4B2BBF1070FE0D9069B0AEB03093C
S3150801391055464FF0020815F8013B009343463246D7
S315080139202146384600F0C6FC0834A4B24D45F2D10A
S315080139300BF00703BDF81C40002BD9D095F8008081
S31508013940E51FADB21C44073CA4B2C8E709B0BDE8FF
S31508013950F08F70B4BDF80C40013C1444A4B2C58F75
S31508013960B0F84260964215D3AC4204D2A24294BF43
S3150801397000220122FAB1013B0B449BB2828FB0F8B7
S31508013980400088420DD3934217D2994294BF002032
S3150801399001200EE0AC420BD3A24294BF00220122C1
S315080139A0E8E793420BD3994294BF0020012000E037
S315080139B0002070BC70470020FBE70120F9E70020D2
S315080139C0F7E710B58C6800230121A04710BD10B593
S315080139D08C6800230321A04710BD10B58C6800230D
S315080139E01A460421A04710BD10B58C680023012290
S315080139F00421A04710BD10B58C6800230221A047F9
S31508013A0010BD10B58C6800230521A04710BD2DE90E
S31508013A10F84F07468B46551E0026B0464FF0FF0A5B
S31508013A204FF0010941E0FF2C11D0FE2C4BD0EF2CB1
S31508013A304CD8DF2C14D8CF2C1AD8BF2C20D814F088
S31508013A40800F45D12046FFF77FFE46462DE05246B8
S31508013A5059463846FFF7D5FF0646A0B3464624E041
S31508013A6004F00F0259463846FFF7C5FF46461CE0E3
S31508013A7004F00F0259463846FFF7A9FF464614E0F7
S31508013A8059463846FFF7A9FF2401023404F0FE041B
S31508013A902046FFF759FE59463846FFF7A5FF204647
S31508013AA0FFF752FE464600E04E4615F8014F002E36
S31508013AB0B9D1FF2CF8D0224659463846FFF7A1FF5F
S31508013AC00028F2D106463046BDE8F88F4646ECE7AF
S31508013AD04646EAE72DE9F04103F1FF3E013A53FA7A
S31508013AE082FC00240F4B104A1EF8015F661C03EB8B
S31508013AF0040805F00F0717443F7D88F8087002345B
S31508013B00E4B253FA86F602EB15152D7D3572E645B4
S31508013B10EAD18C68054B80220621A0470120BDE821
S31508013B20F08100BF780A002084FD0208800A00207F
S31508013B3001207047F8B506460D464B681F7A1C8862
S31508013B4007FB042404F0FF040E4AFFF760FF224630
S31508013B5029463046FFF755FF621CD2B22946304640
S31508013B60FFF74FFF002229463046FFF744FF5C2244
S31508013B7029463046FFF745FF012229463046FFF719
S31508013B803AFFF8BDA8FD02082DE9F04F83B00646B5
S31508013B900D4690469B46A2F10A030B2B0FD8DFE888
S31508013BA003F0060E0E0E0E4162670E0E0E17022266
S31508013BB0FFF707FF314A29463046FFF728FF5B46DC
S31508013BC042462946304600F06DFD03B0BDE8F08F48
S31508013BD0D1F80490D9F80C70B9F80AA04FEA9A0AF4
S31508013BE0B9F80030002BEAD000245FFA8AF3019372
S31508013BF0224629463046FFF79DFF3B46019A29464C
S31508013C003046FFF767FFFFF7A3FD00222946304636
S31508013C10FFF7DDFE57440134E4B2B9F80030A34298
S31508013C20E6D8CCE70122FFF7D2FE00222946304624
S31508013C30FFF7E1FEC12229463046FFF7E2FE0122DF
S31508013C4029463046FFF7D7FE9BF800205208294639
S31508013C503046FFF7D6FEFFF77BFD002229463046A0
S31508013C60FFF7B5FEABE7064AFFF7D1FE0120ACE741
S31508013C70044AFFF7CCFE0120A7E700BFB8FD0208FA
S31508013C8038FE020844FE02082DE9F04F83B00646C5
S31508013C900D4690469B46A2F10A030B2B0FD8DFE887
S31508013CA003F0060E0E0E0E3F5E630E0E0E1702226F
S31508013CB0FFF787FE2F4A29463046FFF7A8FE5B46DF
S31508013CC042462946304600F025FC03B0BDE8F08F90
S31508013CD0D1F80490D9F80C70B9F80AA04FEA9A0AF3
S31508013CE0B9F80030002BEAD000245FFA8AF3019371
S31508013CF0224629463046FFF71DFF3B46019A2946CB
S31508013D003046FFF7E7FE002229463046FFF75FFEF9
S31508013D1057440134E4B2B9F80030A342E8D8CEE7F3
S31508013D200122FFF754FE002229463046FFF763FEBB
S31508013D30C12229463046FFF764FE0122294630464C
S31508013D40FFF759FE9BF80020520829463046FFF72F
S31508013D5058FE002229463046FFF739FEAFE7064AE4
S31508013D60FFF755FE0120B0E7044AFFF750FE012090
S31508013D70ABE700BFB8FD020838FE020844FE020898
S31508013D804218435C507800EB032080B270470078F4
S31508013D90704708B5FFF7FBFF18B1022801D00320C9
S31508013DA008BD062008BD0020704790F9290001309A
S31508013DB080B2704708B50621FFF7E2FF08BD08B5CE
S31508013DC00821FFF7DDFF08BD807A7047C07A704782
S31508013DD02DE9F84F80460E46D0F808B05846FFF749
S31508013DE0D6FF82465846FFF7D4FF8146BAF1010F3E
S31508013DF014BFFF270F275846FFF7E6FF0446584624
S31508013E00FFF7E4FF05465846FFF7D9FF602E03D9A9
S31508013E1010B1584461240AE05846FFF7CBFF402EFB
S31508013E2003D910B15844412401E00BF11100B54200
S31508013E300ED3AC421ED9002088F81C0088F81F0052
S31508013E4088F8200088F81D0088F81E00BDE8F88F5C
S31508013E50002088F81C0088F81F0088F8200088F8D8
S31508013E601D0088F81E00BDE8F88F0130AC42E2D08B
S31508013E700134E4B20378FF2BF7D0B44204D0837837
S31508013E803B404B441844F1E7BAF1000F18D0BAF198
S31508013E90020F15D003F00F02023A88F81E201B09FB
S31508013EA088F81D30437803F00F0288F820201B0993
S31508013EB088F81F3083781B0988F81C30BDE8F88F0D
S31508013EC088F81F30437888F82030C37888F81C3082
S31508013ED0037988F81D30437988F81E30BDE8F88FD4
S31508013EE02DE9F04F85B007468A4616461946FFF76B
S31508013EF06FFF002853D00546B868FFF74AFF80468A
S31508013F0097F81F9097F8204097F91D309A441FFAA1
S31508013F108AF319460393A2B297F91E301344F61A87
S31508013F20B6B200924B4632463846FFF712FDA0B1AB
S31508013F3009F10709C9F3C40302935CB304F1FF3A13
S31508013F405FFA8AFA0AF1010AB2441FFA8AFA454463
S31508013F50013BDBB203F1010B13E097F91C001BE0EF
S31508013F6015F8013B0093434632462146384600F090
S31508013F70A1F90834A4B2A945F2D10136B6B2B245BF
S31508013F8008D0029B002BF8D005EB0B09039C4FF0D8
S31508013F900008E5E797F91C0005B0BDE8F08F002099
S31508013FA0FAE72DE9F04180460C4617461E46436A54
S31508013FB098470744337893B1BFB200253A4621465C
S31508013FC04046FFF78DFF80B20444A4B20544ADB262
S31508013FD016F8013F002BF1D12846BDE8F0810025EE
S31508013FE0FAE78368CBB190F82820BAB95A7980F8EC
S31508013FF029201B7B80F82A3090F9293090F92A204C
S315080140009B1A9BB290F82B20402A04D0DBB202FB04
S3150801401003F3C3F38F1380F82C307047012A06D0B7
S315080140205A7B80F829209B7B80F82A30E4E7DA7BE3
S3150801403080F829201B7C80F82A30DDE708B50022A4
S3150801404080F82820FFF7CDFF08BD08B5012380F8C1
S315080140502830FFF7C6FF08BD014B4362704700BF12
S31508014060A73D0108014B4362704700BFAB3D0108FC
S3150801407070B50D46097871B1064600243046FFF73A
S31508014080A7FE96F91C301C44A4B215F8011F002995
S31508014090F4D1204670BD0024FBE7000083688B42FB
S315080140A007D010B504468160FFF79BFF014B636299
S315080140B010BD7047A73D010810B50C68A04710BD93
S315080140C038B504460D46836B0220984700230A2219
S315080140D029462046FFF7F0FF0546A36B03209847BC
S315080140E0A36B00209847284638BD38B504460D46C7
S315080140F0836B02209847A36B01209847002314225B
S3150801410029462046FFF7D8FF04F13C031722294622
S315080141102046FFF7D1FFA36B0020984738BD70B53D
S3150801412004460D46836B02209847A36B01209847E6
S315080141300023152229462046FFF7BEFF064620B969
S31508014140A36B00209847304670BD04F13C03172243
S3150801415029462046FFF7B0FFF2E700B583B002AB68
S3150801416003F8012D0F22FFF7A7FF03B05DF804FB43
S3150801417010B5C285038600F12E033222FFF79CFF94
S3150801418010BD00B583B00DF106034622FFF794FF73
S31508014190BDF8060003B05DF804FB00B583B00DF168
S315080141A006034722FFF788FFBDF8060003B05DF84E
S315080141B004FB08B500234822FFF77EFF08BD10B5AA
S315080141C004464168FFF7DDFF208061682046FFF756
S315080141D0E4FF608061682046FFF7EBFFE07404F1B5
S315080141E03C03172261682046FFF766FF10BD10B52C
S315080141F004464168FFF764FF034608B9184610BD2F
S315080142002046FFF7DCFF0123F8E700002DE9F0411E
S3150801421004460F46904600258560C560457401260B
S31508014220067422238374856180F83460FFF714FFCE
S3150801423084F8286084F8295084F82A50402384F8A1
S315080142402B3084F82C50054BA3636760C7F80880A8
S315080142502046FFF7CCFFBDE8F08100BF914A01086F
S3150801426008B54168FFF741FF08BD10B504468369E3
S3150801427003B1984761682046FFF751FF10BD08B59D
S315080142800A464168FFF769FF08BD08B500231022F1
S315080142904168FFF711FF08BD08B5002311224168DF
S315080142A0FFF70AFF08BD08B513460A464168FFF736
S315080142B05FFF08BD38B54568C185028680F8333089
S315080142C09DF8103080F8323000F12E033B22294642
S315080142D0FFF7F2FE38BD80F834107047C37C282BEF
S315080142E004D0022B0CBF032001207047FF20704722
S315080142F0C37C302B06D010B50446FFF7EFFF84F8D0
S31508014300340010BDFF2380F8343080F8353070470B
S31508014310002282800388013BC380027270470288AB
S31508014320838813449BB2838041888B420DD2037ADA
S3150801433001330372C3881A4492B291429CBF01F1B8
S31508014340FF3292B2C2800120704700207047C368CD
S3150801435042891A44002103F8011B9A42FBD170478E
S3150801436010B4C3888B4234BF00230123914294BF02
S3150801437000210121848843EA010094428CBF002070
S3150801438000F001000B4018435DF8044B7047002309
S315080143900B8083884B804389013B8B80C388CB8004
S315080143A0704708B54B884A79012A03D0032A08D0F1
S315080143B01A4602E003F1080292B21946FFF7D0FF46
S315080143C008BDA3F108011A468BB2F6E770B49DF849
S315080143D00C60C4684589AD088088121AD2B212FBEE
S315080143E005F2880810FA82F2490001F0060136B989
S315080143F003208840C0B2A55C25EA0000A05403F05A
S31508014400030303FA01F1A35C1943A15470BC704775
S31508014410C368428903EB4202002103F8011B9A4251
S31508014420FBD1704730B583B04C888388A34206D840
S31508014430C388A34203D30D884389AB4201D803B08D
S3150801444030BD8B79009222462946FFF7BFFFF6E772
S31508014450F8B507460D460C7900260CE03246294682
S315080144603846FFF7DFFF09E02B8801332B8064000C
S3150801447014F0FF041CD014F0800FEFD16B79032BD5
S31508014480F5D801A252F823F06944010899440108B4
S31508014490A1440108A94401086B8801336B80E6E74A
S315080144A02B88013B2B80E2E76B88013B6B80DEE7BB
S315080144B0F8BD00BFF8B507460D460C79012606E09A
S315080144C02B8801332B80A40014F0FF0420D0A30904
S315080144D0AB71324629463846FFF7A4FF6B79032BA1
S315080144E0F1D801A252F823F0C1440108F9440108A0
S315080144F001450108094501086B8801336B80E2E72C
S315080145002B88013B2B80DEE76B88013B6B80DAE762
S31508014510F8BD00BF38B51D464C68143A342A1CD874
S31508014520DFE802F03E461B501B1B1B1B1B1B1B1BFC
S315080145301B1B1B1B1B1B1B1B1B1B1B1B37311B1B8A
S315080145401B1B2A1B1B1B1B1B1B1B1B1D1B1B1B1B9B
S315080145501B1B1B1B1B1B565A5E00012341E02946E8
S315080145602046FFF71EFF08B901233AE029462046EF
S31508014570FFF76EFF012334E0002229462046FFF7A4
S3150801458051FF01232DE029462046FFF793FF01231A
S3150801459027E0012229462046FFF744FF012320E0B0
S315080145A02046FFF7B5FE2046FFF732FF012318E044
S315080145B02046FFF7B4FE034698B12046FFF728FFC9
S315080145C001230EE029462046FFF7E1FE012308E014
S315080145D063892B80012304E063882B80012300E093
S315080145E00223184638BD30B4C4684589AD088088A9
S315080145F0121AD2B212FB05F2880810FA82F24900A1
S3150801460001F0060103208840C0B203F003038B4082
S31508014610A15C21EA00011943A15430BC70474A88BC
S31508014620838893420DD8C38893420AD310B50C8860
S315080146304389A34200D810BD8B792146FFF7D3FFE2
S31508014640F9E7704770B506460D460C790BE0294621
S315080146503046FFF7E4FF09E02B8801332B8064001D
S3150801466014F0FF041CD014F0800FF0D16B79032BE2
S31508014670F5D801A252F823F05946010889460108DE
S3150801468091460108994601086B8801336B80E6E774
S315080146902B88013B2B80E2E76B88013B6B80DEE7C9
S315080146A070BD00BF38B51D464C68143A342A1CD86B
S315080146B0DFE802F030381B421B1B1B1B1B1B1B1B95
S315080146C01B1B1B1B1B1B1B1B1B1B1B1B1B1B1B1B2B
S315080146D01B1B2A1B1B1B1B1B1B1B1B1D1B1B1B1B0A
S315080146E01B1B1B1B1B1B484C5000012333E029468F
S315080146F02046FFF756FE08B901232CE02946204635
S31508014700FFF7A0FF012326E029462046FFF787FF8A
S31508014710012320E02046FFF71AFE2046FFF7F8FDA1
S31508014720012318E02046FFF7FAFD034698B1204613
S31508014730FFF70DFE01230EE029462046FFF727FE67
S31508014740012308E063892B80012304E063882B8019
S31508014750012300E00223184638BD2DE9F04782B04F
S3150801476082460C4617469846072B17D9A3F1080522
S3150801477025F0070501F108031D44ADB2FF264FF0E8
S31508014780000900964B463A4621465046FFF792FDE8
S315080147900834A4B2AC42F4D108F00708B8F1000F06
S315080147A002D102B0BDE8F08788F00703013303F0B0
S315080147B00703FF2202FA03F3DBB2009300233A460A
S315080147C021465046FFF776FDEBE72DE9F04782B023
S315080147D082460F4614469846072B17D9A3F10805B2
S315080147E025F0070502F108031D44ADB2FF264FF077
S315080147F0010900964B46224639465046FFF75AFDAF
S315080148000834A4B2AC42F4D108F00708B8F1000F95
S3150801481002D102B0BDE8F08788F00703013303F03F
S315080148200703FF2202FA03F3DBB2009301232246B0
S3150801483039465046FFF73EFDEBE72DE9F04182B0D8
S3150801484006460F4615469846BDF820400094FFF7E0
S3150801485080F810B902B0BDE8F08143462A463946C8
S315080148603046FFF77AFF23462A4639463046FFF790
S31508014870ACFF08F1FF31394423462A4689B230464E
S31508014880FFF7A3FF013C2C444346A2B23946304602
S31508014890FFF763FFDEE72DE9F04180460F4615462F
S315080148A01E46BDF8184033462A4639464046FFF7A4
S315080148B054FF0135ADB2013CA4B2002CF3D1BDE8D9
S315080148C0F0812DE9F04182B005460E461746984615
S315080148D0BDF820400094FFF73CF810B902B0BDE8D6
S315080148E0F081009443463A4631462846FFF7D3FFFE
S315080148F0F4E7002070472DE9F843054617461C469C
S315080149004E68A2F11703302B1AD8DFE803F02019F5
S3150801491019191919191919191919191919191919F8
S31508014920191919617E1919191961191919191919F3
S3150801493019197E19191919191919191919535A0011
S3150801494023463A463146FFF7B7FBBDE8F8832346C7
S3150801495017223146FFF7B0FB31462846FFF711FC0F
S31508014960B4F804906FEA090981441FFA89F93146B6
S315080149702846FFF706FC2788FF430744BFB231469E
S315080149802846FFF70AFCB4F806806FEA080880444F
S315080149901FFA88F831462846FFF7FFFB6388DB4391
S315080149A01844A4F80090A4F80280A780E0800120AA
S315080149B0BDE8F8833146FFF7E4FB20800120BDE816
S315080149C0F8833146FFF7E9FB20800120BDE8F8832B
S315080149D03146FFF7E2FBB4F802806FEA0808804423
S315080149E01FFA88F831462846FFF7CBFB2388DB43B5
S315080149F018442080A4F8028023463A4631462846C0
S31508014A00FFF75AFB0120BDE8F8833146FFF7C5FBDE
S31508014A10B4F802806FEA080880441FFA88F831461C
S31508014A202846FFF7AEFB2388DB4318442080A4F809
S31508014A3002806379023303F00303637123463A461E
S31508014A4031462846FFF738FB0120BDE8F883000008
S31508014A5008B54268044B9A4200D008BD5B684360BA
S31508014A60FFF7ADFBF9E700BF8C00002008B54368E6
S31508014A70054A93421CBF53604260044A024B1A60BE
S31508014A80FFF79DFB08BD00BF8C000020F748010811
S31508014A907047FF2808DDB0F5007F07DBB0F5407FDA
S31508014AA0B4BFA520A7207047A1207047A32070474F
S31508014AB070B584B0841840F2FE339C4202DD0020B2
S31508014AC004B070BD15460E460446FFF7E2FF0A23F9
S31508014AD00293019500960123E2B2C1B20248FBF79F
S31508014AE03FFB0120ECE700BFF0D3002070B586B08C
S31508014AF0841840F2FE339C4202DD002006B070BDE8
S31508014B0015460E460446FFF7C4FF0A23029301958C
S31508014B1005AB00930123E2B2C1B20648FBF720FBBD
S31508014B209DF814209DF8153043EA022333800120AD
S31508014B30E4E700BFF0D3002070B584B0841840F2D2
S31508014B40FE339C4202DD002004B070BD15460E46B8
S31508014B500446FFF79EFF0A23029301950096012357
S31508014B60E2B2C1B20248FBF7FBFA0120ECE700BF4B
S31508014B70F0D30020FF2808DDB0F5007F07DBB0F58C
S31508014B80407FB4BFA420A6207047A0207047A2206A
S31508014B907047000070B584B0841840F2FE339C4219
S31508014BA002DD002004B070BD15460E460446FFF727
S31508014BB0E1FF0A230293019500960123E2B2C1B2ED
S31508014BC00348FBF729FA0420FAF7CAF80120E9E7AE
S31508014BD0F0D3002070B584B0841840F2FE339C42AD
S31508014BE002DD002004B070BD15460E460446FFF7E7
S31508014BF0C1FF0A230293019500960123E2B2C1B2CD
S31508014C000348FBF709FA0420FAF7AAF80120E9E7AD
S31508014C10F0D3002030B587B00B8819128DF814101F
S31508014C208DF81530811840F2FE33994202DD0020D5
S31508014C3007B030BD15460446FFF79CFF0A230293C9
S31508014C40019505AB00930123E2B2C1B20348FBF714
S31508014C50E3F90420FAF784F80120E9E7F0D3002004
S31508014C600170002242708270C2704260C2600261A5
S31508014C700F494161A1F1B561A1F58B318161C2612C
S31508014C800262426202854285C26240F6B8310186F5
S31508014C900849416341F288310187428702218187A8
S31508014CA0C287082180F8401080F84120704700BF6C
S31508014CB0008BD482801A060070B582B0047861F040
S31508014CC07F018DF800108DF801208DF802309DF8CE
S31508014CD018308DF803309DF81C308DF80430032CFC
S31508014CE001DD02B070BD0B4E0B4D002236F81410D3
S31508014CF02846FAF7F3FE4FF47A7305226946074800
S31508014D00FDF70BFB012236F814102846FAF7E6FEE2
S31508014D10E7E700BFA0000020000C024094D1002064
S31508014D2000B583B0CBB20193C1F307230093C1F356
S31508014D3007430A0E2D21FFF7BFFF03B05DF804FBF9
S31508014D4000B583B0084A8A42A8BF0A46D3B201937E
S31508014D50C2F307230093C2F30743120E2721FFF775
S31508014D60ABFF03B05DF804FB00FE7F0000B583B01E
S31508014D704FF6FF728A42A8BF0A46D3B20193C2F31D
S31508014D8007230093C2F30743120E2821FFF794FF66
S31508014D9003B05DF804FB30B583B005460C464FF603
S31508014DA0FF728A42A8BF0A46D3B20193C2F3072308
S31508014DB00093C2F30743120E2621FFF77DFF214612
S31508014DC02846FFF7D3FF03B030BD2DE9F04383B082
S31508014DD006460D46042301930024009423462246E1
S31508014DE02021FFF769FF2F0EC5F30748C5F30729E9
S31508014DF0EDB20195CDF8009043463A462121304659
S31508014E00FFF75AFF0195CDF8009043463A462D2102
S31508014E103046FFF751FF019400942346224620218C
S31508014E203046FFF749FF03B0BDE8F08300B583B00C
S31508014E300192009100221021FFF73EFF03B05DF8B1
S31508014E4004FB0000042B00DD70472DE9F0411C46E8
S31508014E5016460D46DFF834800A4F002238F813103B
S31508014E603846FAF73BFEC823B2B229460648FDF78B
S31508014E7054FA012238F814103846FAF72FFEBDE81D
S31508014E80F08100BF000C024094D10020A000002050
S31508014E90F0B587B00546274B93E8030004908DF8D3
S31508014EA01410C823052204A92348FDF736FA2978E0
S31508014EB00122224B33F811102148FAF70FFE214F30
S31508014EC02B78214E012237F813103046FAF706FEE1
S31508014ED00A20F9F745FFA1238DF8083000248DF83B
S31508014EE009408DF80A408DF80B408DF80C402B7857
S31508014EF0052202A92846FFF7A5FF0A20F9F730FF80
S31508014F00AD238DF800308DF801408DF802408DF8FB
S31508014F1003408DF804402B78052269462846FFF799
S31508014F2091FF2B78224637F813103046FAF7D6FD4B
S31508014F3007B0F0BD3473030894D10020A000002007
S31508014F40000C0240A80000200008024030B591B0CC
S31508014F50044605783A4B03F1280292E803000E90BD
S31508014F608DF83C1003F1380292E803000C908DF895
S31508014F70341003F1400292E803000A908DF82C10D0
S31508014F8093228DF8202000228DF821208DF82220E9
S31508014F908DF823208DF8242003F1480292E80300B6
S31508014FA006908DF81C1003F1500292E80300049054
S31508014FB08DF8141003F1580292E8030002908DF857
S31508014FC00C10603393E8030000908DF804102B460B
S31508014FD005220EA92046FFF735FF2B4605220EA905
S31508014FE02046FFF72FFF2B4605220CA92046FFF77F
S31508014FF029FF2B4605220AA92046FFF723FF2B4640
S31508015000052208A92046FFF71DFF2B46052206A9FA
S315080150102046FFF717FF2B46052204A92046FFF76E
S3150801502011FF2B46052202A92046FFF70BFF2B4647
S31508015030052269462046FFF705FF11B030BD00BFBE
S315080150403473030830B58BB004460578264B03F153
S31508015050080292E8030008908DF8241003F1100263
S3150801506092E8030006908DF81C1003F1680292E895
S31508015070030004908DF81410203393E8030002907E
S315080150808DF80C1080238DF8003000238DF801303F
S315080150908DF802308DF803308DF804302B46052241
S315080150A008A92046FFF7CEFE2B46052208A9204669
S315080150B0FFF7C8FE2B46052206A92046FFF7C2FEC2
S315080150C02B46052204A92046FFF7BCFE2B460522DE
S315080150D002A92046FFF7B6FE2B4605226946204659
S315080150E0FFF7B0FE0BB030BD3473030830B587B097
S315080150F0044605781B4B93E8030004908DF81410B9
S31508015100AD238DF8083000238DF809308DF80A3063
S315080151108DF80B308DF80C30A1228DF800208DF812
S3150801512001308DF802308DF803308DF804302B46A6
S31508015130052204A92046FFF785FE2B46052204A968
S315080151402046FFF77FFE2B46052202A92046FFF7D8
S3150801515079FE2B46052269462046FFF773FE07B0FE
S3150801516030BD00BF3C73030830B593B004460578DB
S315080151703D4B03F1700292E8030010908DF844103C
S31508015180A5228DF8382000228DF839208DF83A208D
S315080151908DF83B208DF83C2003F1780103C90C906A
S315080151A08DF8341003F1800103C90A908DF82C108B
S315080151B003F1880103C908908DF8241003F19001C1
S315080151C003C906908DF81C1003F1980103C90490D0
S315080151D08DF81410A0218DF808108DF809208DF886
S315080151E00A208DF80B208DF80C200B4493E8030058
S315080151F000908DF804102B46052210A92046FFF7CA
S3150801520021FE2B4605220EA92046FFF71BFE2B463B
S3150801521005220CA92046FFF715FE2B4605220AA9E9
S315080152202046FFF70FFE2B46052208A92046FFF761
S3150801523009FE2B46052206A92046FFF703FE2B4643
S31508015240052204A92046FFF7FDFD2B46052202A9E2
S315080152502046FFF7F7FD2B46052269462046FFF74C
S31508015260F1FD13B030BD00BF347303082DE9F041D9
S31508015270044690461F469DF818509DF81C60012962
S315080152801CD002291DD02046FFF76EFFC4F83480D2
S3150801529041462046FFF754FD278639462046FFF743
S315080152A07AFD84F8405084F841609DF820303246F2
S315080152B029462046FFF7BAFDBDE8F081FFF7C2FE91
S315080152C0E1E7FFF743FEDEE782B001238DF80730F9
S315080152D09DF8070002B0704700B583B005990191A2
S315080152E00499009101460448FCF77CFD003018BF7B
S315080152F0012003B05DF804FB0010002000B583B05F
S31508015300059901910499009101460448FCF731FE7B
S31508015310003018BF012003B05DF804FB001000201F
S315080153202DE9F04F8BB0804600250095694B5A6CE4
S3150801533042F400625A645A6C02F400620092009ABE
S3150801534001951A6B42F480021A631A6B02F4800201
S315080153500192019A02951A6B42F002021A631A6BBC
S3150801536002F002020292029A03951A6B42F00402B3
S315080153701A631A6B02F004020392039A04951A6BD4
S3150801538042F008021A631B6B03F008030493049B9B
S3150801539007230593022706970795032608960C24E3
S315080153A0099405A94C48FAF71DFA4FF410630593B9
S315080153B0069707950896099405A94848FAF712FA2F
S315080153C04FF00409CDF814900697079508960994A5
S315080153D005A94348FAF706FA2A4605213120F9F7BD
S315080153E04DFF3120F9F77AFF3E4C4FF0006BC4F8B8
S315080153F064B0A566E5664FF4806AC4F870A04FF4F8
S31508015400805363674FF48043A3672023E3674FF410
S315080154104033C4F88030C4F88490C4F888604FF4E7
S315080154200003C4F88C304FF40013C4F890302746B3
S315080154302D4B47F8603FC8F85870C4F8988038462D
S31508015440FAF754F83846F9F7B1FFC4F8C4B040235F
S31508015450C4F8C830C4F8CC50C4F8D0A04FF480536F
S31508015460C4F8D4304FF48043C4F8D8302023C4F8A4
S31508015470DC304FF44033C4F8E030C4F8E490C4F8A3
S31508015480E8604FF40003C4F8EC304FF40013C4F895
S31508015490F0302646154B46F8C03FC8F85C60C4F89C
S315080154A0F8803046FAF722F83046F9F77FFF2A46A0
S315080154B006213B20F9F7E2FE3B20F9F70FFF2A46C2
S315080154C006214520F9F7DAFE4520F9F707FF0BB063
S315080154D0BDE8F08F0038024000040240000802408F
S315080154E0000C02400010002058640240A0640240EB
S315080154F010B5144B144A1A6000225A609A60DA6091
S315080155001A614FF4804159619A61FFF7DDFE01285E
S3150801551001D0022010BD0B4C00212046FFF700FFE9
S3150801552004F590712046FCF7A1F908B1012010BDD8
S315080155304FF400612046FCF791FB003018BF0120AB
S3150801554010BD00BF00100020002C014008B502481C
S31508015550FBF7FEFF08BD00BF0010002008B5024B8F
S31508015560D86DFAF74DF808BD0010002008B5024BB2
S31508015570986DFAF745F808BD0010002008B50248ED
S31508015580FCF70CFE08BD00BF0010002008B5014657
S315080155900148FCF721F808BD0010002000000000B2
S315080155A070B582B0002501951F4B1A6C42F00102B5
S315080155B01A641B6C03F0010301931C4C4FF08043E2
S315080155C023600126DE606560A56010EE100AF2F719
S315080155D099FF02460B4612A1D1E90001F3F710F92A
S315080155E00022134BF2F72EFEF3F7D8FA07EE900ACC
S315080155F0FCEEE77AC4ED037A256165612046FDF77D
S3150801560063FA2046FDF727F92A4631461C20F9F7A1
S3150801561035FE1C20F9F762FE02B070BDAFF30080BB
S31508015620000000002A759541003802403812002012
S315080156300000F03F10B5144C04F13C011348F9F78A
S31508015640B5FA0122124904F14000F8F797FBC0B1F7
S315080156500D2804D00F48F9F7CDFA002010BD002215
S31508015660114604F13C00F8F789FF0028F2D101221E
S31508015670074904F14000F8F781FB0028EAD1012027
S3150801568010BD012010BD00BF3812002038FD0208E8
S31508015690707703087412002010B504460649F8F716
S315080156A056FE08B9012010BD2046F8F77EFEB0FA6D
S315080156B080F0400910BD00BFAC140020F0B5ADF56F
S315080156C0597D304A137852782F49B1F894120091CE
S315080156D02E4945A817F07CFF0A2245A94DA8F8F7D7
S315080156E08FFB18B100200DF5597DF0BD45AA284953
S315080156F005A817F06DFF05A8F3F7A0FA04AB024653
S3150801570005A94DA8F8F796FC002836D11E4BD3F803
S315080157109832002B1DDD1F4C00251F4EA4F5277757
S31508015720E3680293A36801936368009323682A4692
S31508015730314605A817F04CFF04AB024605A94DA84A
S31508015740F8F778FCD8B901351034D7F89832AB4256
S31508015750E6DC4DA8F8F7E2FD04460B49B1F89432A8
S315080157600133A1F89432022201F525710520FFF7CC
S3150801577051FAB4FA84F04009B5E70020B3E70020EE
S31508015780B1E700BF9800002038120020747703089B
S315080157908C770308D4140020907703082DE9F0418B
S315080157A0ADF5567D0A4A137852780A49B1F894122A
S315080157B00091094943A817F00BFF0A2243A94BA8F0
S315080157C0F8F71EFB50B100200DF5567DBDE8F081B6
S315080157D09800002038120020A4770308BD4E72787D
S315080157E0BD4C1346214603A817F0F2FE03A8F3F7AA
S315080157F025FA02AB024603A94BA8F8F71BFC327837
S315080158001346214603A817F0E3FE03A8F3F716FA91
S3150801581002AB024603A94BA8F8F70CFCAF4DB5F845
S31508015820EC2C1346214603A817F0D2FE03A8F3F77A
S3150801583005FA02AB024603A94BA8F8F7FBFBA84BEE
S31508015840B3F894221346214603A817F0C1FE03A80C
S31508015850F3F7F4F902AB024603A94BA8F8F7EAFBFA
S3150801586095F8EE2C9F4F1346394603A817F0B0FE5C
S3150801587003A8F3F7E3F902AB024603A94BA8F8F725
S31508015880D9FB95F8EF2C1346214603A817F0A0FE7D
S3150801589003A8F3F7D3F902AB024603A94BA8F8F715
S315080158A0C9FBD5F8F03C1A46214603A817F090FE25
S315080158B003A8F3F7C3F902AB024603A94BA8F8F705
S315080158C0B9FBD5F8F43C1A46214603A817F080FE21
S315080158D003A8F3F7B3F902AB024603A94BA8F8F7F5
S315080158E0A9FB95F8F82C1346214603A817F070FE74
S315080158F003A8F3F7A3F902AB024603A94BA8F8F7E5
S3150801590099FBB5F8602D1346214603A817F060FEEA
S3150801591003A8F3F793F902AB024603A94BA8F8F7D4
S3150801592089FB95F85C2D95F85C3D5BB252B2394618
S3150801593003A817F04DFE03A8F3F780F902AB024658
S3150801594003A94BA8F8F776FBD5F8603D1A46214618
S3150801595003A817F03DFE03A8F3F770F902AB024658
S3150801596003A94BA8F8F766FBB5F8642D134621463B
S3150801597003A817F02DFE03A8F3F760F902AB024658
S3150801598003A94BA8F8F756FBB5F8662D1346214629
S3150801599003A817F01DFE03A8F3F750F902AB024658
S315080159A003A94BA8F8F746FBB5F8682D1346214617
S315080159B003A817F00DFE03A8F3F740F902AB024658
S315080159C003A94BA8F8F736FB95F86A2D1346214625
S315080159D003A817F0FDFD03A8F3F730F902AB024659
S315080159E003A94BA8F8F726FB95F86B2D13463946FC
S315080159F003A817F0EDFD03A8F3F720F902AB024659
S31508015A0003A94BA8F8F716FB95F86C2D1346214602
S31508015A1003A817F0DDFD03A8F3F710F902AB024658
S31508015A2003A94BA8F8F706FB41F28813EA5CDFF8ED
S31508015A30BC801346414603A817F0CAFD03A8F3F72D
S31508015A40FDF802AB024603A94BA8F8F7F3FA264D6F
S31508015A5095F8F4201346414603A817F0B9FD03A8A3
S31508015A60F3F7ECF802AB024603A94BA8F8F7E2FAFA
S31508015A7095F8F4201346214603A817F0A9FD03A8B3
S31508015A80F3F7DCF802AB024603A94BA8F8F7D2FAFA
S31508015A90B5F8F620B5F8F6309BB292B2214603A8BE
S31508015AA017F096FD03A8F3F7C9F802AB024603A956
S31508015AB04BA8F8F7BFFAB5F8F8201346214603A80C
S31508015AC017F086FD03A8F3F7B9F802AB024603A956
S31508015AD04BA80DE098000020BC770308E8BB00201E
S31508015AE038120020C4770308E0CC0020CC770308DD
S31508015AF0F8F7A0FA95F8FA2095F8FA30214603A89E
S31508015B0017F066FD03A8F3F799F802AB024603A955
S31508015B104BA8F8F78FFA95F8FB2095F8FB30214644
S31508015B2003A817F055FD03A8F3F788F802AB024658
S31508015B3003A94BA8F8F77EFA95F8FC2095F8FC30EE
S31508015B40214603A817F044FD03A8F3F777F802AB3B
S31508015B50024603A94BA8F8F76DFA73681A46214657
S31508015B6003A817F035FD03A8F3F768F802AB024658
S31508015B7003A94BA8F8F75EFAD5F800311A4621466B
S31508015B8003A817F025FD03A8F3F758F802AB024658
S31508015B9003A94BA8F8F74EFAD5F804311A46214657
S31508015BA003A817F015FD03A8F3F748F802AB024658
S31508015BB003A94BA8F8F73EFA328A1346214603A8E9
S31508015BC017F006FD03A8F3F739F802AB024603A955
S31508015BD04BA8F8F72FFA328B1346214603A817F07C
S31508015BE0F7FC03A8F3F72AF802AB024603A94BA868
S31508015BF0F8F720FA95F808211346214603A817F065
S31508015C00E7FC03A8F3F71AF802AB024603A94BA867
S31508015C10F8F710FAD5F80C311A46214603A817F0F9
S31508015C20D7FC03A8F3F70AF802AB024603A94BA867
S31508015C30F8F700FA327E1346394603A817F0C8FC6E
S31508015C4003A8F2F7FBFF02AB024603A94BA8F8F734
S31508015C50F1F995F810211346214603A817F0B8FC67
S31508015C6003A8F2F7EBFF02AB024603A94BA8F8F724
S31508015C70E1F995F811211346214603A817F0A8FC66
S31508015C8003A8F2F7DBFF02AB024603A94BA8F8F714
S31508015C90D1F995F812211346214603A817F098FC65
S31508015CA003A8F2F7CBFF02AB024603A94BA8F8F704
S31508015CB0C1F995F813211346214603A817F088FC64
S31508015CC003A8F2F7BBFF02AB024603A94BA8F8F7F4
S31508015CD0B1F995F814211346214603A817F078FC63
S31508015CE003A8F2F7ABFF02AB024603A94BA8F8F7E4
S31508015CF0A1F995F815211346214603A817F068FC62
S31508015D0003A8F2F79BFF02AB024603A94BA8F8F7D3
S31508015D1091F995F81C211346394603A817F058FC42
S31508015D2003A8F2F78BFF02AB024603A94BA8F8F7C3
S31508015D3081F995F81C211346214603A817F048FC5A
S31508015D4003A8F2F77BFF02AB024603A94BA8F8F7B3
S31508015D5071F995F81D211346214603A817F038FC59
S31508015D6003A8F2F76BFF02AB024603A94BA8F8F7A3
S31508015D7061F995F81E211346214603A817F028FC58
S31508015D8003A8F2F75BFF02AB024603A94BA8F8F793
S31508015D9051F9B5F820211346214603A817F018FC36
S31508015DA003A8F2F74BFF02AB024603A94BA8F8F783
S31508015DB041F92E4695F822211346214603A817F0E4
S31508015DC007FC03A8F2F73AFF02AB024603A94BA860
S31508015DD0F8F730F9BF4D95F920201346394603A83F
S31508015DE017F0F6FB03A8F2F729FF02AB024603A94F
S31508015DF04BA8F8F71FF996F928211346394603A83F
S31508015E0017F0E6FB03A8F2F719FF02AB024603A94E
S31508015E104BA8F8F70FF92A8C1346214603A817F061
S31508015E20D7FB03A8F2F70AFF02AB024603A94BA860
S31508015E30F8F700F96A8C1346214603A817F0C8FB40
S31508015E4003A8F2F7FBFE02AB024603A94BA8F8F733
S31508015E50F1F8AA8C1346214603A817F0B9FB03A843
S31508015E60F2F7ECFE02AB024603A94BA8F8F7E2F8F3
S31508015E70EA8C1346214603A817F0AAFB03A8F2F7F2
S31508015E80DDFE02AB024603A94BA8F8F7D3F895F84D
S31508015E9028201346214603A817F09AFB03A8F2F710
S31508015EA0CDFE02AB024603A94BA8F8F7C3F895F84D
S31508015EB029201346214603A817F08AFB03A8F2F7FF
S31508015EC0BDFE02AB024603A94BA8F8F7B3F895F84D
S31508015ED02A201346214603A817F07AFB03A8F2F7EE
S31508015EE0ADFE02AB024603A94BA8F8F7A3F895F84D
S31508015EF02B201346214603A817F06AFB03A8F2F7DD
S31508015F009DFE02AB024603A94BA8F8F793F895F84C
S31508015F102C201346214603A817F05AFB03A8F2F7CB
S31508015F208DFE02AB024603A94BA8F8F783F895F84C
S31508015F302D201346214603A817F04AFB03A8F2F7BA
S31508015F407DFE02AB024603A94BA8F8F773F895F84C
S31508015F502E201346214603A817F03AFB03A8F2F7A9
S31508015F606DFE02AB024603A94BA8F8F763F895F84C
S31508015F702F201346214603A817F02AFB03A8F2F798
S31508015F805DFE02AB024603A94BA8F8F753F895F84C
S31508015F9030201346214603A817F01AFB03A8F2F787
S31508015FA04DFE02AB024603A94BA8F8F743F895F84C
S31508015FB031201346214603A817F00AFB03A8F2F776
S31508015FC03DFE02AB024603A94BA8F8F733F895F84C
S31508015FD032201346214603A817F0FAFA03A8F2F766
S31508015FE02DFE02AB024603A94BA8F8F723F895F84C
S31508015FF033201346214603A817F0EAFA03A8F2F755
S315080160001DFE02AB024603A94BA8F8F713F895F84B
S3150801601034201346214603A817F0DAFA03A8F2F743
S315080160200DFE02AB024603A94BA8F8F703F895F84B
S3150801603035201346214603A817F0CAFA03A8F2F732
S31508016040FDFD02AB024603A94BA8F7F7F3FF95F846
S3150801605036201346214603A817F0BAFA03A8F2F721
S31508016060EDFD02AB024603A94BA8F7F7E3FF95F846
S3150801607037201346214603A817F0AAFA03A8F2F710
S31508016080DDFD02AB024603A94BA8F7F7D3FFB6F825
S3150801609028211346214603A817F09AFA03A8F2F70E
S315080160A0CDFD02AB024603A94BA8F7F7C3FFB6F825
S315080160B02A211346214603A817F08AFA03A8F2F7FC
S315080160C0BDFD02AB024603A94BA8F7F7B3FFB6F825
S315080160D02C2101E0980000201346214603A817F059
S315080160E077FA03A8F2F7AAFD02AB024603A94BA861
S315080160F0F7F7A0FFB6F82E211346214603A817F095
S3150801610067FA03A8F2F79AFD02AB024603A94BA860
S31508016110F7F790FFB6F830211346214603A817F082
S3150801612057FA03A8F2F78AFD02AB024603A94BA860
S31508016130F7F780FFB6F832211346214603A817F070
S3150801614047FA03A8F2F77AFD02AB024603A94BA860
S31508016150F7F770FFB6F834211346214603A817F05E
S3150801616037FA03A8F2F76AFD02AB024603A94BA860
S31508016170F7F760FFB6F836211346214603A817F04C
S3150801618027FA03A8F2F75AFD02AB024603A94BA860
S31508016190F7F750FFB6F838211346214603A817F03A
S315080161A017FA03A8F2F74AFD02AB024603A94BA860
S315080161B0F7F740FFB6F83A211346214603A817F028
S315080161C007FA03A8F2F73AFD02AB024603A94BA860
S315080161D0F7F730FF95F838201346214603A817F03C
S315080161E0F7F903A8F2F72AFD02AB024603A94BA861
S315080161F0F7F720FF95F940201346394603A817F00B
S31508016200E7F903A8F2F71AFD02AB024603A94BA860
S31508016210F7F710FF95F840201346214603A817F013
S31508016220D7F903A8F2F70AFD02AB024603A94BA860
S31508016230F7F700FF95F841201346214603A817F002
S31508016240C7F903A8F2F7FAFC02AB024603A94BA861
S31508016250F7F7F0FE95F842201346214603A817F0F2
S31508016260B7F903A8F2F7EAFC02AB024603A94BA861
S31508016270F7F7E0FE96F83C211346214603A817F0E6
S31508016280A7F903A8F2F7DAFC02AB024603A94BA861
S31508016290F7F7D0FE95F843201346214603A817F0D1
S315080162A097F903A8F2F7CAFC02AB024603A94BA861
S315080162B0F7F7C0FE96F83D211346214603A817F0C5
S315080162C087F903A8F2F7BAFC02AB024603A94BA861
S315080162D0F7F7B0FE96F83E211346214603A817F0B4
S315080162E077F903A8F2F7AAFC02AB024603A94BA861
S315080162F0F7F7A0FE96F83F211346214603A817F0A3
S3150801630067F903A8F2F79AFC02AB024603A94BA860
S31508016310F7F790FE96F840211346214603A817F091
S3150801632057F903A8F2F78AFC02AB024603A94BA860
S31508016330F7F780FE96F841211346214603A817F080
S3150801634047F903A8F2F77AFC02AB024603A94BA860
S31508016350F7F770FE344696F942213D46134639460B
S3150801636003A817F035F903A8F2F768FC02AB024651
S3150801637003A94BA8F7F75EFE96F94321134639465A
S3150801638003A817F025F903A8F2F758FC02AB024651
S3150801639003A94BA8F7F74EFE96F944211346394649
S315080163A003A817F015F903A8F2F748FC02AB024651
S315080163B003A94BA8F7F73EFE96F945211346394638
S315080163C003A817F005F903A8F2F738FC02AB024651
S315080163D003A94BA8F7F72EFE96F946211346394627
S315080163E003A817F0F5F803A8F2F728FC02AB024652
S315080163F003A94BA8F7F71EFE96F947211346394616
S3150801640003A817F0E5F803A8F2F718FC02AB024651
S3150801641003A94BA8F7F70EFE96F948211346394604
S3150801642003A817F0D5F803A8F2F708FC02AB024651
S3150801643003A94BA8F7F7FEFD96F9492113463946F4
S3150801644003A817F0C5F803A8F2F7F8FB02AB024652
S3150801645003A94BA8F7F7EEFDC14F97F94420134658
S31508016460294603A817F0B4F803A8F2F7E7FB02AB2D
S31508016470024603A94BA8F7F7DDFD96F94A2113460B
S31508016480294603A817F0A4F803A8F2F7D7FB02AB2D
S31508016490024603A94BA8F7F7CDFD96F94B211346FA
S315080164A0294603A817F094F803A8F2F7C7FB02AB2D
S315080164B0024603A94BA8F7F7BDFD96F94C211346E9
S315080164C0294603A817F084F803A8F2F7B7FB02AB2D
S315080164D0024603A94BA8F7F7ADFD96F94D211346D8
S315080164E0294603A817F074F803A8F2F7A7FB02AB2D
S315080164F0024603A94BA8F7F79DFD96F94E211346C7
S31508016500294603A817F064F803A8F2F797FB02AB2C
S31508016510024603A94BA8F7F78DFD96F94F211346B5
S31508016520294603A817F054F803A8F2F787FB02AB2C
S31508016530024603A94BA8F7F77DFD96F950211346A4
S31508016540294603A817F044F803A8F2F777FB02AB2C
S31508016550024603A94BA8F7F76DFD96F95121134693
S31508016560294603A817F034F803A8F2F767FB02AB2C
S31508016570024603A94BA8F7F75DFD96F95221134682
S31508016580294603A817F024F803A8F2F757FB02AB2C
S31508016590024603A94BA8F7F74DFD96F95321134671
S315080165A0294603A817F014F803A8F2F747FB02AB2C
S315080165B0024603A94BA8F7F73DFD96F95421134660
S315080165C0294603A817F004F803A8F2F737FB02AB2C
S315080165D0024603A94BA8F7F72DFD96F9552113464F
S315080165E0294603A816F0F4FF03A8F2F727FB02AB26
S315080165F0024603A94BA8F7F71DFD96F9562113463E
S31508016600294603A816F0E4FF03A8F2F717FB02AB25
S31508016610024603A94BA8F7F70DFD96F9572113462C
S31508016620294603A816F0D4FF03A8F2F707FB02AB25
S31508016630024603A94BA8F7F7FDFC96F9582113461C
S31508016640294603A816F0C4FF03A8F2F7F7FA02AB26
S31508016650024603A94BA8F7F7EDFC96F9592113460B
S31508016660294603A816F0B4FF03A8F2F7E7FA02AB26
S31508016670024603A94BA8F7F7DDFC96F95A211346FA
S31508016680294603A816F0A4FF03A8F2F7D7FA02AB26
S31508016690024603A94BA8F7F7CDFCB6F85C21314EA3
S315080166A01346314603A816F093FF03A8F2F7C6FA74
S315080166B002AB024603A94BA8F7F7BCFC94F95E2185
S315080166C01346294603A816F083FF03A8F2F7B6FA7C
S315080166D002AB024603A94BA8F7F7ACFCD4F878310C
S315080166E01A46294603A816F073FF03A8F2F7A6FA75
S315080166F002AB024603A94BA8F7F79CFCD4F88831EC
S315080167001A46294603A816F063FF03A8F2F796FA74
S3150801671002AB024603A94BA8F7F78CFCD4F88031E3
S315080167201A46314603A816F053FF03A8F2F786FA6C
S3150801673002AB024603A94BA8F7F77CFCD4F88431CF
S315080167401A46314603A816F043FF03A8F2F776FA6C
S3150801675002AB024603A94BA8F7F76CFC04E000BF9D
S3150801676098000020BC77030897F845201346314660
S3150801677003A816F02DFF03A8F2F760FA02AB02464A
S3150801678003A94BA8F7F756FCD4F888311A463146BF
S3150801679003A816F01DFF03A8F2F750FA02AB02464A
S315080167A003A94BA8F7F746FCD4F88C311A463146AB
S315080167B003A816F00DFF03A8F2F740FA02AB02464A
S315080167C003A94BA8F7F736FCD4F890311A4629469F
S315080167D003A816F0FDFE03A8F2F730FA02AB02464B
S315080167E003A94BA8F7F726FCD4F894311A4629468B
S315080167F003A816F0EDFE03A8F2F720FA02AB02464B
S3150801680003A94BA8F7F716FCD4F898311A46294676
S3150801681003A816F0DDFE03A8F2F710FA02AB02464A
S3150801682003A94BA8F7F706FCD4F89C311A46294662
S3150801683003A816F0CDFE03A8F2F700FA02AB02464A
S3150801684003A94BA8F7F7F6FBD4F8A0311A4629464F
S3150801685003A816F0BDFE03A8F2F7F0F902AB02464B
S3150801686003A94BA8F7F7E6FBB7F9462013462946CD
S3150801687003A816F0ADFE03A8F2F7E0F902AB02464B
S3150801688003A94BA8F7F7D6FB94F9A4211346294681
S3150801689003A816F09DFE03A8F2F7D0F902AB02464B
S315080168A003A94BA8F7F7C6FB97F9482013462946CB
S315080168B003A816F08DFE03A8F2F7C0F902AB02464B
S315080168C003A94BA8F7F7B6FB94F9A5211346294660
S315080168D003A816F07DFE03A8F2F7B0F902AB02464B
S315080168E003A94BA8F7F7A6FB94F9A621134629464F
S315080168F003A816F06DFE03A8F2F7A0F902AB02464B
S3150801690003A94BA8F7F796FB94F9A721134629463D
S3150801691003A816F05DFE03A8F2F790F902AB02464A
S3150801692003A94BA8F7F786FB97F949201346294689
S3150801693003A816F04DFE03A8F2F780F902AB02464A
S3150801694003A94BA8F7F776FB94F9A821134629461C
S3150801695003A816F03DFE03A8F2F770F902AB02464A
S3150801696003A94BA8F7F766FB94F9A921134629460B
S3150801697003A816F02DFE03A8F2F760F902AB02464A
S3150801698003A94BA8F7F756FB97F94A201346294658
S3150801699003A816F01DFE03A8F2F750F902AB02464A
S315080169A003A94BA8F7F746FB97F84B20C14E1346A8
S315080169B0314603A816F00CFE03A8F2F73FF902AB1D
S315080169C0024603A94BA8F7F735FB94F8AA21134603
S315080169D0314603A816F0FCFD03A8F2F72FF902AB1E
S315080169E0024603A94BA8F7F725FB94F8AB211346F2
S315080169F0314603A816F0ECFD03A8F2F71FF902AB1E
S31508016A00024603A94BA8F7F715FBD4F8AC311A4689
S31508016A10294603A816F0DCFD03A8F2F70FF902AB25
S31508016A20024603A94BA8F7F705FB94F8B0211346CC
S31508016A30314603A816F0CCFD03A8F2F7FFF802AB1E
S31508016A40024603A94BA8F7F7F5FA94F8B1211346BC
S31508016A50294603A816F0BCFD03A8F2F7EFF802AB26
S31508016A60024603A94BA8F7F7E5FA94F8B2211346AB
S31508016A70294603A816F0ACFD03A8F2F7DFF802AB26
S31508016A80024603A94BA8F7F7D5FA94F8B32113469A
S31508016A90294603A816F09CFD03A8F2F7CFF802AB26
S31508016AA0024603A94BA8F7F7C5FA94F8B421134689
S31508016AB0294603A816F08CFD03A8F2F7BFF802AB26
S31508016AC0024603A94BA8F7F7B5FA94F8B521134678
S31508016AD0294603A816F07CFD03A8F2F7AFF802AB26
S31508016AE0024603A94BA8F7F7A5FA94F8B621134667
S31508016AF0294603A816F06CFD03A8F2F79FF802AB26
S31508016B00024603A94BA8F7F795FA94F8B721134655
S31508016B10294603A816F05CFD03A8F2F78FF802AB25
S31508016B20024603A94BA8F7F785FA94F8B821134644
S31508016B30294603A816F04CFD03A8F2F77FF802AB25
S31508016B40024603A94BA8F7F775FA94F8B921134633
S31508016B50314603A816F03CFD03A8F2F76FF802AB1D
S31508016B60024603A94BA8F7F765FA94F8BA21134622
S31508016B70294603A816F02CFD03A8F2F75FF802AB25
S31508016B80024603A94BA8F7F755FA94F8BB21134611
S31508016B90294603A816F01CFD03A8F2F74FF802AB25
S31508016BA0024603A94BA8F7F745FA94F8BC21134600
S31508016BB0314603A816F00CFD03A8F2F73FF802AB1D
S31508016BC0024603A94BA8F7F735FAD4F8C0311A4695
S31508016BD0314603A816F0FCFC03A8F2F72FF802AB1E
S31508016BE0024603A94BA8F7F725FAD4F8C4311A4681
S31508016BF0314603A816F0ECFC03A8F2F71FF802AB1E
S31508016C00024603A94BA8F7F715FA94F8C8211346C3
S31508016C10294603A816F0DCFC03A8F2F70FF802AB25
S31508016C20024603A94BA8F7F705FAD4F8DC311A4648
S31508016C30294603A816F0CCFC03A8F1F7FFFF02AB1F
S31508016C40024603A94BA8F7F7F5F9D4F8EC311A4629
S31508016C50294603A816F0BCFC03A8F1F7EFFF02AB1F
S31508016C60024603A94BA8F7F7E5F994F8EC21134670
S31508016C70314603A816F0ACFC03A8F1F7DFFF02AB17
S31508016C80024603A94BA8F7F7D5F994F8ED2113465F
S31508016C90314603A816F09CFC03A8F1F7CFFF02AB17
S31508016CA0024603A94BA8F7F7C5F994F9EE2113464D
S31508016CB0294601E0BC77030803A816F089FC03A856
S31508016CC0F1F7BCFF02AB024603A94BA8F7F7B2F9E5
S31508016CD0D4F8F0311A46294603A816F079FC03A818
S31508016CE0F1F7ACFF02AB024603A94BA8F7F7A2F9E5
S31508016CF0D4F8F421D4F8F431294603A816F068FC2F
S31508016D0003A8F1F79BFF02AB024603A94BA8F7F7C5
S31508016D1091F9D4F8F821D4F8F831294603A816F0E0
S31508016D2057FC03A8F1F78AFF02AB024603A94BA851
S31508016D30F7F780F994F8FC211346314603A816F0B3
S31508016D4047FC03A8F1F77AFF02AB024603A94BA851
S31508016D50F7F770F9B4F80C221346314603A816F072
S31508016D6037FC03A8F1F76AFF02AB024603A94BA851
S31508016D70F7F760F994F80C221346314603A816F082
S31508016D8027FC03A8F1F75AFF02AB024603A94BA851
S31508016D90F7F750F9D4F820321A46294603A816F00F
S31508016DA017FC03A8F1F74AFF02AB024603A94BA851
S31508016DB0F7F740F994F820221346294603A816F056
S31508016DC007FC03A8F1F73AFF02AB024603A94BA851
S31508016DD0F7F730F994F821221346294603A816F045
S31508016DE0F7FB03A8F1F72AFF02AB024603A94BA852
S31508016DF0F7F720F994F822221346294603A816F034
S31508016E00E7FB03A8F1F71AFF02AB024603A94BA851
S31508016E10F7F710F994F823221346294603A816F022
S31508016E20D7FB03A8F1F70AFF02AB024603A94BA851
S31508016E30F7F700F994F824221346294603A816F011
S31508016E40C7FB03A8F1F7FAFE02AB024603A94BA852
S31508016E50F7F7F0F894F825221346294603A816F001
S31508016E60B7FB03A8F1F7EAFE02AB024603A94BA852
S31508016E70F7F7E0F894F826221346294603A816F0F0
S31508016E80A7FB03A8F1F7DAFE02AB024603A94BA852
S31508016E90F7F7D0F8D4F828321A46314603A816F07F
S31508016EA097FB03A8F1F7CAFE02AB024603A94BA852
S31508016EB0F7F7C0F8D4F82C221346314603A816F082
S31508016EC087FB03A8F1F7BAFE02AB024603A94BA852
S31508016ED0F7F7B0F83E46B7F94C202C461346294633
S31508016EE003A816F075FB03A8F1F7A8FE02AB024644
S31508016EF003A94BA8F7F79EF8BE4D95F83022BE4F69
S31508016F001346394603A816F063FB03A8F1F796FE64
S31508016F1002AB024603A94BA8F7F78CF895F931227B
S31508016F201346214603A816F053FB03A8F1F786FE7C
S31508016F3002AB024603A94BA8F7F77CF8B5F832224B
S31508016F401346394603A816F043FB03A8F1F776FE64
S31508016F5002AB024603A94BA8F7F76CF8D5F8343209
S31508016F601A46394603A816F033FB03A8F1F766FE5D
S31508016F7002AB024603A94BA8F7F75CF8306DF1F7A7
S31508016F80C1FA02460B469D4903A816F021FB03A840
S31508016F90F1F754FE02AB024603A94BA8F7F74AF8E4
S31508016FA0736D1A46214603A816F012FB03A8F1F7DA
S31508016FB045FE02AB024603A94BA8F7F73BF8B5F91C
S31508016FC038221346214603A816F002FB03A8F1F757
S31508016FD035FE02AB024603A94BA8F7F72BF8B5F91C
S31508016FE03A221346214603A816F0F2FA03A8F1F746
S31508016FF025FE02AB024603A94BA8F7F71BF8B36DAA
S315080170001A46214603A816F0E3FA03A8F1F716FE75
S3150801701002AB024603A94BA8F7F70CF8D5F83C32A0
S315080170201A46394603A816F0D3FA03A8F1F706FE5D
S3150801703002AB024603A94BA8F6F7FCFFD5F8403286
S315080170401A46214603A816F0C3FA03A8F1F7F6FD76
S3150801705002AB024603A94BA8F6F7ECFFD5F8443272
S315080170601A46214603A816F0B3FA03A8F1F7E6FD76
S3150801707002AB024603A94BA8F6F7DCFFF36D1A46E5
S31508017080214603A816F0A4FA03A8F1F7D7FD02AB27
S31508017090024603A94BA8F6F7CDFFDFF86481D8F8B5
S315080170A098321A46214603A816F092FA03A8F1F770
S315080170B0C5FD02AB024603A94BA8F6F7BBFF336E23
S315080170C01A46214603A816F083FA03A8F1F7B6FD76
S315080170D002AB024603A94BA8F6F7ACFFB6F8642043
S315080170E01346394603A816F073FA03A8F1F7A6FD65
S315080170F002AB024603A94BA8F6F79CFFB36E1A46E4
S31508017100214603A816F064FA03A8F1F797FD02AB26
S31508017110024603A94BA8F6F78DFFB6F96C2013466C
S31508017120214603A816F054FA03A8F1F787FD02AB26
S31508017130024603A94BA8F6F77DFFB5F9482213467F
S31508017140214603A816F044FA03A8F1F777FD02AB26
S31508017150024603A94BA8F6F76DFFB5F94A2213466D
S31508017160214603A816F034FA03A8F1F767FD02AB26
S31508017170024603A94BA8F6F75DFFD5F89C321A46D5
S31508017180214603A816F024FA03A8F1F757FD02AB26
S31508017190024603A94BA8F6F74DFFB6F97820134620
S315080171A0214603A816F014FA03A8F1F747FD02AB26
S315080171B0024603A94BA8F6F73DFFB6F98020134608
S315080171C0214603A816F004FA03A8F1F737FD02AB26
S315080171D0024603A94BA8F6F72DFF95F99022134607
S315080171E0214603A816F0F4F903A8F1F727FD02AB27
S315080171F0024607E0E0CC0020BC770308D4770308F1
S315080172003812002003A94BA8F6F714FFB6F8802018
S315080172101346394603A816F0DBF903A8F1F70EFD64
S3150801722002AB024603A94BA8F6F704FFB6F88C2071
S315080172301346394603A816F0CBF903A8F1F7FEFC65
S3150801724002AB024603A94BA8F6F7F4FE96F98C2081
S315080172501346214603A816F0BBF903A8F1F7EEFC7D
S3150801726002AB024603A94BA8F6F7E4FEB6F8B0202E
S315080172701346394603A816F0ABF903A8F1F7DEFC65
S3150801728002AB024603A94BA8F6F7D4FE96F9B0203D
S315080172901346214603A816F09BF903A8F1F7CEFC7D
S315080172A002AB024603A94BA8F6F7C4FEB6F8B2200C
S315080172B01346394603A816F08BF903A8F1F7BEFC65
S315080172C002AB024603A94BA8F6F7B4FED6F8B430CA
S315080172D01A46214603A816F07BF903A8F1F7AEFC76
S315080172E002AB024603A94BA8F6F7A4FE4BF2AC6320
S315080172F058F803201346214603A816F069F903A88E
S31508017300F1F79CFC02AB024603A94BA8F6F792FEDD
S31508017310D5F898321A46394603A816F059F903A83A
S31508017320F1F78CFC02AB024603A94BA8F6F782FEDD
S3150801733095F898221346394603A816F049F903A881
S31508017340F1F77CFC02AB024603A94BA8F6F772FEDD
S31508017350D5F89C321A46394603A816F039F903A816
S31508017360F1F76CFC02AB024603A94BA8F6F762FEDD
S31508017370D5F8A0321A46394603A816F029F903A802
S31508017380F1F75CFC02AB024603A94BA8F6F752FEDD
S31508017390D5F8A4321A46394603A816F019F903A8EE
S315080173A0F1F74CFC02AB024603A94BA8F6F742FEDD
S315080173B0D5F8A8321A46394603A816F009F903A8DA
S315080173C0F1F73CFC02AB024603A94BA8F6F732FEDD
S315080173D095F8AC221346214603A816F0F9F803A836
S315080173E0F1F72CFC02AB024603A94BA8F6F722FEDD
S315080173F0D5F8B0321A46394603A816F0E9F803A8B3
S31508017400F1F71CFC02AB024603A94BA8F6F712FEDC
S31508017410D5F8B4321A46214603A816F0D9F803A8B6
S31508017420F1F70CFC02AB024603A94BA8F6F702FEDC
S31508017430D5F8B8321A46214603A816F0C9F803A8A2
S31508017440F1F7FCFB02AB024603A94BA8F6F7F2FDDE
S31508017450D5F85C231346214603A816F0B9F803A804
S31508017460F1F7ECFB02AB024603A94BA8F6F7E2FDDE
S3150801747096F9B8201346214603A816F0A9F803A8D9
S31508017480F1F7DCFB02AB024603A94BA8F6F7D2FDDE
S3150801749096F9B9201346214603A816F099F803A8C8
S315080174A0F1F7CCFB02AB024603A94BA8F6F7C2FDDE
S315080174B0B5F862231346394603A816F089F803A8D6
S315080174C0F1F7BCFB02AB024603A94BA8F6F7B2FDDE
S315080174D095F862231346394603A816F079F803A8E6
S315080174E0F1F7ACFB02AB024603A94BA8F6F7A2FDDE
S315080174F04BA8F6F713FF0446B8F894320133A8F8F7
S315080175009432022208F525710520FDF783FBB4FAAA
S3150801751084F04009FEF758B970B596B005460C4691
S315080175204F263246002102A815F049FF52238DF84D
S31508017530083011238DF8093080238DF80A30FF238E
S315080175408DF80C3063788DF80F3023788DF810306C
S31508017550A3788DF81130E3788DF8123023798DF8F8
S31508017560133063798DF81430A3798DF8153000231B
S31508017570E371A989A868EB7D0193AB7D0093334636
S3150801758002AAF2F747FB16B070BDA0F12C00C3E7BB
S3150801759008B52C30F3F772FB08BD10B47F2380F8C9
S315080175A0303080F8313080F8323080F83330416B32
S315080175B06FF317014163C26E6FF31702C2660023A8
S315080175C080F8373080F8383090F8524044F080041B
S315080175D080F8524090F8564044F0800480F85640AE
S315080175E090F85B4044F0800480F85B4090F85F4077
S315080175F044F0800480F85F4090F8644044F08004C9
S3150801760080F8644090F8684044F0800480F8684047
S31508017610082464F3030180F83410114664F3030166
S3150801762080F86C10120E63F3030280F86F2080F85D
S315080176307A3080F8733080F8723080F8763080F8C6
S31508017640753080F8743080F8783080F8773080F8B3
S3150801765079305DF8044B704710B584B004467F2332
S3150801766080F8303080F8313080F8323080F83330A5
S31508017670416B6FF317014163C26E6FF31702C2665E
S31508017680002380F8373080F8383090F8520040F0FF
S31508017690800084F8520094F8560040F0800084F87F
S315080176A0560094F85B0040F0800084F85B0094F87B
S315080176B05F0040F0800084F85F0094F8640040F0B1
S315080176C0800084F8640094F8680040F0800084F82B
S315080176D06800082060F3030184F83410114660F34A
S315080176E0030184F86C10120E63F3030284F86F2009
S315080176F084F87A3084F8733084F8723084F87630F6
S3150801770084F8753084F8743084F8783084F87730E2
S3150801771084F8793043238DF80C3002238DF80D3027
S31508017720A189E27D0192A27D009203AAA068F2F7DF
S3150801773071FA636813B1984704B010BD002384F841
S31508017740743084F87530142384F87630012384F86C
S315080177507930F1E770B586B0634B93F9543143B18B
S31508017760012B30D0022B60D0032B00F0908006B09D
S3150801777070BD5E4A536C23F0100353645C4C4FF49E
S31508017780C0612046F8F70CF92520F7F7B3FD4FF449
S31508017790C0630193574B02930123039301A9204622
S315080177A0F8F720F8002206211720F7F767FD1720BA
S315080177B0F7F794FD002207212820F7F75FFD282017
S315080177C0F7F78CFDD3E74FF4C0614948F8F7E8F8B5
S315080177D01720F7F78FFD2820F7F78CFD4248464B0F
S315080177E0C0F864334FF46143C0F868330023C0F826
S315080177F06C33C0F87033C0F874330C22C0F87823A0
S31508017800C0F87C33C0F8803300F55970FBF74EFB9E
S3150801781050B93548D0F864335B680122374900F519
S315080178205970FBF797FCA2E7FEE74FF4C0613048B1
S31508017830F8F7B6F81720F7F75DFD2820F7F75AFD90
S3150801784029482D4BC0F864334FF4E133C0F8683347
S315080178500023C0F86C33C0F87033C0F874330C22B7
S31508017860C0F87823C0F87C33C0F8803300F5597026
S31508017870FBF71CFB50B91C48D0F864335B6801223E
S315080178801E4900F55970FBF765FC70E7FEE7174AD4
S31508017890536C23F010035364154D4FF4C061284609
S315080178A0F8F77EF81720F7F725FD2820F7F722FDC8
S315080178B04FF48066019601230293002403940494ED
S315080178C001A92846F7F78EFF4FF400730193029436
S315080178D00394049401A92846F7F784FF2246314602
S315080178E02846F8F7FBF842E7E0CC002000380240CA
S315080178F000000240000031100010014054C9002068
S3150801790000B5ADB0002101913C4B1A6C42F0805292
S315080179101A641B6C03F0805301930291384B1A6861
S3150801792042F440421A601B6803F44043029305235C
S315080179301F93012320932193022325934FF4800259
S315080179402692102227924FF4B4722892299308227C
S315080179502A922B931FA8F9F7EDF9002849D1F8F7D0
S3150801796023FD002846D10F231A9302231B930023D4
S315080179701C934FF4A0531D934FF480531E93052176
S315080179801AA8F8F7AFFD002835D14FF448730393C9
S31508017990102309934FF4C0730A9302230C93082307
S315080179A00B9301230E934FF4807313934FF00063E7
S315080179B018930023149303A8F8F7A2FEE0B900224E
S315080179C04FF480011046F8F73FFDF8F763FE0D4BBB
S315080179D0A3FB00308009F7F79BFC0420F7F7BCFCF2
S315080179E0002211464FF0FF30F7F748FC2DB05DF83D
S315080179F004FBFEE7FEE7FEE7FEE700BF00380240AC
S31508017A0000700040D34D6210F8B51D4CB4F8D4137C
S31508017A1004F5697749003846FDF7BDF9B4F8181435
S31508017A2004F57A7649003046FDF7B5F9B4F85C04F1
S31508017A30F0F756FD0022134BF0F7B8FDF1F78EF873
S31508017A4004F22C4501462846FDF7A5F9B4F8A01419
S31508017A5004F58E6449002046FDF79DF90021384654
S31508017A60FDF76EF900213046FDF76AF9002128462F
S31508017A70FDF766F900212046FDF762F9F8BD00BF5A
S31508017A80E0CC00200000F83F2DE9F04788B000233C
S31508017A9006938DF81C3021228DF8182004938DF851
S31508017AA014306F238DF81030344C0126344D4FF0C5
S31508017AB00008DFF8D09009F2B4470CE0314A82F8A1
S31508017AC0A613C2F8A83308B0BDE8F08789F8EA1307
S31508017AD0C9F8EC330136A246424621882846F7F70B
S31508017AE0FDFF4FF47A73052206A93846FAF715FC05
S31508017AF0012221882846F7F7F1FF424634F8021B8E
S31508017B002846F7F7EBFF4FF47A730093052302AA89
S31508017B1004A93846FAF7D0FC0122BAF8001028461B
S31508017B20F7F7DCFF9DF808109DF809209DF80A3043
S31508017B301B0443EA02639DF80C2013439DF80B20AE
S31508017B4043EA0223721E032A14D801A050F822F030
S31508017B506B7B0108617B0108CD7A0108BD7A0108B2
S31508017B6089F82E14C9F83034B4E789F87214C9F8BB
S31508017B707434AFE7032EADDDA5E700BFA0000020F2
S31508017B80000C0240E0CC00202DE9F04F89B000231B
S31508017B9006938DF81C3022228DF8182004938DF84F
S31508017BA014306F238DF810303D4C04F1080A254630
S31508017BB03C4E4FF00009DFF8F4802F464A4635F867
S31508017BC0021B3046F7F78AFF4FF47A73052206A996
S31508017BD04046FAF7A2FB012239883046F7F77EFFBD
S31508017BE05545EAD101252F4F4FF0000ADFF8B88035
S31508017BF008F2B4490CE02C4A82F8A613C2F8B43349
S31508017C0009B0BDE8F08F88F8EA13C8F8F8330135EA
S31508017C106E1EA346524634F8021B3846F7F75EFF36
S31508017C204FF47A730093052302AA04A94846FAF782
S31508017C3043FC0122BBF800103846F7F74FFF9DF8C1
S31508017C4008109DF809209DF80A301B0443EA0263CF
S31508017C509DF80C2013439DF80B2043EA0223B3F544
S31508017C60000FC8BF03F17F43032E15D801A252F8AE
S31508017C7026F000BF8F7C0108857C0108077C010876
S31508017C80F77B010888F82E14C8F83C34BFE788F852
S31508017C907214C8F88034BAE7032DB8DDB0E700BF1F
S31508017CA0A0000020000C0240E0CC002094D1002066
S31508017CB070B5FFF769FF4FF400717948F7F708FFC8
S31508017CC0002866D1774B5D686D424FF400517448C0
S31508017CD0F7F7FEFE00286BD1724B5D684FF48041C1
S31508017CE06F48F7F7F5FE002871D16E4B5C684FF4C3
S31508017CF000616B48F7F7ECFE002877D1694B5C68A1
S31508017D006442694B93F92431012B00F0AE80664B2E
S31508017D1093F92531012B08BF0024644E4FF47A717B
S31508017D203046FDF738F885EAE571A1EBE57130468D
S31508017D30FDF706F8002D00F0A780002D0ADD5A4B45
S31508017D40D3F8B813D3F8BC339942D8BF1946574864
S31508017D50FCF7E6FF002D59DB554D4FF47A7128469D
S31508017D60FDF719F884EAE471A1EBE4712846FCF7FA
S31508017D70E7FF002C58D0002C5FDD4B4BD3F8FC13E2
S31508017D80D3F800349942D8BF19464948FCF7C8FFC9
S31508017D9070BD4FF480714248F7F79AFE002891D0DA
S31508017DA080213F48F7F794FE002500288DD189E701
S31508017DB04FF480513A48F7F78BFE00288CD04FF4E0
S31508017DC000613748F7F784FE002887D184E74FF426
S31508017DD000513348F7F77CFE002886D080213048C9
S31508017DE0F7F776FE0024002881D17EE74FF48061FB
S31508017DF02B48F7F76DFE002880D04FF4007128480C
S31508017E00F7F766FE00287FF47CAF77E7264BD3F8B1
S31508017E10B823D3F8BC138A42CEBF03F5697011465D
S31508017E202248FCF77DFF97E74FF4FA612846FCF7ED
S31508017E30B2FF00212846FCF783FF1B4BD3F8FC133E
S31508017E40D3F800349942C8BF19461948FCF768FFA8
S31508017E5070BD164C4FF47A712046FCF79CFF002141
S31508017E602046FCF76DFF00240EE00F4B93F92531F0
S31508017E70012BEED00D4D4FF47A712846FCF78BFF96
S31508017E8000212846FCF75CFF084D4FF4FA612846A5
S31508017E90FCF781FF00212846FCF752FF5CE700BF8B
S31508017EA00010024098000020E0CC002084D0002079
S31508017EB0C8D0002070B5FFF767FE4FF400718648F9
S31508017EC0F7F706FE002874D1844BD3F860546D4247
S31508017ED04FF400518048F7F7FBFD002878D17F4B16
S31508017EE0D3F860544FF480417B48F7F7F1FD002839
S31508017EF07FD17A4BD3F8A4444FF400617648F7F75B
S31508017F00E7FD002840F08680744BD3F8A444644208
S31508017F10724B93F92631012B00F0C0806F4B93F910
S31508017F202731012B08BF00246C4B03F22C46B3F80A
S31508017F305C143046FCF72FFF85EAE571A1EBE57184
S31508017F403046FCF7FDFE002D00F0B980002D0ADD54
S31508017F50624BD3F84014D3F844349942D8BF194632
S31508017F605F48FCF7DDFE002D65DB5C4B03F58E658E
S31508017F70B3F8A0142846FCF70EFF84EAE471A1EBD6
S31508017F80E4712846FCF7DCFE41F288312846FCF705
S31508017F90EDFE002C5DD0002C66DD504BD3F8841421
S31508017FA0D3F888349942D8BF19464E48FCF7B8FE2B
S31508017FB070BD4FF480714848F7F78AFD002883D0D1
S31508017FC080214548F7F784FD0025002880D17BE705
S31508017FD04FF480514048F7F77BFD00283FF47FAF07
S31508017FE04FF400613C48F7F773FD00287FF47AAF38
S31508017FF075E74FF400513848F7F76AFD00283FF452
S3150801800078AF80213448F7F763FD002400287FF410
S3150801801073AF6EE74FF480612F48F7F759FD0028D3
S315080180203FF472AF4FF400712B48F7F751FD002862
S315080180307FF46EAF68E7294BD3F84024D3F844148C
S315080180408A42CEBF03F22C4011462548FCF768FE4A
S315080180508BE7A5F58E63B3F8A0142846FCF79BFEBB
S3150801806000212846FCF76CFE1C4BD3F88414D3F880
S3150801807088349942C8BF19461A48FCF751FE70BDA3
S31508018080164B03F22C44B3F85C142046FCF783FE26
S3150801809000212046FCF754FE002410E00F4B93F90B
S315080180A02731012BECD00D4B03F22C45B3F85C14A8
S315080180B02846FCF770FE00212846FCF741FE074BCF
S315080180C003F22C45B3F85C142846FCF764FE00213C
S315080180D02846FCF735FE48E700100240E0CC0020B0
S315080180E00CD1002050D1002008B54FF480417048CA
S315080180F0F7F7EEFCD0B96F4AB2F8283101339BB2D3
S31508018100A2F8283101216C4A82F8381040F2E1427E
S3150801811093423FDD13F0070F3CD11022654B83F8DC
S315080181203F213222644B83F8382009E00021634855
S31508018130F2F76EFD0028DED100225E4BA3F8282156
S315080181404FF480615A48F7F7C3FC00284FD1594AC2
S31508018150B2F82A3101339BB2A2F82A310121564AD3
S3150801816082F8381040F2E242934268DD544AA2FB93
S315080181700312D20802EB8202A3EB420292B2002A50
S315080181805DD112224B4B83F83F2132224A4B83F8A9
S31508018190382036E040F2ED22934211DD494AA2FB2E
S315080181A00312D208C2EB02129A1A92B242B91022EB
S315080181B0404B83F83F2114223F4B83F83820BFE711
S315080181C0F92BBDDD404AA2FB0312D20802EB82025B
S315080181D002EB82029B1A9BB2002BB1D11022354BBE
S315080181E083F83F210522344B83F83820A8E702217A
S315080181F03248F2F70DFD0028A9D100222D4BA3F82C
S315080182002A214FF400412A48F7F762FC002843D196
S31508018210284AB2F8323101339BB2A2F83231FA2B2D
S3150801822044DD2A4A82FB03121211FA2101FB123399
S31508018230012B3BD10F221F4B83F83F2108BD40F28A
S31508018240EE22934211DD1F4AA2FB0312D208C2EBAA
S3150801825002129A1A92B242B91222164B83F83F2198
S315080182601422154B83F83820CBE7FA2BC9DD164AB9
S31508018270A2FB0312D20802EB820202EB82029B1ACC
S315080182809BB2002BBDD112220A4B83F83F2105224E
S31508018290094B83F83820B4E70E210848F2F7B8FCF1
S315080182A00028B5D10022034BA3F8322108BD00BF2F
S315080182B000100240E0CC00209800002018D20020CF
S315080182C0CDCCCCCC898888881F85EB51D34D6210DB
S315080182D010B510211348F2F79BFCF0B1124AB2F817
S315080182E0383101339BB2A2F83831FA2B19DD0F4A1E
S315080182F082FB03121211FA2101FB1233012B10D151
S31508018300094B93F8213563B1074C04F20C50F2F787
S3150801831050F90023A4F8383110BD0022024BA3F806
S31508018320382110BD18D20020E0CC0020D34D6210B0
S3150801833070B52DED048BF0EE408A4F48D0F86034C5
S3150801834007EE903AF8EE677A87EE809A002100F5F3
S31508018350A760F2F790FC494B93F91E30022B04D023
S31508018360032B05D023B1803803E0C0F1800000E07B
S315080183700020414B93F92631012B25D000F10D033D
S315080183801A2B68D9002820DA07EE900AB8EEE78A90
S31508018390F1EE497A17EE900AF0F7B4F80022384B55
S315080183A0F0F704F904460D4668EE087A17EE900AC6
S315080183B0F0F7A8F802460B4620462946F0F7F6F8E4
S315080183C0F0F7A4FB04461DE0002007EE900AF8EE3C
S315080183D0E77A67EEA77A17EE900AF0F793F804465C
S315080183E00D4619EE100AF0F78DF80022244BF0F726
S315080183F0DDF802460B4620462946F0F7D7F8F0F78E
S3150801840085FB04461C4E06F22C4584EAE471A1EB71
S31508018410E4712846FCF794FCB6F85C3407EE903A0A
S31508018420F8EEE77A87EEA87AFCEEC77A17EE901A85
S315080184302846FCF7B0FC002C0FDDD6F84014D6F818
S3150801844044349942CEBF284619460E48FCF768FCC3
S31508018450BDEC048B70BD0020B7E7002CF8DA064B9B
S31508018460D3F84014D3F844349942C8BF194605488D
S31508018470FCF756FCECE700BFE0CC00209800002092
S315080184800000103F0CD10020F8B52DED028BB0EE9F
S31508018490608A854DD5F8A43407EE903AF8EE677AE6
S315080184A0C7EE808A05F5A76509212846F2F7DAFBA2
S315080184B0044608212846F2F7D5FB221A7B4B93F985
S315080184C01F30022B3CD0032B00D003B90022764B78
S315080184D093F92731012B35D082EAE273A3EBE273D4
S315080184E0002BC0F28780002A2DDA82EAE270A0EB1F
S315080184F0E270EFF7F5FF9FED681B41EC100B13F0E7
S31508018500D3FB57EC106BF1EE687A17EE900AEFF78A
S31508018510F9FF63A3D3E90023F0F772F904460D4680
S3150801852030463946F0F73AFBEFF7ECFF02460B46C1
S3150801853020462946F0F73AF8F0F7E8FA06462AE01F
S315080185405242C4E7002282EAE270A0EBE270EFF73A
S31508018550C7FF9FED511B41EC100B13F0A5FB57EC20
S31508018560106B18EE900AEFF7CDFF4DA3D3E9002360
S31508018570F0F746F904460D4630463946F0F70EFB44
S31508018580EFF7C0FF02460B4620462946F0F70EF8DC
S31508018590F0F7BCFA0646444D05F58E6486EAE6719F
S315080185A0A1EBE6712046FCF7CBFBB5F8A03407EE44
S315080185B0903AF8EEE77A87EE887AFCEEC77A17EEF4
S315080185C0901A2046FCF7E7FB002E33DB2B46D5F83D
S315080185D08454D3F88844A54218DD1C46294603F578
S315080185E08E60FCF79DFBD4F874349D4204D0BDEC33
S315080185F0028BF8BD0022A6E7802284F87E25002298
S3150801860084F87F25012284F88525F0E7264D214641
S3150801861005F58E60FCF784FBD5F874349C42E6D1E7
S31508018620802285F87E25002285F87F25012285F896
S315080186308525DCE71C4BD3F88444D3F88854AC422F
S3150801864013DD1C46294603F58E60FCF769FBD4F851
S3150801865074349D42CBD1802284F87E25002284F889
S315080186607F25012284F88525C1E70F4D214605F5A9
S315080186708E60FCF755FBD5F874349C42B7D180223D
S3150801868085F87E25002285F87F25012285F885252E
S31508018690ADE700BFAFF30080333333333333F33FF2
S315080186A044BEA9E048238840E0CC00209800002079
S315080186B0F8B52DED048BB0EE409AF0EE608AD548F8
S315080186C0D0EDF67AF8EE677AC7EE809A022100F5C0
S315080186D0A760F2F7D0FAD04B93F91C30022B65D07C
S315080186E0032B66D0002B64D0803800F10D031A2BBA
S315080186F098BF002080EAE074A4EBE074E4B2C54BAD
S3150801870093F92431012B56D0002856DB07EE900A3F
S31508018710F8EEE77A67EEA77A17EE900AEFF7F2FE18
S3150801872006460F4619EE900AEFF7ECFE0022BB4B00
S31508018730EFF73CFF02460B4630463946EFF736FF60
S31508018740F0F7E4F9054685EAE571A1EBE571B44868
S31508018750FCF7F6FA002D63DDAE48D0F8B863D0F819
S31508018760BC53B0F8D43307EE903AF8EEE77A87EEC1
S31508018770897AFCEEC77A17EE901A00F56970FCF74C
S315080187800AFBAE4239DDA34D314605F56970FCF7A2
S31508018790C7FAD5F8A8339E4244D185F87E4500220A
S315080187A085F87F25012285F885253BE0C0F1800003
S315080187B09BE700209EE70020A8E707EE900AB8EE9F
S315080187C0E78AF1EE697A17EE900AEFF79BFE002227
S315080187D0924BEFF7EBFE06460F4668EE087A17EE60
S315080187E0900AEFF78FFE02460B4630463946EFF7F9
S315080187F0DDFEF0F78BF90546A5E7864E294606F50F
S315080188006970FCF78DFAD6F8A8339D420AD186F825
S315080188107E45002286F87F25012286F8852501E016
S31508018820002D18DB7B48D0F81C3407EE903AF8EE99
S31508018830677A87EEA89A032100F5A760F2F71BFA73
S31508018840754B93F91D30022B42D0032B43D0002BD5
S3150801885041D0823840E06F48D0F8B853D0F8BC63AD
S31508018860B0F8D43307EE903AF8EEE77A87EE897ACC
S31508018870FCEEC77A17EE901A00F56970FCF78BFAC9
S31508018880B54212DD634D314605F56970FCF748FAC4
S31508018890D5F8A8339E42C5D185F87E45002285F8CC
S315080188A07F25012285F88525BCE75A4E294606F516
S315080188B06970FCF735FAD6F8A8339D42B2D186F825
S315080188C07E45002286F87F25012286F88525A9E7B7
S315080188D0C0F1820000E000204E4B93F92531012BAF
S315080188E02AD000F10D031A2B72D980EAE075A5EB9F
S315080188F0E075EDB2002821DA07EE900AB8EEE78AAC
S31508018900F1EE497A17EE900AEFF7FCFD0022434B88
S31508018910EFF74CFE06460F4668EE087A17EE900A00
S31508018920EFF7F0FD02460B4630463946EFF73EFEB5
S31508018930F0F7ECF806461EE00025284607EE900AF1
S31508018940F8EEE77A67EEA77A17EE900AEFF7DAFDFF
S3150801895006460F4619EE100AEFF7D4FD00222F4BF3
S31508018960EFF724FE02460B4630463946EFF71EFE60
S31508018970F0F7CCF8064686EAE671A1EBE6712948D6
S31508018980FCF7DEF9002E4FDB2248D0F8FC73D0F84D
S315080189900064B0F8183407EE903AF8EEE77A87EEF5
S315080189A0A87AFCEEC77A17EE901A00F57A70FCF7EA
S315080189B0F2F9B74219DD174E394606F57A70FCF712
S315080189C0AFF9D6F8EC339F4205D0BDEC048BF8BD60
S315080189D000252846B2E72C4486F87E45002286F80B
